:100000000C94891A0C94BA1A0C94BA1A0C94BA1A51
:100010000C94BA1A0C94BA1A0C94BA1A0C94BA1A10
:100020000C94BA1A0C94BA1A0C94BA1A0C94BA1A00
:100030000C94BA1A0C94BA1A0C94BA1A0C94BA1AF0
:100040000C94BA1A0C94FED90C94BA1A0C94BA1ADD
:100050000C94BA1A0C94BA1A0C941CC10C94BCAC33
:100060000C94BA1A0C9448560C943E560C94BA1A36
:100070000C94BA1A0C94BA1A0C94BA1A0C94BA1AB0
:100080000C942A340C94BA1A0C94BA1A0C94BA1A16
:100090000C94BA1A0C94BA1A0C94BA1A0C94BA1A90
:1000A0000C94BA1A0C94BA1A0C94FC330C94BA1A25
:1000B0000C94BA1A0C94BA1A0C94BA1A0C94BA1A70
:1000C0000C94BA1A0C94BA1A0C94BA1A0C944537B8
:1000D0000C940F370C94BA1A0C94BA1A0C94BA1ADE
:1000E0000C94BA1A084AD73B3BCE016E84BCBFFDC4
:1000F000C12F3D6C74319ABD56833DDA3D00C77FF8
:1001000011BED9E4BB4C3E916BAAAABE0000008090
:100110003F05A84CCDB2D44EB93836A9020C50B91F
:10012000918688083CA6AAAA2ABE000000803F004B
:100130000C9486560C9405A90C9460A80C941DA8E8
:100140000C94D0370C94EF370D941F240D94D212D9
:100150000C94CFAB0C944EA80C946EA80C9464A88D
:100160000C94FBA80D94910C0D94760E0C9448A859
:100170000C9474A90D94FE130D9489120C9433A958
:100180000D94400E0C943DA90C947EA90D94CA02C6
:100190000C94F6A50C943E420D944B0B0C94B3AA10
:1001A0000D94CC0F0C94A2AB0D94B90F0D94580F75
:1001B0000D940C130C943BA80C94FE440D94EB127C
:1001C0000D94B9120D94FA040C94E2560D94D004D7
:1001D0000C9421A90C94C4560D94FF120D94ED13A8
:1001E0000C946AA80C94DF370C94DB370C94DE5621
:1001F0000C9419A90C9459440C94E3370D94B00D48
:100200000C94B2370C9452A80C9483370D94210FA0
:100210000C94EEA90C9488A90C9404570C94F2AB9E
:100220000C94EB370C9447A90C94F6A80C94F25656
:100230000C94C6440D94E40E0D943D240C94E737C1
:100240000D94E00C0C945CA80C940FA90D94E11291
:100250000C946AAA0C9433A80D94770F0C943EA8C2
:100260000C940BAA0C9412AB0D94B1080D94440F8E
:100270000C9456A80C9437A80C94F7AA0C948544B7
:100280000C9473A50C9456A90D94140D0C94DA5685
:100290000C9409380C9490AB0C948D420C94F63766
:1002A0000C9401380C940C570C94B5560C9460A91E
:1002B0000D94A1170C9418A80C94E6560C94EEA873
:1002C0000D94C1140D94B0120C94F5A50C94EE5637
:1002D0000D947C100C942FA80C94D3560D94C40C40
:1002E0000C9444A80C9491420D94EB030C94C137E8
:1002F0000C94EA560D940D0F0C94F9560C946AA9BF
:100300000D9462060D9433070C9429A90C94D737E9
:100310000D94B6124E414E494E495459494E46CD60
:10032000CCCC3D0AD7233C17B7D13877CC2B3295AC
:1003300095E6241FB14F0A000020410000C842008A
:10034000401C4620BCBE4CCA1B0E5AAEC59D740054
:10035000407A10F35A00A0724E18090010A5D4E894
:100360000000E87648170000E40B54020000CA9A27
:100370003B000000E1F50500008096980000004079
:10038000420F000000A086010000001027000000BE
:1003900000E803000000006400000000000A000004
:1003A0000000000100000000002C76D888DC674FB8
:1003B0000823DFC1DFAE59E1B1B796E5E3E453C6E8
:1003C0003AE651997696E8E6C28426EB898C9B62E0
:1003D000ED407C6FFCEFBC9C9F40F2BAA56FA5F48A
:1003E00090055A2AF75C936B6CF9676DC11BFCE0B2
:1003F000E40D47FEF520E6B500D0ED902E03009405
:100400003577050080841E080000204E0A00000099
:10041000C80C333333330F986E12831141EF8D21A3
:1004200014893BE65516CFFEE6DB18D1844B381B0A
:10043000F77C1D901DA4BBE424203284725E2281CF
:1004400000C9F124ECA1E53D27434F4D4D554E49E0
:10045000434154494F4E0044525952554E00455263
:10046000524F525300494E464F004543484F0045B6
:1004700072726F722077726974696E6720746F2070
:10048000454550524F4D210A0053544F505045445A
:100490002E20005072696E7465722073746F7070D4
:1004A00065642064756520746F206572726F727365
:1004B0002E2046697820746865206572726F7220FC
:1004C000616E6420757365204D39393920746F2051
:1004D000726573746172742E202854656D70657234
:1004E00061747572652069732072657365742E205E
:1004F0005365742069742061667465722072657337
:1005000074617274696E67290A004E6F20436865D2
:10051000636B73756D2077697468206C696E6520F4
:100520006E756D6265722C204C617374204C696E1F
:10053000653A20004E6F20436865636B73756D20CC
:1005400077697468206C696E65206E756D6265727E
:100550002C204C617374204C696E653A20006368EE
:1005600065636B73756D206D69736D617463682C61
:10057000204C617374204C696E653A20004C696EA2
:1005800065204E756D626572206973206E6F7420F0
:100590004C617374204C696E65204E756D62657296
:1005A0002B312C204C617374204C696E653A20000D
:1005B0004D3131300053657269616C207374617420
:1005C0007573206D69736D617463680A0077616982
:1005D000740A0053442072656164206572726F7200
:1005E0000A002121204B494C4C20636175736564DE
:1005F00020627920746F6F206D75636820696E6169
:1006000063746976652074696D65202D2063757249
:1006100072656E7420636F6D6D616E643A20004880
:100620006F74656E642049646C652054696D656FF4
:10063000757400486F74656E642049646C6520545D
:10064000696D656F75740A003D3D6F6E46696C613A
:100650006D656E7452756E6F75743D3D0070617599
:100660007365004D363030002066696C616D656ED3
:10067000745F72756E6F7574200066696C616D656C
:100680006E745F72756E6F757420540046696C618C
:100690006D656E7452756E6F75742054002A2A2A27
:1006A000496E6974696E67206361726420697320A2
:1006B0004F4B2A2A2A004D6564696120496E736593
:1006C00072746564004D656469612052656D6F7672
:1006D0006564004D313030305300627573793A20D3
:1006E00070617573656420666F7220696E707574D1
:1006F0000A00627573793A207061757365642066CB
:100700006F7220757365720A00627573793A207092
:10071000726F63657373696E670A002A2A2A6B69B0
:100720006C6C2A2A2A00706F7765726F6666004BC0
:10073000494C4C45442E20005072696E74657220FD
:1007400068616C7465642E206B696C6C2829206369
:10075000616C6C6564210A0053544F505045442E1F
:1007600020005072696E7465722073746F707065CA
:10077000642064756520746F206572726F72732EC9
:100780002046697820746865206572726F722061F6
:100790006E6420757365204D39393920746F20726D
:1007A0006573746172742E202854656D7065726172
:1007B000747572652069732072657365742E205399
:1007C0006574206974206166746572207265737443
:1007D000617274696E67290A006563686F3A004543
:1007E00072726F723A0042696C696E656172204C78
:1007F0006576656C696E6720477269643A0A002104
:10080000212053544F502063616C6C6564206265F5
:100810006361757365206F6620424C546F75636821
:10082000206572726F72202D20726573746172740C
:100830002077697468204D3939390A002121205305
:10084000544F502063616C6C656420626563617510
:100850007365206F6620424C546F75636820657223
:10086000726F72202D2072657374617274207769C3
:100870007468204D3939390A002F2F616374696F0C
:100880006E3A0070726F6D70745F00656E64005335
:10089000656E64204D31303820746F207265737539
:1008A0006D650A00496E736572742066696C616DCE
:1008B000656E7420616E642073656E64204D313006
:1008C000380A005265686561742066696E697368EC
:1008D00065642E0052656865617420446F6E650022
:1008E000526568656174696E672E2E2E00526568C8
:1008F000656174004865617465722054696D656F47
:1009000075740053656E64204D31303820746F204B
:1009100068656174206E6F7A7A6C650A004E6F7A32
:100920007A6C65205061726B656400486F74656E07
:100930006420746F6F20636F6C640A00706175735C
:1009400065640050617573650044697361626C652C
:1009500052756E6F75740050757267654D6F726574
:10096000005061757365640073686F770062757419
:10097000746F6E00626567696E004C6F616420463B
:10098000696C616D656E74004C6F61642046696CC2
:10099000616D656E74205400496E736572742066D3
:1009A000696C616D656E7420616E642073656E6440
:1009B000204D3130380A00726573756D65640052E0
:1009C0006573756D696E670057616974696E67203C
:1009D000666F72206865617475702E0A004C6561DF
:1009E00076696E6720473236003F537065636966EB
:1009F00069656420582C5920636F6F7264696E6159
:100A00007465206F7574206F6620626F756E6473F5
:100A10002E0A003F28522965706561742076616C4A
:100A20007565206E6F7420706C61757369626C659A
:100A30003B206D757374206265206174206C656164
:100A4000737420312E0A003F285229657065617445
:100A5000206D7573742062652073706563696669C3
:100A60006564207768656E206E6F74207573696E9B
:100A70006720616E204C43442E0A003F537065632B
:100A80006966696564206E6F7A7A6C652074656D3D
:100A90007065726174757265206E6F7420706C6120
:100AA000757369626C652E0A003F537065636966F1
:100AB0006965642066696C616D656E742073697A1E
:100AC00065206E6F7420706C61757369626C652E41
:100AD0000A003F53706563696669656420707269D6
:100AE0006D65206C656E677468206E6F7420706C25
:100AF00061757369626C652E0A003F5072696D659D
:100B0000206C656E677468206D7573742062652053
:100B1000737065636966696564207768656E206EC9
:100B20006F74207573696E6720616E204C43442E8C
:100B30000A003F537065636966696564206E6F7A69
:100B40007A6C652073697A65206E6F7420706C61B1
:100B5000757369626C652E0A003F52657472616339
:100B600074696F6E204D756C7469706C6965722064
:100B70006D7573742062652073706563696669655D
:100B8000642E0A003F53706563696669656420528C
:100B9000657472616374696F6E204D756C746970F1
:100BA0006C696572206E6F7420706C617573696218
:100BB0006C652E0A003F5370656369666965642041
:100BC0006C6179657220686569676874206E6F74FE
:100BD00020706C61757369626C652E0A0043292E62
:100BE0000A003F53706563696669656420626564E5
:100BF0002074656D7065726174757265206E6F74B6
:100C000020706C61757369626C65202834302D002A
:100C1000473236207374617274696E672E2E2E0A05
:100C2000004F46460A00466164652048656967686A
:100C3000742000426564204C6576656C696E67209F
:100C4000004661696C656420746F20656E61626C3A
:100C50006520426564204C6576656C696E670A00A4
:100C6000496E76616C6964206D6573682E0A005068
:100C7000726F62696E6720506F696E740025532031
:100C800025692F2569002E0A002F0050726F6269B6
:100C90006E67206D65736820706F696E7420002028
:100CA0002844525952554E29004732392041757413
:100CB0006F20426564204C6576656C696E67003F05
:100CC00020284C2C522C462C4229206F7574206F02
:100CD0006620626F756E64732E0A003F2856296580
:100CE00072626F7365206C6576656C20696D706CDF
:100CF00061757369626C652028302D34292E0A00D5
:100D0000426164205A2076616C75650A004E6F203E
:100D100062696C696E65617220677269640A004479
:100D20006576696174696F6E0025533A20257300FA
:100D300046696E6973686564210A003A207A3A2030
:100D400000206F662000476F696E6720746F3A203D
:100D5000580043570A00206469723A0020616E67A8
:100D60006C653A00537461727420726164697573C2
:100D70003A004D343820506F696E740025533A2084
:100D800025642F256400506F736974696F6E696EF6
:100D900067207468652070726F62652E2E2E0A00BF
:100DA0003F4C656773206F66206D6F76656D656E6D
:100DB0007420696D706C61757369626C6520283090
:100DC0002D3135292E0A003F2028582C5929206F13
:100DD0007574206F6620626F756E64732E0A005002
:100DE000726F6265206F7574206F6620626F756E1A
:100DF0006473003F53616D706C652073697A652080
:100E00006E6F7420706C61757369626C6520283434
:100E10002D3530292E0A004D3438205A2D50726F4E
:100E20006265205265706561746162696C6974798C
:100E300020546573740A003F2856296572626F73E7
:100E400065206C6576656C20696D706C6175736981
:100E5000626C652028302D34292E0A005374616E8F
:100E60006461726420446576696174696F6E3A20CA
:100E7000002052616E67653A2000204D61783A206B
:100E800000204D696E3A2000205369676D613A2059
:100E9000004D65616E3A20005741524E494E472140
:100EA000204C6F77205A204A65726B206D61792043
:100EB0006C65616420746F20756E77616E74656413
:100EC000207061757365732E0A004F4646004F4EC1
:100ED0000020204D61783A2000200020204D696ECE
:100EE0003A2000536F667420656E6473746F70737C
:100EF0003A20003D3D4F6E506F7765724C6F7373B3
:100F0000526573756D653D3D004D32342053256C3F
:100F1000642054256C64004739322E3920452573EE
:100F200000473120462564004739322E39205A25A2
:100F300073004731205A302046323030004731208C
:100F400058257320592573204633303030004D34F6
:100F5000323020532569205A2573004D3130362018
:100F600050256920532569004D32303020442573C7
:100F70000047323852305859004739322E3920450F
:100F800030205A300A47315A2573004D313039200C
:100F9000532569004D31393020532569004D3432D5
:100FA00030205330205A300020496E76616C6964DD
:100FB000206578747275646572200047322F47335C
:100FC0002062616420706172616D65746572730A7C
:100FD00000536C6565702E2E2E005A2050726F6281
:100FE000652050617374204265640A005A20507273
:100FF0006F62652050617374204265640047323827
:101000004C30004D3131372050726F62652066617F
:10101000696C65642E0A4732380A0070726F626527
:101020005F72657769706500473239205265747266
:1010300079696E670050726F62696E6720466169F8
:101040006C6564004D31313720426564206C6576F3
:10105000656C696E67206661696C65642E0A47304D
:10106000205A31300A4D3330302050323520533839
:1010700038300A4D333030205035302053300A4D4F
:101080003330302050323520533838300A4D333029
:1010900030205035302053300A4D3330302050321C
:1010A0003520533838300A4D333030205035302019
:1010B00053300A47342053310070726F62655F66A7
:1010C00061696C6564004D31313720426564206C84
:1010D0006576656C696E6720646F6E652E00205AB8
:1010E0003A200020593A200042656420583A2000F6
:1010F0004D65736820706F696E74206F7574206F12
:10110000662072616E67650A004D302053746F70FF
:10111000004D312053746F7000436F6E74696E75AB
:101120006500436C69636B20746F20526573756D45
:10113000652E2E2E004E6F204D6F76652E00456E6B
:10114000642066696C65206C6973740A0042656787
:10115000696E2066696C65206C6973740A004E6F55
:10116000206D656469610A00526573756D696E670B
:1011700020534400286E6F2066696C652900437512
:101180007272656E742066696C653A2000507269EF
:101190006E742074696D653A20000A53746174732B
:1011A0003A2046696C616D656E7420757365643AAA
:1011B00020002C204C6F6E67657374206A6F623A52
:1011C0002000546F74616C2074696D653A2000537F
:1011D000746174733A20002C204661696C65643A2E
:1011E00020002C2046696E69736865643A200050BF
:1011F00072696E74733A200053746174733A2000FC
:10120000436F6F6C696E672E2E2E0048656174699E
:101210006E672E2E2E0045202553006F6B006F66E3
:1012200066006A0465045E04570449044445425557
:10123000473A004D31313320530042656420436FFB
:101240006F6C696E672E2E2E0042656420486561C2
:1012500074696E672E2E2E00544D33442045352080
:10126000506C7573204F46462E002F2F00205200E1
:10127000416363656C65726174696F6E3A205000FA
:101280004D32303620580046523A0020466C6F7777
:101290003A20003A200020536572766F2000206FBC
:1012A0007574206F662072616E67650A00536572FF
:1012B000766F200020643A0020693A0020703A00DE
:1012C000496E76616C6964206578747275646572C4
:1012D0000A0020643A0020693A0020703A006469EC
:1012E0007300656E0043290A0061626C6564202802
:1012F0006D696E2074656D702000436F6C642065AD
:101300007874727564657320617265200050494479
:10131000204175746F74756E6500504944204175A5
:10132000746F74756E65206661696C656421204216
:101330006164206865617465722069640A004669A9
:101340006C616D656E742072756E6F757420646962
:101350007374616E636520286D6D293A20004669BB
:101360006C616D656E742072756E6F757420004DC2
:1013700034323120696E636F7272656374207061FC
:1013800072616D657465722075736167650A004DE1
:1013900065736820706F696E74206F7574206F6656
:1013A0002072616E67650A004F666673657473200C
:1013B0004170706C696564004572723A20546F6FB9
:1013C000206661722100546F6F2066617220667220
:1013D0006F6D207265666572656E636520706F69FA
:1013E0006E740A00454550524F4D204F4B0A002E57
:1013F0000A002028302D313029002076616C756577
:10140000206F7574206F662072616E67650041649D
:1014100076616E6365204B3D00506F7765722D6C71
:101420006F7373207265636F766572792000436114
:10143000703A004D4541545041434B00434F4F4C8F
:1014400045525F54454D5045524154555245004315
:1014500048414D4245525F54454D504552415455C7
:10146000524500424142595354455050494E47005D
:1014700041524353004D4F54494F4E5F4D4F4445E9
:101480005300544845524D414C5F50524F544543D0
:1014900054494F4E004C4F4E475F46494C454E41D4
:1014A0004D45004155544F5245504F52545F53449F
:1014B0005F5354415455530053445F575249544568
:1014C000005245504541540053444341524400505A
:1014D000524F4D50545F535550504F525400454D4C
:1014E000455247454E43595F504152534552004380
:1014F0004153455F4C494748545F4252494748541D
:101500004E45535300544F47474C455F4C4947485D
:10151000545300534F4654574152455F504F57451F
:1015200052004255494C445F50455243454E540089
:101530004C4556454C494E475F44415441005A5F23
:1015400050524F42450052554E4F5554004155544C
:101550004F4C4556454C005052494E545F4A4F42FD
:101560000050524F4752455353004155544F524536
:10157000504F52545F54454D5000564F4C554D45B9
:101580005452494300454550524F4D0042494E4147
:1015900052595F46494C455F5452414E534645525D
:1015A0000053455249414C5F584F4E5F584F464695
:1015B000004649524D574152455F4E414D453A4DC7
:1015C00061726C696E20322E302E375F4457372E91
:1015D0003320544D334420453550454D444242203C
:1015E0002841707220323420323032312032313A88
:1015F00033313A33302920534F555243455F434FDF
:1016000044455F55524C3A68747470733A2F2F6793
:1016100069746875622E636F6D2F496E73616E69B0
:1016200074794175746F6D6174696F6E2F4D61725D
:101630006C696E2F747265652F437265616C697495
:10164000794477696E5F322E302050524F544F43A9
:101650004F4C5F56455253494F4E3A312E30204D34
:10166000414348494E455F545950453A544D3344DF
:1016700020453520506C75732045585452554445CB
:10168000525F434F554E543A3120555549443A63C1
:10169000656465326132662D343161322D34373400
:1016A000382D396231322D63353563363266333643
:1016B0003766660A0050726F6265204F6666736512
:1016C00074205A0050726F6265204F6666736574AD
:1016D000205A00290A0020746F20003F5A206F759D
:1016E00074206F662072616E6765202800290A00E9
:1016F00020746F20003F59206F7574206F66207230
:10170000616E676520282D00290A0020746F200073
:101710003F58206F7574206F662072616E67652078
:10172000282D0050726F6265204F666673657420C5
:1017300058004D383400446F6E65207072696E74C5
:10174000696E672066696C650A004D3737004D3356
:10175000310043616E6E6F74206F70656E2073751B
:101760006264697220002569730025696D2025690E
:1017700073002569682025696D2025697300256936
:1017800064202569682025696D2025697300256915
:101790007920256964202569682025696D202569DF
:1017A00073003D3D4477696E20496E697420436F34
:1017B0006D706C6574653D3D002A2A2A4E6F7A7AF9
:1017C0006C6554656D705374617475735B325D2024
:1017D0003D003D3D48656174696E6720446F6E65EC
:1017E000204368616E67652046696C616D656E7443
:1017F0003D3D002020737461727470726F67726572
:10180000737320003D3D7761697477617920353DC0
:101810003D003D3D7761697477617920343D3D003D
:101820003D3D7761697477617920333D3D003D3DF1
:101830007761697477617920313D3D003D3D6F6E80
:101840005072696E7454696D657253746F7070650F
:10185000643D3D003D3D6F6E466163746F72795229
:10186000657365743D3D00270A0A000027202700A4
:101870002027002D006E6F74696669636174696F5B
:101880006E200063616E63656C005072696E742037
:1018900041626F72746564004469736D69737300AB
:1018A00055492041626F7274656400726573756D8D
:1018B00065004D3234002A2A2A43506C6179205445
:1018C0006F6E652A2A2A003D3D6F6E5072696E74F4
:1018D00054696D65725061757365643D3D00486F74
:1018E0006D696E67204661696C6564006F70656E36
:1018F00000545249474745524544003A2000666922
:101900006C616D656E74007A5F6D696E00795F6DF4
:10191000617800785F6D6178005265706F727469EC
:101920006E6720656E6473746F7020737461747574
:10193000730A0020746F6F206C6F6E672065787477
:10194000727573696F6E2070726576656E7465640A
:101950000A0020636F6C6420657874727573696F18
:101960006E2070726576656E7465640A00486F6DEE
:10197000652025732573257320466972737400579B
:1019800061726E696E673A20486F6D696E672042BA
:10199000756D702044697669736F72203C20310A3E
:1019A000000202040000B4430000B4430000000041
:1019B0000000B4430000B4430000C84300000041ED
:1019C00000000041000000400101FF000000010094
:1019D0000000010000800055555500000040003314
:1019E000333300AAAA2A004992240000002000C72D
:1019F000711C0099991900D1451700555515003BE8
:101A0000B113002449120011111100000010000F41
:101A10000F0F00E3380E0043790D00CCCC0C00C34F
:101A2000300C00E8A20B0064210B00AAAA0A007087
:101A30003D0A009DD80900427B090092240900DC80
:101A4000D30800888808001042080000000800F051
:101A5000C107008787070075500700711C07003E0B
:101A6000EB0600A1BC0600699006006666060070E1
:101A70003E06006118060017F4050074D105005BEE
:101A8000B00500B29005006272050055550500785A
:101A9000390500B81E0500050505004EEC04008759
:101AA000D40400A1BD040090A7040049920400C121
:101AB0007D0400EE690400C7560400444404005C41
:101AC0003204000821040041100400000004003F1B
:101AD000F00300F8E0030026D20300C3C30300CCE8
:101AE000B503003AA803000A9B0300388E0300C028
:101AF0008103009F750300D0690300505E03001D41
:101B000053030034480300913D03003333030016B0
:101B1000290300381F030097150300300C0300034E
:101B20000303000BFA020049F10200BAE802005C6C
:101B3000E002002DD802002DD0020059C80200B0EA
:101B4000C0020031B90200DAB10200AAAA0200A064
:101B5000A30200BC9C0200FA9502005C8F0200DF29
:101B600088020082820200457C020027760200275C
:101B7000700200436A02007C640200D05E02003FF3
:101B8000590200C8530200FFFDFCFAF8F6F4F2F027
:101B9000EEECEAE9E7E5E3E1E0DEDCDAD9D7D5D43B
:101BA000D2D0CFCDCBCAC8C7C5C3C2C0BFBDBCBAD7
:101BB000B9B7B6B4B3B2B0AFADACAAA9A8A6A5A444
:101BC000A2A1A09E9D9C9A99989795949392908F8C
:101BD0008E8D8B8A8988878684838281807F7E7DB3
:101BE0007B7A797877767574737271706F6E6D6CBD
:101BF0006B6A696867666564636261605F5E5D5CAD
:101C00005B5A5958585756555453525150504F4E8D
:101C10004D4C4B4A4A494847464645444342424157
:101C2000403F3E3E3D3C3B3B3A3938383736353510
:101C3000343332323130302F2E2E2D2C2B2B2A29BB
:101C40002928272726252524232322212120201F58
:101C50001E1E1D1C1C1B1B1A1919181817161615E9
:101C60001514131312121111100F0F0E0E0D0D0C6F
:101C70000C0B0A0A090908080707060605050404EB
:101C8000030302020100003D3D6F6E5072696E74E5
:101C900054696D6572537461727465643D3D0000F2
:101CA00000B4430000B4430000C84300000000003B
:101CB000000000000000003D3D6F6E53746F7265C0
:101CC00053657474696E67733D3D003D3D6F6E43AF
:101CD0006F6E66696775726174696F6E53746F7247
:101CE000655772697474656E3D3D0053657474691F
:101CF0006E67732053746F726564000A20696E69A1
:101D000074207A70726F62655F7A6F66667365744D
:101D1000203D20003D3D6F6E436F6E6669677572B2
:101D20006174696F6E53746F7265526561643D3D95
:101D300000454550524F4D20496E697469616C6988
:101D40007A65640A003B20003A0A0020204D3630B4
:101D500033200020440020204D34313220530046EF
:101D6000696C616D656E742072756E6F7574207329
:101D7000656E736F723A002055004C0046696C61C5
:101D80006D656E74206C6F61642F756E6C6F61642D
:101D9000206C656E677468733A0020204D393030CE
:101DA000204B004C696E65617220416476616E6300
:101DB000653A0020204D3835312058005A2D507298
:101DC0006F6265204F66667365740020204D343164
:101DD00033205300506F7765722D4C6F7373205210
:101DE00065636F766572793A0020440020490020CF
:101DF000204D333034205000204400204900202062
:101E00004D3330312050005049442073657474695B
:101E10006E67733A00204A0020204732392057204D
:101E2000490020204D3432302053004175746F201A
:101E3000426564204C6576656C696E673A002020C7
:101E40004D323036205800486F6D65206F666673DE
:101E500065743A0020580020530020204D32303560
:101E6000204200416476616E6365643A20423C6DB5
:101E7000696E5F7365676D656E745F74696D655FCC
:101E800075733E20533C6D696E5F66656564726173
:101E900074653E20543C6D696E5F74726176656C4A
:101EA0005F66656564726174653E20583C6D61785B
:101EB0005F785F6A65726B3E20593C6D61785F792F
:101EC0005F6A65726B3E205A3C6D61785F7A5F6A2B
:101ED00065726B3E20453C6D61785F655F6A657237
:101EE0006B3E0020540020520020204D3230342020
:101EF0005000416363656C65726174696F6E202880
:101F0000756E6974732F7332293A20503C70726970
:101F10006E745F616363656C3E20523C72657472DF
:101F20006163745F616363656C3E20543C747261ED
:101F300076656C5F616363656C3E0020204D3230D6
:101F4000312058004D6178696D756D20416363657E
:101F50006C65726174696F6E2028756E6974732F79
:101F60007332293A0020204D3230332058004D6121
:101F700078696D756D20666565647261746573203E
:101F800028756E6974732F73293A005374657073E2
:101F90002070657220756E69743A0020440020201C
:101FA0004D3230302053002044697361626C6564A7
:101FB0000A0046696C616D656E742073657474699E
:101FC0006E67733A0020286D6D290020204732315A
:101FD000202020203B20556E69747320696E206D8F
:101FE0006D003D3D6F6E4C6F616453657474696E36
:101FF00067733D3D0000803B4400803B440000206F
:1020000041000096420000A0420000A042000048AB
:10201000440000BE42D0070000D00700006400006A
:10202000004B00000024F4D43050C38E20C2A240E4
:1020300017828B7011127A910D816CD90AA861E117
:1020400008C7586607615143061E4B5D05C145A789
:10205000041A411104093D9803713931034036DBFC
:102060000265339102D4305402802E1D02632CEE9F
:1020700001752AC501B028A001102781018F2564B0
:10208000012B244B01E0223401AC211F018D200DD6
:1020900001801FFC00841EED00971DDF00B81CD2DC
:1020A00000E61BC600201BBC00641AB200B219A8CF
:1020B000000A19A0006A189900D117910040178BE7
:1020C00000B516840031167E00B31579003A1573F9
:1020D00000C7146F0058146A00EE1366008813637B
:1020E0000025135E00C7125B006C125700151254D6
:1020F00000C111510070114F0021114B00D6104941
:10210000008D1047004610440002104200C00F40EE
:1021100000800F3E00420F3C00060F3B00CB0E3804
:1021200000930E37005C0E3500270E3400F30D329D
:1021300000C10D3100900D3000600D2E00320D2DCC
:1021400000050D2C00D90C2B00AE0C2900850C29A4
:10215000005C0C2700350C27000E0C2600E80B2431
:1021600000C40B2400A00B23007D0B23005A0B217D
:1021700000390B2100180B2000F80A1F00D90A1E95
:1021800000BB0A1E009D0A1D00800A1D00630A1C78
:1021900000470A1B002C0A1B00110A1A00F7091A33
:1021A00000DD091900C4091900AB091900920917CB
:1021B000007B091800630917004C09160036091640
:1021C00000200916000A091500F5081500E008149A
:1021D00000CC081400B8081400A4081400900813D8
:1021E000007D0812006B0813005808120046081200
:1021F0000034081100230811001208110001081111
:1022000000F0071000E0071000D0071000C0071012
:1022100000B0070F00A107100091070E0083070F01
:102220000074070F0065070E0057070E0049070EE0
:10223000003B070D002E070E0020070D0013070DB1
:102240000006070D00F9060C00ED060D00E0060C77
:1022500000D4060C00C8060C00BC060C00B0060C2E
:1022600000A4060B0099060C008D060B0082060BDD
:102270000077060B006C060B0061060A0057060B80
:10228000004C060A0042060A0038060A002E060A1A
:102290000024060A001A060A001006090007060AAA
:1022A00000FD050900F4050900EB050900E2050938
:1022B00000D9050900D0050900C7050900BE0509B8
:1022C00000B5050800AD050800A50509009C050836
:1022D00000940508008C050800840508007C0508AA
:1022E00000740508006C050700650508005D05071A
:1022F00000560508004E0507004705070040050881
:102300000038050700310507002A050700230507E7
:10231000001C050600160507000F05070008050646
:102320000002050700FB040600F5040700EE0406A2
:1023300000E8040600E2040700DB040600D50406FA
:1023400000CF040600C9040600C3040600BD04064D
:1023500000B7040600B1040500AC040600A604069C
:1023600000A00405009B04060095040500900406E7
:10237000008A04050085040500800406007A04052F
:102380000075040500700405006B04050066040573
:1023900000610405005C04050057040500520405B3
:1023A000004D04050048040500430405003E0404F4
:1023B000003A04050035040500300404002C04052F
:1023C0000027040400230405001E0404001A04046A
:1023D0000016040500110404000D0404000904059E
:1023E000000404040000040400FC030400F80304D7
:1023F00000F4030400F0030400EC030400E8030409
:1024000000E4030400E0030400DC030400D8030438
:1024100000D4030400D0030400CC030400C8030369
:1024200000C503030024F404D9201BC40C5C0E98DF
:1024300004C4095F0265077101F405F900FB04B3E8
:102440000048048700C10369005803550003034591
:1024500000BE023A008402310053022A00290225FC
:102460000004022000E4011C00C8011900AF01179C
:102470000098011400840113007101100061011023
:102480000051010E0043010D0036010B002B010B22
:102490000020010B00150109000C010900030108CF
:1024A00000FB000800F3000800EB000700E4000652
:1024B00000DE000600D8000600D2000600CC0005B1
:1024C00000C7000500C2000500BD000400B90004FB
:1024D00000B5000400B1000400AD000400A9000430
:1024E00000A5000300A20003009F0004009B00035E
:1024F0000098000300950002009300030090000381
:10250000008D0002008B000300880002008600029C
:102510000084000300810002007F0002007D0002B1
:10252000007B0002007900020077000100760002C3
:10253000007400020072000100710002006F0002CE
:10254000006D0001006C0002006A000100690002D9
:1025500000670001006600010065000100640002E0
:10256000006200010061000100600001005F0002E4
:10257000005D0001005C0001005B0001005A0001E9
:1025800000590001005800010057000100560001E9
:1025900000550001005400010053000000530001E9
:1025A000005200010051000100500001004F0001E5
:1025B000004E0000004E0001004D0001004C0001E3
:1025C000004B0000004B0001004A000100490001DF
:1025D00000480000004800010047000100460000DC
:1025E00000460001004500000045000100440001D4
:1025F00000430000004300010042000000420001CF
:10260000004100000041000100400001003F0000C7
:10261000003F0001003E0000003E0001003D0000C0
:10262000003D0001003C0000003C0000003C0001B7
:10263000003B0000003B0001003A0000003A0001AE
:1026400000390000003900010038000000380000A7
:10265000003800010037000000370001003600009C
:102660000036000000360001003500000035000093
:102670000035000100340000003400000034000187
:10268000003300000033000000330001003200007E
:102690000032000000320001003100000031000073
:1026A0000031000100300000003000000030000167
:1026B000002F0000002F0000002F0000002F00015D
:1026C000002E0000002E0000002E0001002D000052
:1026D000002D0000002D0000002D0001002C000046
:1026E000002C0000002C0000002C0001002B00003A
:1026F000002B0000002B0000002B0001002A00002E
:10270000002A0000002A0000002A00010029000021
:102710000029000000290000002900000029000114
:102720000028000000280000002800000028000009
:1027300000280001002700000027000000270000FB
:1027400000270000002700010026000000260000EE
:1027500000260000002600000026000100250000E1
:1027600000250000002500000025000000250000D5
:1027700000250001002400000024000000240000C7
:1027800000240000002400010023000000230000BA
:1027900000230000002300000023000000230000AD
:1027A000002300010022000000220000002200009F
:1027B0000022000000220000002200010021000091
:1027C0000021000000210000002100000021000085
:1027D0000021000000210001002000000020000076
:1027E0000020000000200000002000000020000069
:1027F0000020000000200001001F0000001F00005A
:10280000001F0000001F0000001F0000001F00004C
:10281000001F0001001E0000001E0000001E00003E
:10282000001E000000232C0000B8220000561800F3
:10283000003A0F0000B8080000B104000071020067
:10284000003E01000020436F756E7420583A00234B
:10285000646566696E652044454641554C545F0089
:1028600000626564004B6420004B6920004B7020BF
:1028700000504944204175746F74756E6520666917
:102880006E697368656421205075742074686520D2
:102890006C617374204B702C204B6920616E642036
:1028A0004B6420636F6E7374616E74732066726F15
:1028B0006D2062656C6F7720696E746F20436F6E58
:1028C00066696775726174696F6E2E680A00504997
:1028D00044204175746F74756E65206661696C651E
:1028E00064212074696D656F75740A005049442035
:1028F0004175746F74756E65206661696C656421DD
:102900002054656D706572617475726520746F6FA7
:1029100020686967680A00204B643A2000204B69F0
:102920003A2000204B703A200020436C6173736999
:102930006320504944200A00204E6F206F76657254
:1029400073686F6F740A002054753A2000204B752D
:102950003A2000206D61783A2000206D696E3A209F
:102960000020643A200020626961733A20005049D7
:1029700044204175746F74756E6520737461727450
:102980000A00504944204175746F74756E65206665
:1029900061696C6564212054656D70657261747540
:1029A000726520746F6F20686967680A0042656409
:1029B00000453100626564002C2073797374656D85
:1029C0002073746F7070656421204865617465724E
:1029D0005F49443A200048656174696E672046612A
:1029E000696C65640048656174696E672066616939
:1029F0006C6564004D3131322053687574646F77B3
:102A00006E001000C90210012C014001220170016A
:102A10001801B0010E01F00104015002FA00B002E9
:102A2000F0003003E600D003DC009004D200700513
:102A3000C800A006BE000008B400B009AA00D00B70
:102A4000A000600E960060118C0000158200201915
:102A50007800C01D6E00A0226400B0275A00902CA0
:102A6000500000314600E0343C0010383200903A0B
:102A70002800603C1E00A03D1400803E0A00203F5C
:102A80000000544845524D414C2052554E4157414B
:102A90005900546865726D616C2052756E61776182
:102AA00079004572723A204D415854454D50004DC1
:102AB000415854454D50207472696767657265646A
:102AC000004572723A204D494E54454D50004D49D3
:102AD0004E54454D50207472696767657265640095
:102AE000202F002042403A0020403A0020573A0070
:102AF00020573A00496E76616C696420657874727B
:102B0000756465720A007C3C3E5E2B3D3F2F5B5D29
:102B10003B2C2A225C0043616E6E6F74206F7065DF
:102B20006E207375626469722000534420496E6997
:102B300074204661696C0053442063617264206FA5
:102B40006B0A006F70656E526F6F74206661696CFE
:102B500065640A00766F6C756D652E696E69742008
:102B60006661696C65640A004E6F2053442063619E
:102B700072640A000A4D3234004D3233202573004E
:102B80002E0A006F70656E206661696C65642C208A
:102B900046696C653A200046696C652073656C6512
:102BA000637465640A002053697A653A20004669B7
:102BB0006C65206F70656E65643A2000454E442058
:102BC000535542524F5554494E450A002220706FCA
:102BD00073002220706172656E743A220053554270
:102BE000524F5554494E452043414C4C207461721C
:102BF0006765743A220053756263616C6C204F768E
:102C00006572666C6F7700457863656564656420FE
:102C10006D617820535542524F5554494E452064BA
:102C2000657074683A002E0A0044656C6574696FBB
:102C30006E206661696C65642C2046696C653A207B
:102C40000046696C652064656C657465643A005380
:102C500044207072696E74696E67206279746520B1
:102C6000004E6F74205344207072696E74696E67F1
:102C70000A0057726974696E6720746F2066696C08
:102C8000653A2000667265736800646F696E67005C
:102C90002066696C653A20004E6F7720002F6175C1
:102CA000746F25632E67002020506C616E6E657214
:102CB00042756666657242797465733A20002046F3
:102CC000726565204D656D6F72793A2000436F6DB6
:102CD00070696C65643A2041707220323420323061
:102CE00032310A00204C6173742055706461746540
:102CF000643A20323032312D30342D3138207C206E
:102D0000417574686F723A2054696E794D616368D9
:102D1000696E657333440A00322E302E375F445794
:102D2000372E330A004D61726C696E0020536F6656
:102D300074776172652052657365740A002057616B
:102D4000746368646F672052657365740A0020427B
:102D5000726F776E206F75742052657365740A0008
:102D60002045787465726E616C2052657365740AD3
:102D700000506F77657255700A0073746172740A3F
:102D8000004732385859004D313030310065727289
:102D90006F722077726974696E6720746F2066693C
:102DA0006C650A00446F6E6520736176696E6720FA
:102DB00066696C652E0A004D323900456E64737485
:102DC0006F70730025532025632025632025632021
:102DD000256300205A3A0020593A0020583A0065ED
:102DE0006E6473746F7073206869743A2000000019
:102DF0000A0B02090C0D0E08070304010000000075
:102E000000000000000000000000000000000000C2
:102E1000000000000000000000001211100000007F
:102E200000000000000000000000000000000000A2
:102E3000000000006001F4017001EA019001E0016E
:102E4000B001D601D001CC010002C2013002B801AC
:102E50006002AE019002A401D0029A012003900109
:102E600070038601C0037C0130047201A004680174
:102E700020055E01B005540160064A0120074001AB
:102E8000F0073601F0082C01100A2201500B18013E
:102E9000C00C0E01500E04013010FA002012F00098
:102EA0005014E600C016DC007019D200501CC80097
:102EB000501FBE007022B400B025AA00F028A00068
:102EC000202C9600302F8C0010328200A034780025
:102ED000F0366E00E0386400803A5A00403B5500FE
:102EE000E03B5000F03C4600C03D3C00603E3200FC
:102EF000E03E2800303F1E00503F1900703F140094
:102F0000A03F0A00C03F0000D03FF6FFE03FECFFCB
:102F100050726F62696E67204661696C656400205B
:102F20005A3A200020593A200042656420583A203D
:102F3000003D3D6F6E55736572436F6E6669726DCD
:102F400052657175697265643D3D00220A00556ED7
:102F50006B6E6F776E20636F6D6D616E643A2022C9
:102F6000002042002050006F6B00204500205A00D6
:102F7000205900204D393220580020453A00205A6F
:102F80003A0020593A00583A0020746F6F206C6F55
:102F90006E6720657874727573696F6E20707265E4
:102FA00076656E7465640A0020636F6C64206578D2
:102FB00074727573696F6E2070726576656E746574
:102FC000640A0043616E6E6F7420656E74657220D2
:102FD0007375626469723A20004D323520500A4D93
:102FE000323400526573756D650055492050617526
:102FF0007365004E6F204D61746368203A0050671E
:103000005570005067446F776E0049732046696CB5
:103010006520004973204469722000476F55704451
:10302000697200486173204D656469610046696C8E
:10303000656E616D652053656C6563746564004DF4
:103040003130303043004D313030300046696C61F2
:103050006D656E7420537461742030202D20330010
:1030600046696C616D656E74205374617420302004
:103070002D20320046696C616D656E742053746159
:10308000742030202D2031002046696C616D656E02
:103090007420526573706F6E7365204E6F005265B9
:1030A00073756D652059657320647572696E67204C
:1030B0007072696E74000A204E6F2046696C616DF3
:1030C000656E7400496E76616C6964204F70746936
:1030D0006F6E004D3530300053746F72652053654C
:1030E0007474696E677300426564205049442053CC
:1030F000746172746564004D3939390A4D32383063
:1031000050305331363000424C546F756368205252
:1031100065736574004D3530320A4D3530300049E5
:103120006E697420454550524F4D00486F74656E6E
:103130006420504944205374617274656400456E84
:10314000676C69736820416C7265616479205365AE
:1031500074004368696E657365204E6F7420537503
:1031600070706F7274656400496E4C616E6743687D
:103170006F696365000A202A2A2A72656364617494
:103180002E646174615B305D203D004732380A4730
:1031900031204631303030205A313000556E737551
:1031A00070706F72746564204F7074696F6E205315
:1031B000656C65637465640047323652323535009C
:1031C0004D3139305335350A4732380A4732390ADA
:1031D0004D3430300A4D313034533231350A4732B4
:1031E000380A4D313039533231350A4D343230538B
:1031F000310A47315831303059313030463530306E
:10320000300A47315A300A4D3530300A4D313137A6
:1032100020536574205A204F6666736574004731E9
:10322000204631303030205A302E30004732380AB4
:103230004731204631303030205A302E30004D3565
:103240003030005A204F6666736574203A2025732B
:10325000004D353030005A204F6666736574203A51
:10326000202573004732380A473146313530305A0D
:10327000302E30004732385A0A4731463135303027
:103280005A302E30004D383400473146313030301E
:103290005A302E30004732380A473146313030300C
:1032A0005A302E30004D616E75616C5365745465F3
:1032B0006D70005A204F6666736574203A2025733E
:1032C0000053746F7020547269676765726564009B
:1032D00053746F70204E6F0053746F705072696E2C
:1032E000740048616E646C652044617461204164BF
:1032F0006A75737420322053657474696E67205345
:10330000637265656E200048616E646C652044617F
:103310007461205072696E7446696C652033205365
:10332000657474696E672053637265656E2000482A
:10333000616E646C652044617461205072696E74C2
:1033400046696C6520322053657474696E6720533A
:10335000637265656E20004D38340048616E646CA0
:10336000652044617461205072696E7446696C65B1
:1033700020506F73740048616E646C652044617402
:1033800061205072696E7446696C652050726500E8
:10339000426567696E537769746368003D3D2043F9
:1033A0006865636B6B65793D3D007265636461744C
:1033B0002E61646472203D3D007265636461742E09
:1033C000646174615B305D203D3D007761697477B5
:1033D0006179203D3D0020202A2A2A2A2A2A2A52C1
:1033E00054535F48616E646C65446174612A2A2A93
:1033F0002A2A2A2A2A2000526573656E643A200020
:1034000000002200250028002B002E00310034008F
:1034100002010000050108010B0100002100240049
:1034200027002A002D0030003300010100000401B4
:1034300007010A0105050505070508080808020235
:1034400002020A0A0808040404040101010101013E
:1034500001010303030303030303040707070C0C21
:103460000C0C0C0C0C0C02020202060606060606E8
:1034700006060B0B0B0B0B0B0B0B0102102020088D
:1034800008102040102040800201020108040201BF
:10349000010204081020408080402010080402012E
:1034A0008004020180402010080402010804020187
:1034B000010204081020408001020408102040800E
:1034C000544D334420453520506C7573205265614E
:1034D00064792E005072696E74696E672E2E2E000C
:1034E0005072696E7420506175736564006E6F74FC
:1034F000696669636174696F6E20005049442054A5
:10350000756E652046696E697368656400001C010C
:10351000A40011241FBECFEFD1E2DEBFCDBF00E07B
:103520000CBF14E0A0E0B2E0E0EAFAE602E00BBF74
:1035300002C007900D92A032B107D9F726E1A0E2B0
:10354000B4E001C01D92A33BB207E1F71AE1C8E85D
:10355000DAE100E006C021970109802FFE010F94F7
:103560007D31C738D10780E00807A9F70F94D51E31
:103570000D943E350C9400009F92AF92BF92CF9273
:10358000DF92EF92FF920F931F93CF93DF9300D0C0
:103590001F921F92CDB7DEB7E7E8FBE10027BB27FC
:1035A000462F572FA82FAA2341F4A52F542FB85FD9
:1035B000AA2319F4A52F5527B85FA03138F45295E6
:1035C000A295452F4F70507FA42BBC5FA03428F4E8
:1035D000550FAA1F550FAA1FBE5FA03818F4550F2C
:1035E000AA1FB395550FAA1FEA0FF01F449151E08F
:1035F000AA27B85081F1C8F0B0FF02C0440F551F90
:10360000B1FF04C0440F551F440F551FB2FF06C041
:1036100052954295142F1F70407F512BB3FF1BC052
:10362000A52F542F44270C942B1BB195B0FF02C03B
:1036300055954795B1FF04C05595479555954795C4
:10364000B2FF05C05295407F4295452B5F70B3FF96
:1036500002C0452F5527DD24CC24BB24B2E0649F53
:10366000D018C108B00AB00B749FC018B108B00BD5
:10367000849FB018B109659FC018B108B00B759F41
:10368000B018B109859FB0196A9FB018B1097A9F27
:10369000B0194D9DA12C99243327992722275D9D90
:1036A000A00C911C301F901F201FAD9D900C311D50
:1036B000901F201F4C9DA00C911C301F901F201F9D
:1036C0005C9D900C311D901F201FAC9D300D911DF5
:1036D000201F4B9D900C311D901F201F5B9D300DB6
:1036E000911D201FAB9D900D211D4B9F300D911DF5
:1036F000201F5B9F900D211DAB9F200DB1E0BB24CF
:10370000CC24DD24639FD018C108B00AB00B739F8E
:10371000C018B108B00B839FB018B109699FC018D9
:10372000B108B00B799FB018B109899FB019629F99
:10373000B018B109729FB019D61AC70AB80A20F09A
:10374000B1E03B0F901F201F1124792F632F90E0D1
:10375000822F0F900F900F900F900F90DF91CF91CD
:103760001F910F91FF90EF90DF90CF90BF90AF909F
:103770009F900895AF92BF92CF92DF92EF92FF9207
:103780000F931F93CF93DF93C1EBDCE004E019E0CC
:1037900081ECA82E8CE0B82EC12CD12C7601C394DC
:1037A00069917991899199910F94BB2A28893989D6
:1037B0004A895B890F941C2B0F94F932F8016193AD
:1037C0007193819391938F01C616D706E806F90687
:1037D00010F46B017C01AC16BD0611F76FEF7FEFA3
:1037E000CB01A70196010F94FA302093140930936E
:1037F00015094093160950931709DF91CF911F9136
:103800000F91FF90EF90DF90CF90BF90AF90089511
:10381000CF92DF92EF92FF9280912008882309F4E3
:1038200057C0C0901C08D0901D08E0901E08F09072
:103830001F0820E030E0A901C701B6010F94B62AA5
:10384000882309F445C020E030E040E05FE3C70191
:10385000B6010F941C2B9B01AC010F941C2B2BED7C
:103860003FE049E450E40F941C2B9B01AC0160E065
:1038700070E080E89FE30F9480326B017C01C0927E
:10388000AD0CD092AE0CE092AF0CF092B00C609107
:103890007D0270917E02072E000C880B990B0F940D
:1038A000BD2A2AE037ED43E25CE30F941C2BA7010D
:1038B00096010F941C2B6093790270937A02809387
:1038C0007B0290937C02FF90EF90DF90CF90089561
:1038D000C12CD12C80E8E82E8FE3F82ED0CF0F93A7
:1038E0001F93CF93DF9350E0FC01E40FF51F80811D
:1038F000440F551F440F551F42545A4FEA01882365
:1039000029F188819981AA81BB81EB010881198104
:103910002A813B810097A105B10569F40C591F4F1D
:103920002F4F3F4FDA010D931D932D933C93139727
:103930008FEF808306C0081B190B2A0B3B0B37FD4A
:10394000F7CFDF91CF911F910F91089518821982BF
:103950001A821B82F6CFCF93DF9324E0829FC001AF
:103960001124EC01C950D74FFC01E35DF74F8F5D87
:10397000974FDC012D913D914D915C91608171815A
:10398000828193810F948631688379838A839B83B4
:10399000DF91CF9108958091B9059091BA05A091DA
:1039A000BB05B091BC058093490290934A02A09355
:1039B0004B02B0934C028091B7059091B80590935B
:1039C000800280937F0208958091490290914A027B
:1039D000A0914B02B0914C028093B9059093BA0527
:1039E000A093BB05B093BC0580917F0290918002AB
:1039F0009093B8058093B70584E690E09093800299
:103A000080937F0208958091FC129091FD12891B92
:103A1000877089F48091040E81110DC08091F90C9A
:103A20009091FA0C892B39F481E09091C70691119D
:103A300003C080E0089581E00895CF93DF93DB0118
:103A4000F9019C919130C1F0943080F094509C9396
:103A50008830D1F480819181009771F00197918332
:103A60008083480F591FEA01188206C08C3539F44B
:103A70009C5F9C93943041F4DF91CF9108958B33F8
:103A800039F781E08C93F8CF20813181B9016F5FE4
:103A90007F4F71836083420F531FEA0188838081C7
:103AA00091818F3591056CF7E7CF0F931F9381E0DC
:103AB0000091B0141091B1142091B2143091B3144C
:103AC0004091AC145091AD146091AE147091AF144C
:103AD000041715072607370708F480E01F910F9198
:103AE000089590E080E00895282F90911B0883307E
:103AF00021F495FD0FC094FD0FC0892F90E0B0E038
:103B0000A0E004C0B695A795979587952A95D2F71A
:103B10008170089581E0089580E00895FC01659129
:103B200075918591949108958F929F92AF92BF92D3
:103B3000CF92DF92EF92FF92CF93DF93EC018090D0
:103B4000F3089090F408A090F508B090F60820E0F3
:103B500030E0A901C501B4010F94B62A882309F405
:103B600054C0C880D980EA80FB80A7019601C501B6
:103B7000B4010F94B62A18160CF04CC02091EB0833
:103B80003091EC084091ED085091EE08C701B60164
:103B90000F94B62A882331F1C092EB08D092EC083A
:103BA000E092ED08F092EE082091EF083091F008D5
:103BB0004091F1085091F208688179818A819B8156
:103BC0000F941C2B9B01AC0160E070E080E89FE348
:103BD0000F94853160930F0270931002809311024D
:103BE0009093120260910F02709110028091110265
:103BF00090911202DF91CF91FF90EF90DF90CF90E4
:103C0000BF90AF909F908F90089560E070E080E843
:103C10009FE3F0CF60E070E0CB01ECCFCF92DF927A
:103C2000EF92FF92CF93DF93EC01CC80DD80EE80AA
:103C3000FF8027E137EB41ED58EBC701B6010F9448
:103C4000E63387FD23C023E030E044EB53E4C701B3
:103C5000B6010F94B62A1816CCF0C880D980EA8035
:103C6000FB8027E137EB41ED58EBC701B6010F941C
:103C7000E63387FD0BC0C1E023E030E044EB53E4C2
:103C8000C701B6010F94B62A18160CF4C0E08C2FA9
:103C9000DF91CF91FF90EF90DF90CF9008952FEBC1
:103CA000280F2A3108F047C0E22FF0E08091530539
:103CB00090915405A0915505B091560504C0B69554
:103CC000A795979587952A95D2F780FD02C08170B8
:103CD0000895EB5CFA4FE081EE2341F18091AD074E
:103CE0009091AE07E80FF92FF11D808190ED980FAC
:103CF0009A3030F08E3251F4818180538A3098F4BA
:103D0000F0932405E093230581E008958D3211F0AE
:103D10008B3249F4818190ED980F9A3088F38E327E
:103D200011F48281EACFF0E0E0E0EACF10922405BE
:103D300010922305E9CF80E008950E944F1E88234A
:103D400041F081E02091230530912405232B09F4D3
:103D500080E008958F929F92AF92BF92CF92DF92B0
:103D6000EF92FF92C090F505D090F605E090F70530
:103D7000F090F80520E030E0A901C701B6010F94EA
:103D8000B62A8823E1F1A701960160E070E080E89F
:103D90009FE30F9480326B017C018090F905909035
:103DA000FA05A090FB05B090FC0520E030E0A901E9
:103DB000C501B4010F94B62A882329F1A501940105
:103DC00060E070E080E89FE30F948032C092FC04D2
:103DD000D092FD04E092FE04F092FF04609300058F
:103DE000709301058093020590930305FF90EF9077
:103DF000DF90CF90BF90AF909F908F900895C12C8F
:103E0000D12C7601CACF60E070E0CB01DFCF129AEF
:103E100008955F9A8091AB0C8E7F8093AB0C8A9A49
:103E20008091AB0C8D7F8093AB0C809108018095C5
:103E30008170809306018091AB0C8B7F8093AB0CDB
:103E40000C94071F269A2E9A0895833B21E092072F
:103E500014F083EB91E090936112809360120C94C4
:103E600076E9E1E3F6E01082118212821382148275
:103E70000C9476E94F925F926F927F928F929F920D
:103E8000AF92BF92CF92DF92EF92FF920F931F9368
:103E9000CF93DF93EC012091ED053091EE05409139
:103EA000EF055091F005688179818A819B810F949B
:103EB00085316B017C012091F1053091F205409133
:103EC000F3055091F4056C817D818E819F810F9463
:103ED00085314B015C01A70196016091030270914D
:103EE000040280910502909106020F94B62A88235D
:103EF00009F450C0C0920302D0920402E09205027D
:103F0000F09206022091FC043091FD044091FE04E1
:103F10005091FF04C701B6010F941C2B2B013C01EB
:103F20000F9428336B017C0120E030E0A9010F944D
:103F3000B62A87FD70C020E030E040E450E4C701BD
:103F4000B6010F94E63318162CF4C12CD12CC0E422
:103F5000EC2EFE2CA7019601C301B2010F9485310E
:103F60006093F4047093F5048093F6049093F7043F
:103F7000C701B6010F94F2326093F204062E000CD2
:103F8000770B6F5F7F4F6430710514F064E070E071
:103F90006093F004D09101021091F204A501940104
:103FA00060910702709108028091090290910A02C3
:103FB0000F94B62A811133C0D11381C02091D80447
:103FC0003091D9044091DA045091DB046091F404FB
:103FD0007091F5048091F6049091F7040F941C2BD6
:103FE0002091DC043091DD044091DE045091DF0427
:103FF0000F948631DF91CF911F910F91FF90EF9039
:10400000DF90CF90BF90AF909F908F907F906F90F8
:104010005F904F900895C12CD12C76019BCF809258
:10402000070290920802A0920902B0920A0220911F
:104030000005309101054091020550910305C5012D
:10404000B4010F941C2B4B015C010F9428336B01BE
:104050007C0120E030E0A9010F94B62A87FDF3C06F
:1040600020E030E040E450E4C701B6010F94E633AD
:1040700018162CF4C12CD12CB0E4EB2EFE2CA70189
:104080009601C501B4010F9485316093F8047093D3
:10409000F9048093FA049093FB04C701B6010F94CE
:1040A000F2326093F304062E000C770B6F5F7F4FA4
:1040B0006430710514F064E070E06093F104C09125
:1040C000F304D11305C0809102028C1709F470C06B
:1040D0008091F2049091F304909302028093010284
:1040E0000C2E000CDD0B25E01203C0011124FC0195
:1040F000EC0FFD1FEE0FFF1FEE0FFF1FE954F84FEF
:1041000020813181428153812093EC043093ED046E
:104110004093EE045093EF040091F104002E000C44
:10412000110BFC01E00FF11FEE0FFF1FEE0FFF1F41
:10413000E954F84F60817181828193810F948531B8
:104140006093E8047093E9048093EA049093EB048D
:104150002091F00435E02303F0011124CE0FDF1F7E
:10416000CC0FDD1FCC0FDD1FC954D84F28813981FA
:104170004A815B812093E4043093E5044093E60494
:104180005093E704E00FF11FEE0FFF1FEE0FFF1F2C
:10419000E954F84F60817181828193810F94853158
:1041A0006093E0047093E1048093E2049093E3044D
:1041B0008090F8049090F904A090FA04B090FB0469
:1041C0002091E8043091E9044091EA045091EB0415
:1041D000C501B4010F941C2B2091EC043091ED0427
:1041E0004091EE045091EF040F9486316B017C01F5
:1041F000C092DC04D092DD04E092DE04F092DF0491
:104200002091E0043091E1044091E2045091E304F4
:10421000C501B4010F941C2B2091E4043091E504F6
:104220004091E6045091E7040F948631A70196016E
:104230000F9485316093D8047093D9048093DA0485
:104240009093DB04BBCEC12CD12C760118CFCF923A
:10425000DF92EF92FF92CF93DF93EC0108960E94DA
:10426000941D6B017C0120E030E0A9010F94B62A77
:1042700020E030E0A901882359F0CE010E943A1FC6
:104280009B01AC01C701B6010F941C2B9B01AC0133
:10429000688579858A859B850F94853168877987BC
:1042A0008A879B87DF91CF91FF90EF90DF90CF902F
:1042B00008952F923F924F925F926F927F928F92CA
:1042C0009F92AF92BF92CF92DF92EF92FF920F93A5
:1042D0001F93CF93DF93D62FC72FFC01808091804F
:1042E000A280B380C501B40120E831E541E050E08F
:1042F0000F94FA30C9016DE671E00F9469316B01DA
:104300007C01C501B40120E13EE040E050E00F94A3
:10431000FA30CA01B90128E130E040E050E00F94E2
:10432000FA30362E272E062F172F8CE3482E512CCD
:10433000612C712CC501B401A30192010F94FA30D4
:10434000B62EA72ECA01B901A30192010F94FA302B
:10435000CB01C114D10479F1AF92BF927F936F93D7
:104360002F923F92FF92EF92DF92CF928EE897E1E9
:104370009F938F93CF93DF930F944D2A8DB79EB762
:104380000E960FB6F8949EBF0FBE8DBF8D2F9C2F3B
:10439000DF91CF911F910F91FF90EF90DF90CF9021
:1043A000BF90AF909F908F907F906F905F904F9055
:1043B0003F902F900895E114F104C9F0AF92BF929D
:1043C0007F936F932F923F92FF92EF928EE797E148
:1043D0009F938F93CF93DF930F944D2AEDB7FEB742
:1043E0003C960FB6F894FEBF0FBEEDBFCFCF012BAA
:1043F000B9F0AF92BF927F936F932F923F9282E773
:1044000097E19F938F93CF93DF930F944D2A8DB7AE
:104410009EB70A960FB6F8949EBF0FBE8DBFB6CF5B
:10442000892BA9F0AF92BF927F936F938AE697E1B1
:104430009F938F93CF93DF930F944D2AEDB7FEB7E1
:1044400038960FB6F894FEBF0FBEEDBF9FCFAF9268
:10445000BF9286E697E19F938F93CF93DF930F945C
:104460004D2A0F900F900F900F900F900F908ECFBE
:10447000EF92FF920F931F93CF93DF93CDB7DEB7E9
:104480008C01EDB6FEB60F94032A01962DB73EB708
:10449000281B390B0FB6F8943EBF0FBE2DBF8DB74A
:1044A0009EB70196B8010F94FC290F94DF1B0FB63D
:1044B000F894FEBE0FBEEDBEDF91CF911F910F911C
:1044C000FF90EF9008958C38910514F08CE890E0FF
:1044D0009093F6118093F5110C9454C1AB01BC017B
:1044E0004093B0145093B1146093B2147093B3140A
:1044F00088E196E10C940CB22F923F924F925F921A
:104500006F927F928F929F92AF92BF92CF92DF92E3
:10451000EF92FF920F931F93CF93DF93CDB7DEB748
:1045200060970FB6F894DEBF0FBECDBF8B876C8748
:10453000042F122F282F30E03E872D87462F50E082
:104540005A87498785E0982E929EC001939E900DD0
:104550001124988B8F87FA01E80FF91FEE0FFF1FC8
:10456000EE0FFF1FE954F84F6081718182819381C2
:104570009B01AC010F947834882309F445C14B8525
:10458000400F6C85610F949EC0011124E985FA8566
:10459000E80FF91FEE0FFF1FEE0FFF1FE954F84F52
:1045A000C080D180E280F380040F909EA00111248E
:1045B000E985FA85E40FF51FEE0FFF1FEE0FFF1FD1
:1045C000E954F84F0081918082807380262F30E07B
:1045D000EF85F889E20FF31FEE0FFF1FEE0FFF1FAD
:1045E000E954F84F20807181798372817A837381D5
:1045F0007B83610F70E0EF85F889E60FF71FEE0F00
:10460000FF1FEE0FFF1FE954F84FF88BEF87F08183
:10461000FC83EF85F889F181FD83EF85F889F281CC
:10462000FE83EF85F889F381FF83FC01E20FF31F1E
:10463000EE0FFF1FEE0FFF1FE954F84F2081288770
:10464000A180B2806380FA01E60FF71FEE0FFF1F13
:10465000EE0FFF1FE954F84F4080518032801381E4
:10466000202F392D482D572D602F792D882D972DEE
:104670000F947834882321F000E0912C812C712C48
:104680009601A701B601C7010F947834882321F061
:10469000C02ED92CE82CF72C2C813D814E815F81D6
:1046A0006C817D818E819F810F947834882321F0E5
:1046B0001C821D821E821F82222D39814A815B81CC
:1046C000622D79818A819B810F947834882339F017
:1046D0002C803D8139834E814A835F815B839201C7
:1046E000432D512FB201832D912F0F9478348823BD
:1046F00021F0412C512C312C10E028853A2D4B2DE6
:10470000562D68857A2D8B2D962D0F94783488231D
:1047100021F04886A52CB32C612E85E02D853E85A1
:10472000829FF001839FF00D112449855A85E40F83
:10473000F51FEE0FFF1FEE0FFF1FE954F84FFA872A
:10474000E9879601A701B601C7010F948631202F92
:10475000392D482D572D0F9485316B017C01222D69
:1047600039814A815B81622D79818A819B810F9495
:1047700086312C813D814E815F810F9485319B0173
:10478000AC01C701B6010F9486316B017C0128850D
:104790003A2D4B2D562D68857A2D8B2D962D0F9405
:1047A00086319201432D512F0F9485319B01AC012D
:1047B000C701B6010F94863120E030E040E450E4B8
:1047C0000F948032E985FA856083718382839383B5
:1047D0006C858B8560960FB6F894DEBF0FBECDBF9B
:1047E000DF91CF911F910F91FF90EF90DF90CF90CD
:1047F000BF90AF909F908F907F906F905F904F9001
:104800003F902F900D941F1A60960FB6F894DEBF5C
:104810000FBECDBFDF91CF911F910F91FF90EF9011
:10482000DF90CF90BF90AF909F908F907F906F90D0
:104830005F904F903F902F90089580912305909125
:104840002405009731F04AE050E070E060E00D94FC
:10485000D12860E070E0CB0108958091230590910C
:104860002405009731F04AE050E070E060E00D94DC
:10487000A32760E070E0CB010895CF93DF93EB01B5
:104880000E949D1E882319F00E942D24EB01CE0169
:10489000DF91CF9108950E942D2497FD0CC00E94B6
:1048A0002D246F3F71058105910509F034F40E94B4
:1048B0002D24862F089580E008958FEF0895CF93DB
:1048C000C62F0E949D1E882319F0CF910C944B2473
:1048D0008C2FCF9108958091230590912405892BE9
:1048E00041F00E944B2491E0811101C090E0892F9A
:1048F000089591E0FCCFCF93DF93C82FD62F0E946D
:104900009D1E882321F0DF91CF910C946B248C2F76
:104910000E944F1E811101C08D2FDF91CF9108950C
:104920000E942D24CB010895CF93DF93EB010E94C9
:104930009D1E882321F0DF91CF910C949024CE010D
:10494000DF91CF9108950F931F93CF93809123050B
:10495000909124050097E9F0FC018F01C1912C2F63
:104960002F7D81F0C53411F0C536B9F7F8011082FA
:1049700070E060E00F944526F801C083CF911F914D
:104980000F91089570E060E0CF911F910F910D9409
:10499000452660E070E0CB01F1CFCF92DF92EF923D
:1049A000FF926A017B010E949D1E882331F0FF90D7
:1049B000EF90DF90CF900C94A324C701B601FF9035
:1049C000EF90DF90CF9008954F925F926F927F9219
:1049D0008F929F92AF92BF92CF92DF92EF92FF920F
:1049E0001F93CF93DF9300D01F92CDB7DEB719820C
:1049F0001A821B821C82CE0101964C018BE9C82EC3
:104A000087E0D82E99E6E92E92E0F92E27EFA22E24
:104A100028E0B22E10E088E5810F0E949D1EF4016F
:104A200081934F01882309F4E0C00E94A3242B0145
:104A30003C01812F0E94741D882309F4CCC0F7012A
:104A40002081318142815381C301B2010F948631AB
:104A5000F60160837183828393831F5FF4E0CF0E3E
:104A6000D11C84E0E80EF11C94E0A90EB11C1330B7
:104A700091F685E40E949D1E8C83882309F4C0C0B2
:104A80000E94A3246B017C0183E00E94741D882393
:104A900071F0209175023091760240917702509129
:104AA0007802C701B6010F9486316B017C01C09278
:104AB000A707D092A807E092A907F092AA078091D1
:104AC000EC05882359F18091B41482FF27C08C81B2
:104AD000882321F18981811103C08A818823F1F023
:104AE0002DEC3CEC4CE45DE360914208709143088E
:104AF00080914408909145080F9486319B01AC0148
:104B000060917102709172028091730290917402AF
:104B10000F94E633181614F40F94651940E050E032
:104B2000BA0186E40E94CD2420E030E0A9010F9470
:104B3000E633181684F40E94A32420E030E040E716
:104B400052E40F9480326093490270934A0280933A
:104B50004B0290934C028091690C83FD28C0809198
:104B6000B206882321F1209175023091760240919E
:104B70007702509178026091A7077091A807809101
:104B8000A9079091AA070F9485312091BF06309113
:104B9000C0064091C1065091C2060F9486316093C1
:104BA000BF067093C0068093C1069093C2060F9013
:104BB0000F900F900F90DF91CF911F91FF90EF908A
:104BC000DF90CF90BF90AF909F908F907F906F902D
:104BD0005F904F900895F50120813181428153818A
:104BE000C301B2010F94853133CFF70180819181E8
:104BF000A281B381F60180839183A283B3832DCFF9
:104C00008091750290917602A0917702B09178021E
:104C10008093A7079093A807A093A907B093AA072A
:104C20004ECFCF92DF92EF92FF926B017C0183E334
:104C3000C816D104E104F10470F082E3C81AD10867
:104C4000E108F10862E370E080E090E00E948DA945
:104C50000E94CEC4ECCFC701B6010E948DA9FF907F
:104C6000EF90DF90CF900C94CEC4CF92DF92EF9272
:104C7000FF920F931F93CF93DF936B017A01EC01A7
:104C8000C854DB4F28813CE0389F8001399F100DCC
:104C9000112427FF24C0FB011182108288818F5FBD
:104CA000888388819801280F311D87FD3A95C901B5
:104CB0002091E712F6012817190629F024F08881BF
:104CC0008C300CF43CC080819181049680349C49E6
:104CD00008F475C0F60180819181049672C08881C4
:104CE0009801280F311D87FD3A95C9012091E712DF
:104CF0002817190699F294F28881A801480F511DCE
:104D000087FD5A95FA01EE0FFF1FE40FF51FE156DC
:104D1000FD4E808187FFC2CF8881F801E80FF11D29
:104D200087FDFA95CF01EE0FFF1FE80FF91FE1563F
:104D3000FD4E808160E08F770E94E8A7AFCF808131
:104D400091812881A801420F511D27FD5A959A0192
:104D5000FA01EE0FFF1FE20FF31FE156FD4E218116
:104D60003281820F931FF70191838083888198019C
:104D7000280F311D87FD3A95F901EE0FFF1FE20F55
:104D8000F31FE156FD4E808187FF20C08881080F08
:104D9000111D87FD1A95F801EE0FFF1FE00FF11F9F
:104DA000E156FD4E808161E08F77DF91CF911F91B9
:104DB0000F91FF90EF90DF90CF900C94E8A780E4E4
:104DC0009CE9F701918380838FEF8883DF91CF91F6
:104DD0001F910F91FF90EF90DF90CF9008950F9368
:104DE0001F93CF93DF9305EC1CE0C9EDD1E1F801EF
:104DF00021913191419151918F0160E070E080E803
:104E00009FE30F9480326993799389939993F1E1A9
:104E1000C93EDF0761F70F94A417DF91CF911F916F
:104E20000F910C94BA1BCF92DF92EF92FF92CF9327
:104E3000DF932091AC0C222329F1EC0108960E940B
:104E4000941D6B017C0120E030E0A9010F94B62A8B
:104E500020E030E0A901882359F0CE010E943A1FDA
:104E60009B01AC01C701B6010F941C2B9B01AC0147
:104E7000688579858A859B850F94863168877987CF
:104E80008A879B87DF91CF91FF90EF90DF90CF9043
:104E900008952F923F924F925F926F927F928F92DE
:104EA0009F92AF92BF92CF92DF92EF92FF920F93B9
:104EB0001F93CF93DF93CDB7DEB76C970FB6F894FF
:104EC000DEBF0FBECDBF8C015B015A834983FC015D
:104ED000EF5AFF4F208131814281538129873A87E0
:104EE0004B875C87CA01B9010F94BB2A6B017C0117
:104EF000D5012D913D914D915C910F941C2B0F94F8
:104F000064322B013C01E981FA81208131814281A7
:104F10005381C701B6010F941C2B0F9464324B01CF
:104F20005C01C301B2010F94F932698B7A8B8B8BD0
:104F30009C8B683771058105910540F428E730E0C6
:104F400040E050E0298B3A8B4B8B5C8BC501B40160
:104F50000F94F9326D877E878F87988B683771053C
:104F60008105910540F448E750E060E070E04D872E
:104F70005E876F87788BF801E35AFF4F408051803E
:104F800062807380C301B2010F94BD2A69837A8362
:104F90008B839C8369897A898B899C890F94BB2A2E
:104FA0006D8B7E8B8F8B988F20E030E0A90169811B
:104FB0007A818B819C810F94B62A882309F4E1C100
:104FC000A7019601C701B6010F941C2B4B015C0190
:104FD0002D893E894F89588DCA01B9010F941C2B28
:104FE0009B01AC01C501B4010F9485314B015C01FB
:104FF00029813A814B815C81CA01B9010F948631C4
:105000009B01AC01C501B4010F9480320F9464324E
:105010000F94F9326D837E838F8398876627772775
:10502000CB0164197509860997090F94BD2A4B01B4
:105030005C016D857E858F8598890F94BB2A2B0135
:105040003C0120E030E0A901C501B4010F94B62A6B
:10505000882309F49AC1A3019201C301B2010F94FC
:105060001C2B698F7A8F8B8F9C8FA7019601C701AC
:10507000B6010F941C2B9B01AC01698D7A8D8B8D31
:105080009C8D0F9485316B017C01A5019401C501B4
:10509000B4010F9486319B01AC01C701B6010F9496
:1050A00080320F942833D80195968D909D90AD90C5
:1050B000BC909897750164012D813E814F81588580
:1050C000C21AD30AE40AF50A0F94F932C61AD70AAB
:1050D000E80AF90AF7FE8EC02D893E894F89588D5E
:1050E000CA01B9010F941C2B6B017C0129813A8103
:1050F0004B815C81CA01B9010F94863169877A8737
:105100008B879C8720E030E0A90169817A818B81BF
:105110009C810F94B62A882309F43BC1C501B401D0
:105120000F94BB2A29853A854B855C850F941C2BEF
:10513000A70196010F9485316D837E838F839887B5
:10514000A3019201C301B2010F941C2B9B01AC017E
:105150006D817E818F8198850F9486312B013C0172
:1051600020E030E040E850E469817A818B819C81C5
:105170000F941C2B9B01AC01C301B2010F94803230
:105180000F9464322B013C0120E030E0A9010F9420
:10519000E63318161CF0412C512C3201C301B20128
:1051A0000F94F9326D837E838F83988786169706D6
:1051B000A806B90620F48D829E82AF82B8866D81E2
:1051C0007E818F8198850F94BB2A29853A854B85EE
:1051D0005C850F941C2BA70196010F9486310F94C8
:1051E00034340F94F93269877A878B879C87C12C76
:1051F000D12C760169857A858B859C8529893A89A8
:105200004B895C89621B730B840B950B0F94BB2A33
:1052100029813A814B815C810F94803220E034E215
:1052200044EF59E40F941C2B0F94F9324B015C01AD
:1052300069857A858B859C852D853E854F85588926
:10524000621B730B840B950B0F94BB2A29813A8147
:105250004B815C810F94803220E034E244EF59E4CA
:105260000F941C2B0F94F9322B013C013FE683165F
:105270009104A104B10408F090C0F401EE0FFF1FE7
:10528000EE0FFF1FE553F64E85919591A591B491D0
:105290008983292E3A2EBD8B4FE6441651046104B2
:1052A000710408F083C0F201EE0FFF1FEE0FFF1F25
:1052B000E553F64E45915591659174919A01CB0154
:1052C0004D815E816F817885D80199964D935D936C
:1052D0006D937C939C974C0D5D1D6E1D7F1DF80199
:1052E00045A756A767A770ABEB5AFF4F49895A8964
:1052F0006B897C894083518362837383D5968D92B9
:105300009D92AD92BC92D897F80141AE52AE63AE79
:1053100074AEFD9649814083218232825D89538338
:105320003496208331838283938369857A858B8544
:105330009C85D1966D937D938D939C93D49778960D
:105340002D853E854F855889208331834283538341
:105350006C960FB6F894DEBF0FBECDBFDF91CF9134
:105360001F910F91FF90EF90DF90CF90BF90AF9083
:105370009F908F907F906F905F904F903F902F9075
:10538000089560E070E0CB0141CE60E070E0CB01B9
:1053900088CE60E070E0CB01F3CEC501B4010E947D
:1053A000BC1A6983272E382E9D8B76CFC301B2019C
:1053B0000E94BC1A9B0184CF8091FC129091FD1237
:1053C000891B877019F490E080E008959091F9129C
:1053D000992351F0833030F48FEF890F19F08093C7
:1053E000F912F1CF1092F9128091FD1227E6829FF7
:1053F000C00111248F5C964FFC01208120FDE3CF7A
:105400002091FD122F5F27702093FA123091FD1228
:105410002091FB12321304C02091FA122093FB1248
:10542000089590916F0081E091FD02C080E00895A1
:1054300090916F009D7F90936F00089580FF04C04E
:105440009091AB0C90FD8E7F81FF05C09091AB0CCD
:10545000969590FD8D7F82FF06C09091AB0C96953E
:10546000969590FD8B7F08958F929F92AF92BF92F9
:10547000CF92DF92EF92FF92CF93DF9320914D0274
:10548000222309F49EC0EC018091BD05C82ED12CC9
:10549000F12CE12C80FF2CC080904F0290905002A4
:1054A000A0905102B0905202288139814A815B81DB
:1054B000C501B4010F94E633181624F4888299824A
:1054C000AA82BB8280905B0290905C02A0905D02F9
:1054D000B0905E02288139814A815B81C501B401A7
:1054E0000F94B62A87FF04C088829982AA82BB8261
:1054F000D701C601B695A7959795879580FF2CC0D3
:105500008090530290905402A0905502B0905602A1
:105510002C813D814E815F81C501B4010F94E6333A
:10552000181624F48C829D82AE82BF8280905F0226
:1055300090906002A0906102B09062022C813D8147
:105540004E815F81C501B4010F94B62A87FF04C064
:105550008C829D82AE82BF8282E0F694E794D794DB
:10556000C7948A95D1F7C0FE2CC0C0905702D09046
:105570005802E0905902F0905A02288539854A85F0
:105580005B85C701B6010F94E633181624F4C8866C
:10559000D986EA86FB86C0906302D0906402E090D0
:1055A0006502F0906602288539854A855B85C701CA
:1055B000B6010F94B62A87FF04C0C886D986EA864A
:1055C000FB86DF91CF91FF90EF90DF90CF90BF905F
:1055D000AF909F908F900895CF92DF92EF92FF92BD
:1055E0000F931F93C12CD12C76018C0125E732E05B
:1055F00041E752E06DE672E089E692E00F944500E3
:105600001F910F91FF90EF90DF90CF9008950D9430
:10561000A4178091AA05659B6EC080618093AA053E
:10562000909103018091AA0591FF67C080628093E9
:10563000AA058091AA054B9B62C084608093AA054D
:105640008091AA059091A905981709F45AC092E093
:105650009093A8058093A9058091C406811105C087
:105660008091AB07882309F459C08091110680FF0F
:1056700010C08091C50680FD0CC08091A70584FFF5
:1056800008C08091070780618093070780E00E942F
:1056900058CD80911106869580FF11C08091C50676
:1056A000869580FD0CC08091A70585FF08C080917C
:1056B000070780628093070781E00E9458CD8091A0
:1056C00011068695869580FF29C08091C50686952E
:1056D000869580FF23C08091AB078823F9F08091E5
:1056E000A70582FF1BC0809107078460809307078E
:1056F00082E00C9458CD8F7E91CF8F7D98CF8B7F99
:105700009DCF8091A805882309F4A6CF815080936E
:10571000A8058111A1CF9093A7059ECF08958091F0
:10572000C406811104C08091AB07882331F062E088
:1057300070E080E090E00C94112608950F931F9381
:1057400080919711813019F50E94C0A90091C6057A
:105750001091C7052091C8053091C905601B710BD8
:10576000820B930B28EE33E040E050E00F94FA30C8
:105770006091CA057091CB058091CC059091CD05C3
:10578000620F731F841F951F1F910F9108956091E1
:10579000CE057091CF058091D0059091D105D6CFDF
:1057A000109297111092C6051092C7051092C80565
:1057B0001092C9051092CE051092CF051092D00517
:1057C0001092D1051092CA051092CB051092CC050B
:1057D0001092CD050895CF92DF92EF92FF92CF9372
:1057E000DF93C62FFC01C080D180E280F38020E0EF
:1057F00030E0A901C701B6010F94B62A20E030E0DD
:10580000A90187FD14C020E030E048EC52E4C70154
:10581000B6010F94E63324E630E040E050E018167D
:1058200034F0C701B6010F94F2329B01AC01C230D3
:10583000A0F4D0E0C45DD64FAFEFB0E00F943B31A1
:1058400024E630E040E050E00F941C312F3F31055A
:1058500019F010F02FEF30E02883DF91CF91FF9007
:10586000EF90DF90CF9008958091090180FD06C0F0
:105870008091B41483FB882780F9089580E008950F
:10588000CF92DF92EF92FF92FC01C080D180E28044
:10589000F380663019F51092360610923706109292
:1058A00038061092390610923A060E9454C120E040
:1058B00030E0A901C701B6010F94B62A87FF1DC0C9
:1058C000C12CD12C7601C701B6010F94F333CB0163
:1058D000FF90EF90DF90CF900C9463220E94311FD5
:1058E00020E030E0A901C701B6010F94B62A87FF76
:1058F00015C0C12CD12C760122C020E030E04CE054
:1059000053E4C701B6010F94E6331816E4F6C12C30
:10591000D12C9CE0E92E93E4F92ED5CF20E030E89D
:1059200049ED53E4C701B6010F94E63318163CF471
:10593000C12C80E8D82E89EDE82E83E4F82EC7012B
:10594000B6010F94F333CB01FF90EF90DF90CF902F
:105950000C94251F9091AB0C977081E0973009F063
:1059600080E008952091A50520FF14C020E83EE3C3
:10597000629FA001639F500D729F500D1124CA01B8
:105980009695879596958795009731F08A950000B2
:10599000E9F708950C9411260895CF93DF931092A0
:1059A0006A0C1092FD0C1092FF0C1092FE0C1092DB
:1059B000A4051092A305CFEFDFEF8091B41485FD0D
:1059C00007C00E946DADD0933313C0933213F5CF4F
:1059D0008FEF9FEF9093331380933213DF91CF912A
:1059E00008958F929F92AF92BF92CF92DF92EF92E3
:1059F000FF920F931F93CF93DF931092580510924D
:105A000057052FE32093520510925105109250052F
:105A100010924F051092530510925405109255059F
:105A2000109256059C01F90190812F5F3F4F9032F3
:105A3000D1F39E34C9F4818190ED980F9A3020F013
:105A40008D3211F08B3281F432969F012F5F3F4FE0
:105A5000808180538A3008F47BC09F012F5F3F4FC5
:105A60008081803209F476C0F093AE07E093AD07F1
:105A70008F010F5F1F4FC0816AE270E0C8010F9471
:105A8000D434009731F0FC01319780818032E1F30A
:105A90001182CD3429F0C43519F0C73409F04BC058
:105AA000F80180810F5F1F4F8032D1F380538A301D
:105AB00008F041C0C093520530E020E04AE0DF0129
:105AC0001196429FC001439F900D11249C012053C9
:105AD00031098081280F311D87FD3A95818190ED34
:105AE000980F9A30C8F130935105209350058E32AB
:105AF00061F4329690E04AE0DF0131968C9150EDEE
:105B0000580F5A3058F190934F05CD01DC010196A2
:105B10004C914032D9F3CD3489F52E31310539F02D
:105B200018F52731310519F02C31310539F5B093CD
:105B30005805A0935705DF91CF911F910F91FF90CA
:105B4000EF90DF90CF90BF90AF909F908F9008958F
:105B5000F9017BCFF90181CFFD01B1CF949F800D79
:105B6000112490ED980FC8CF2537310538F027372D
:105B70003105E8F2203A83E03807C9F2D091AD0749
:105B800040E050E0BA0110E000E0C12CD12C7601D9
:105B9000C394FD0131968C91882309F47FC0813232
:105BA000E1F4CD34D1F420323105B9F440935305FA
:105BB000509354056093550570935605F09358051E
:105BC000E093570563E270E0CF010F94D43400975F
:105BD00009F4B1CFFC011082AECF81548A3108F0B4
:105BE00058C0DF019D91903291F0A0EDA90FAA302D
:105BF000E8F09E3271F4918190539A30B8F001151B
:105C0000110519F48F010150110990E013C0FD0135
:105C1000E8CF9D3211F09B3291F79181A0EDA90F51
:105C2000AA3020F09E3259F79281E6CF9E2F9D1B1D
:105C3000309759F3A82FB0E04601570104C0880CF3
:105C4000991CAA1CBB1C8A95D2F7482959296A2994
:105C50007B29AB5CBA4F9C9380818154DF018A31F0
:105C600008F497CFDF018191882309F492CF90ED5A
:105C7000980F9A30B8F393ED980F923098F38B32D7
:105C800089F3CD010196EC91E03209F082CFDC017D
:105C9000F8CF0115110501F78D01DECF10935805DE
:105CA0000093570540935305509354056093550551
:105CB0007093560540CF4F925F926F927F928F9272
:105CC0009F92AF92BF92CF92DF92EF92FF92CF93CB
:105CD000DF9300D000D01F921F92CDB7DEB75C01DA
:105CE000DB01CD90DD90ED90FC90E091F712F0910A
:105CF000F812FE83ED8384819581A681B781898323
:105D00009A83AB83BC839C01AD01C701B6010F949C
:105D100085312B013C01F50180809180A280B38008
:105D2000AD81BE818D919D910D90BC91A02D8D83F3
:105D30009E83AF83B88727E137EB41ED58EBC30172
:105D4000B2010F94E63387FDD1C023E030E044EB8D
:105D500053E4C301B2010F94B62A18160CF4C6C05E
:105D60002D813E814F815885C501B4010F94853145
:105D70002B013C0127E137EB41ED58EB0F94E63363
:105D800087FDB4C023E030E044EB53E4C301B2012B
:105D90000F94B62A18160CF4A9C020E030E0A9012F
:105DA0006D817E818F8198850F9486312B013C0116
:105DB00020E030E040E450E40F94B62A87FF05C0AD
:105DC000412C512C30E4632E762C27E137EB41ED4A
:105DD00058E3C301B2010F9485319B01AC01C501A9
:105DE000B4010F94E63387FD81C020E030E044EB3E
:105DF00053E46D817E818F8198850F9486312B01CC
:105E00003C0120E030E842EB53E40F94E6331816EF
:105E10003CF4412C20E8522E22EB622E23E4722E19
:105E200027E137EB41ED58E3C301B2010F9486310E
:105E30009B01AC01C501B4010F94B62A18160CF4ED
:105E400055C020E030E0A90169817A818B819C8175
:105E50000F9486314B015C0120E030E040EE51E4CC
:105E60000F94B62A87FF06C0812C912C90EEA92EA4
:105E700091E4B92E27E137EB41ED58E3C501B401B8
:105E80000F9485319B01AC01C701B6010F94E63335
:105E900087FD2CC020E030E044EB53E469817A8137
:105EA0008B819C810F9486314B015C0120E030E0B6
:105EB00046EA53E40F94E633181634F4812C912CFF
:105EC00086EAA82E83E4B82E27E137EB41ED58E3AC
:105ED000C501B4010F9486319B01AC01B1E0B983D7
:105EE000C701B6010F94B62A18160CF419828981DD
:105EF00028960FB6F894DEBF0FBECDBFDF91CF91CD
:105F0000FF90EF90DF90CF90BF90AF909F908F90D9
:105F10007F906F905F904F900895E9E3F8E082EBF7
:105F2000DF011D928A95E9F708958091EC058111B2
:105F300004C00E948D2F0C94CEBA8091B41482FDBF
:105F40000D946519089580913908882361F0909126
:105F5000EA08891308C08091B41483FF04C087E75E
:105F600098E00C9498B980E00895FC0123812111F8
:105F70000C94CDB50895EFE6F0E0808182608083D7
:105F80000895CF92DF92EF92FF92CF93DF93C82FC5
:105F90000E94112A94E0C99FE0011124FE01E15EF4
:105FA000F94FC080D180E280F38081110E94BB2F25
:105FB000C752DE4EC701B6010F94BD2A2881398130
:105FC0004A815B810F941C2BDF91CF91FF90EF9062
:105FD000DF90CF9008958F929F92AF92BF92CF9211
:105FE000DF92EF92FF921F93CF93DF93CDB7DEB78F
:105FF00060970FB6F894DEBF0FBECDBF182F80E0BC
:106000000E94C12F4B015C018092AB059092AC05C0
:10601000A092AD05B092AE0581E00E94C12F6B0148
:106020007C01C092AF05D092B005E092B105F0922C
:10603000B20582E00E94C12F6093B3057093B4054E
:106040008093B5059093B6051D861E861F86188A17
:1060500089829A82AB82BC82CD82DE82EF82F88610
:1060600069877A878B879C8783E00E94C12F6D8721
:106070007E878F87988B8091AC0C882321F0CE018E
:1060800001960E9427211E3FD9F480E1FE0131963E
:10609000A9E6B2E001900D928A95E1F760960FB6FD
:1060A000F894DEBF0FBECDBFDF91CF911F91FF905F
:1060B000EF90DF90CF90BF90AF909F908F9008951A
:1060C00084E0189FF0011124DF01A759BD4F81E042
:1060D00090E08C0F9D1FE80FF91F40815181628174
:1060E00073814D935D936D937C931397D7CFCF922C
:1060F000DF92EF92FF92CF93DF93C82F0E94112A75
:1061000094E0C99FE0011124FE01ED5EF94FC080CB
:10611000D180E280F38081110E94BB2FC752DE4EF6
:10612000C701B6010F94BD2A288139814A815B815C
:106130000F941C2BDF91CF91FF90EF90DF90CF90C9
:1061400008950E94112A9091FD129093FC12909351
:10615000FB129093FA1294E69093F91220ED33E03B
:106160003093300920932F0981110E94BB2F81E0C9
:10617000809312060895CF93DF93CDB7DEB72C97A7
:106180000FB6F894DEBF0FBECDBF0F9482180E94E9
:10619000112A9CE0EFE1F6E0DE01119601900D92EC
:1061A0009A95E1F781110E94BB2FCE0101960E94C2
:1061B00038CD2C960FB6F894DEBF0FBECDBFDF9161
:1061C000CF9108952F923F924F925F926F927F925C
:1061D0008F929F92AF92BF92CF92DF92EF92FF92F7
:1061E0000F931F93CF93DF9300D0CDB7DEB780908E
:1061F000690290906A02A0906B02B0906C0240908D
:106200006D0250906E0260906F0270907002C090AC
:106210007102D0907202E0907302F09074020E94BA
:10622000BA1B0E94081C0BEA1CE18FE492E09B83DE
:106230008A838FE9282E8CE1382E198289810E9469
:10624000AB1CC8010E948E1DEA81FB816193719392
:1062500081939193FB83EA83C1010E948E1DEA81A1
:10626000FB816087718782879387F981FF5FF9835C
:106270000C5F1F4F84E0280E311CF330F9F68DEFD0
:1062800095E00F94E7180E94AA1E0E94EF26A50130
:1062900094016091690270916A0280916B02909101
:1062A0006C020F94B62A81111CC0A3019201609167
:1062B0006D0270916E0280916F02909170020F9446
:1062C000B62A81110EC02091710230917202409164
:1062D000730250917402C701B6010F94B62A882345
:1062E000B9F00F900F900F90DF91CF911F910F9108
:1062F000FF90EF90DF90CF90BF90AF909F908F90E6
:106300007F906F905F904F903F902F900C94BB3098
:106310000F900F900F90DF91CF911F910F91FF90F1
:10632000EF90DF90CF90BF90AF909F908F907F9035
:106330006F905F904F903F902F9008958091ED1156
:106340009091EE11892B79F48091ED119091EE11DD
:10635000892B49F42091ED113091EE1181E0232B2E
:1063600019F480E0089581E0089510920905809164
:10637000220290912302A0912402B09125028093E1
:10638000090690930A06A0930B06B0930C06089595
:106390009091041210920412923071F0943079F0BE
:1063A000913099F4813089F480910905882369F04E
:1063B000109226020C94B5311092AA0C089582EB2B
:1063C00098E19093FA0C8093F90C08959091B4148D
:1063D00093FB882780F993FF06C081E090911B16FC
:1063E000911101C080E00895CF93C091A605CF77A9
:1063F00039F50E94E631882319F18091AC1490910F
:10640000AD14A091AE14B091AF140097A105B105E1
:10641000B9F0BC01CD016D597F4F8F4F9F4F24E6DE
:1064200030E040E050E00F94FA306091B014709189
:10643000B1148091B2149091B3140F94FA30C22F1A
:106440008C2FCF910895ECE2F9E01082118208952B
:1064500081E00895DC01EC918E2F90E0FC01EE0FBD
:10646000FF1FE80FF91FE156FD4E80818F77808373
:1064700008958F929F92AF92BF92CF92DF92EF9248
:10648000FF920F93CF93DF931F92CDB7DEB75C01DE
:106490007B0149016B01C40ED51EF50180819181FC
:1064A0000F94D4308983002311F0F7018083BE015B
:1064B0006F5F7F4FC4010E9460E9F5018081918187
:1064C000019691838083FFEFEF1AFF0AEC14FD041D
:1064D00021F780E00F90DF91CF910F91FF90EF9027
:1064E000DF90CF90BF90AF909F908F9008950F93C3
:1064F000AB010091010621E0022722E036E0BC0159
:1065000082EE95E00E9439320F910895009781F450
:106510001092900082E0809391001092950010926A
:106520009400C19A809171008260809371000895F7
:10653000019761F41092A00082E08093A100109274
:10654000A5001092A40089BB8093720008957F92E9
:106550008F929F92AF92BF92CF92DF92EF92FF9273
:106560000F931F93CF93DF93EC017B0188818831D8
:1065700008F0C3C090E0FC01EE0FFF1FE80FF91F09
:10658000E156FD4E80818F770E944CF019821A826D
:1065900088812CE0622F0F945D31829FB00111241D
:1065A00030E020E0AB01420F531FFA01EE0FFF1F56
:1065B000E40FF51FE156FD4E908197FD08C02F5F57
:1065C0003F4F2C30310571F790E00E948632788081
:1065D000072D10E06801CC0CDD1CF601E00FF11F67
:1065E000E156FD4E80818068808377FC86C080E222
:1065F000E81682E0F8060CF03FC08A8128E532E018
:10660000281B310987FD3395220F331F220F331FBB
:10661000032E000C440B550B898178E8872E912CB2
:10662000881A910887FD9394880C991C880C991CF2
:10663000092C000CAA08BB0860E070E0CB01F7FC55
:106640000AC0B701653B710514F064EB70E0072EDA
:10665000000C880B990B281939094A095B090F941A
:10666000EA3024EB30E040E050E00F941C31820E21
:10667000931EA41EB51E740187E18715D8F02981E9
:1066800088E890E0821B910927FD9395880F991F58
:10669000880F991FE816F90604F502972FB7F894AA
:1066A000E601C00FD11FC156DD4E880F991F9A8396
:1066B00089832FBF62E370E080E090E0DF91CF91AB
:1066C0001F910F91FF90EF90DF90CF90BF90AF9010
:1066D0009F908F907F900C9411262A8188E592E0FC
:1066E000821B910927FD9395880F991F880F991F89
:1066F000E816F90694F6C701D0CFDF91CF911F912C
:106700000F91FF90EF90DF90CF90BF90AF909F9050
:106710008F907F900895CF93DF93EB01682F70E007
:1067200088EE92E10E94A732688179818A819B81FB
:10673000643F21E072078105910520F464EF71E068
:1067400080E090E00E94112689B183FB882780F9C0
:10675000DF91CF910895CF93DF9300D01F92CDB7F3
:10676000DEB78EEE92E0A0E0B0E089839A83AB833F
:10677000BC83BE016F5F7F4F8AE50E948B330F9011
:106780000F900F900F90DF91CF910895CF93DF93EB
:1067900000D01F92CDB7DEB78EEE92E0A0E0B0E061
:1067A00089839A83AB83BC83BE016F5F7F4F8AE08E
:1067B0000E948B330F900F900F900F90DF91CF912D
:1067C0000895CF93DF9300D01F92CDB7DEB784EF4B
:1067D00091E0A0E0B0E089839A83AB83BC83BE01E3
:1067E0006F5F7F4F80EA0E948B330F900F900F9066
:1067F0000F90DF91CF9108951F920F920FB60F92D5
:1068000011240BB60F922F933F934F935F936F9387
:106810007F938F939F93AF93BF93EF93FF9348EA38
:1068200050E064EA70E081E090E00E943526FF913C
:10683000EF91BF91AF919F918F917F916F915F91F8
:106840004F913F912F910F900BBE0F900FBE0F9065
:106850001F9018951F920F920FB60F9211240BB62E
:106860000F922F933F934F935F936F937F938F93E9
:106870009F93AF93BF93EF93FF9348E950E064E990
:1068800070E090E080E00E943526FF91EF91BF918B
:10689000AF919F918F917F916F915F914F913F91B8
:1068A0002F910F900BBE0F900FBE0F901F90189559
:1068B0009091D10095FD0CC09091D00095FF08C03B
:1068C0008093D6008091D00080648093D00008959A
:1068D000209136042F5F2F770FB607FC27C09091C9
:1068E0003704921328C09091D00095FF1EC090915C
:1068F000370440913604941306C09091D1009F7DD7
:106900009093D10012C0E92FF0E0EA5CFB4F328196
:106910009F5F9F773093D600909337043091D000DB
:1069200030643093D000491741F3D9CF90913704A8
:10693000921301C0FBCFE0913604F0E0EA5CFB4F1C
:106940008283209336048091D10080628093D100AD
:1069500008958F929F92AF92BF92CF92DF92EF9263
:10696000FF920F931F93CF93DF937C0121E5E20EFB
:10697000F11CD7014C914A3509F0A4C06C01B2E575
:10698000CB0ED11CF6013081353A09F09BC0EC01E9
:10699000C05BDF4F2881233008F494C08C0100567F
:1069A0001F4FD8014C93E15BFF4F3083319620831A
:1069B000EF54F1093081E05BFF4F30833038B1F4A0
:1069C0003196AC54B1093C913083E854F109AF5A87
:1069D000BF4F50E040E02250330B42175307CCF436
:1069E000808132968D934F5F5F4FF7CF233031F523
:1069F000313809F074C0FC01EC55FF4FDC01AC5A92
:106A0000BF4F2C9120833196885A9F4FDC018C9187
:106A100080834801B12CA12C888190E002968A15D0
:106A20009B050CF43FC0F40181914F010E94583442
:106A30000E94A3E9FFEFAF1ABF0AEECF323821F56B
:106A4000FC01EC5AFF4F30814181E05BFF4F4083F6
:106A500031963083DC01AA55BF4F50E040E023500F
:106A6000330B42175307ACF6FA01EE7FE45AFF4F9F
:106A7000E80FF91F608171817C9311966C931197D7
:106A80004E5F5F4F1296EDCF243019F6333809F67A
:106A9000FC01EC5AFF4F20813181E05BFF4F3083D6
:106AA0003196B0CF80E5DE011D928A95E9F78AE143
:106AB000F80111928A95E9F78AE5D7018C9385EA66
:106AC000F6018083DF91CF911F910F91FF90EF909E
:106AD000DF90CF90BF90AF909F908F900895323805
:106AE00009F097CFADCFAF92BF92CF92DF92EF92E6
:106AF000FF920F931F93CF93DF93EC0184E6C82E90
:106B000080E2D82EE12CF12C02E8A12C90E2B92EE3
:106B100015E000934114C0924214D0924314E092C5
:106B20004414F0924514B0924B14A0924A1410935E
:106B30003E148EEE93E10E94A9348FEFC81AD80A52
:106B4000E80AF80A88E7C81680E2D806E104F104EA
:106B500001F724E630E240E050E0BE018EEE93E122
:106B6000DF91CF911F910F91FF90EF90DF90CF9029
:106B7000BF90AF900C94A8E9CF92DF92EF92FF9272
:106B80000F931F93CF93DF93CDB7DEB77C01CDB6C4
:106B9000DEB60F94032A01962DB73EB7281B390B9A
:106BA0000FB6F8943EBF0FBE2DBF0DB71EB70F5FD7
:106BB0001F4FB701C8010F94FC29F8010190002074
:106BC000E9F73197E01BF10B759720F083E992E02C
:106BD000F801848BC8010E9473350FB6F894DEBEAD
:106BE0000FBECDBEDF91CF911F910F91FF90EF901F
:106BF000DF90CF9008958F929F92AF92BF92CF92E5
:106C0000DF92EF92FF920F931F93CF93DF930E9437
:106C1000CD2C3AE0C32E30E2D32EE12CF12C15E03E
:106C200002E846015701CAE0D0E010924B141092DE
:106C30004A1410933E14009341148092421490928F
:106C40004314A0924414B09245148EEE93E10E9436
:106C5000A93421978FEF881A980AA80AB80A2097B2
:106C600021F78AE0C80ED11CE11CF11C82EDC81688
:106C700080E2D806E104F104A1F6C12C20E2D22E74
:106C8000E12CF12CD5E0C2E810924B1410924A147A
:106C9000D0933E14C0934114C0924214D092431436
:106CA000E0924414F09245148EEE93E10E94A934D0
:106CB00010924B1410924A14D0933E14C093411476
:106CC000D701C6018C529F4FAF4FBF4F80934214E4
:106CD00090934314A0934414B09345148EEE93E123
:106CE0000E94A9348FEFC81AD80AE80AF80A8AE085
:106CF000C81680E2D806E104F10431F69EEDC92EF3
:106D000090E2D92EE12CF12CD5E0C2E810924B1480
:106D100010924A14D0933E14C0934114C09242146E
:106D2000D0924314E0924414F09245148EEE93E115
:106D30000E94A9348FEFC81AD80AE80AF80A86EE2A
:106D4000C81680E2D806E104F10401F7CC24C3940C
:106D500082E1D82EE12CF12C0AE010E0D5E0C2E867
:106D600010934B1400934A14D0933E14C0934114D3
:106D7000C0924214D0924314E0924414F09245140D
:106D80008EEE93E10E94A93410934B1400934A14A1
:106D9000D0933E14C0934114D701C6018096A11D23
:106DA000B11D8093421490934314A0934414B09364
:106DB00045148EEE93E10E94A9348FEFC81AD80AC9
:106DC000E80AF80A85E1C81682E1D806E104F10470
:106DD00039F682E190E090934B1480934A14D0935B
:106DE0003E14C093411484E190E1A0E0B0E08093B0
:106DF000421490934314A0934414B09345148EEE20
:106E000093E1DF91CF911F910F91FF90EF90DF9071
:106E1000CF90BF90AF909F908F900C94A9341F9209
:106E20000F920FB60F9211240BB60F922F938F93E0
:106E30009F93EF93FF938091370420913604821340
:106E400006C08091D1008F7D8093D10012C0E82FC1
:106E5000F0E0EA5CFB4F92818F5F8F779093D600D2
:106E6000809337049091D00090649093D0002817BD
:106E700041F3FF91EF919F918F912F910F900BBE56
:106E80000F900FBE0F901F9018951F920F920FB684
:106E90000F9211240BB60F920F931F932F933F93D2
:106EA0004F935F936F937F938F939F93AF93BF9312
:106EB000CF93DF93EF93FF93C091D60000915A05D3
:106EC000D091590511E01D0F1F7390913504913138
:106ED00008F09FC0E92FF0E08827EE58F84C8F4F5C
:106EE0000D947D318337B237C137D037D737093862
:106EF000DB370938DF37E3370938E737EB37EF3768
:106F0000F63709380138C03229F028F5CA3011F0B7
:106F1000CD3031F5011731F0ED2FF0E0E75AFA4F9F
:106F2000C283D12FD0935905FF91EF91DF91CF917B
:106F3000BF91AF919F918F917F916F915F914F9191
:106F40003F912F911F910F910F900BBE0F900FBE8D
:106F50000F901F901895CD3481F081E0CE3471F000
:106F600080E10CC0CA3338F4C033A0F6C03291F2CD
:106F7000CD32B1F7CFCFCD3499F782E0809335048D
:106F8000C9CFC13359F018F4C03221F2E9CF88E0FB
:106F9000C433A1F38BE0C83389F3E2CF83E0EECFB3
:106FA00084E0C03359F386E0C13341F3D9CF85E0A3
:106FB000C833B1F6E3CF87E0C23391F6DFCF89E083
:106FC000C13371F6DBCF8AE0C03351F6D7CF8CE006
:106FD000C73331F6D3CF8DE0C63311F6CFCFC032F1
:106FE00009F498CF8EE0C33549F2BACF80ED8C0F0B
:106FF0008A3008F08FCF9FE090933504809334045B
:1070000089CFCA3019F0CD3009F084CF1092350401
:1070100081CFCA3019F0CD3009F07CCF8091A8140F
:107020008823A1F3973089F038F4953079F71092DE
:1070300044021092AA0CEACF9A3059F09F3031F7EF
:10704000809134040E94C831E1CF81E08093300602
:10705000DDCF81E080932F06D9CF9091C00095FFBE
:10706000FCCF8093C6000895CF93DF93EC01899104
:10707000882319F00E942D38FACF8DE00E942D3818
:107080008AE0DF91CF910C942D38CF92DF92EF926E
:10709000FF92CF936B017C01C42F4A3069F4F7FE55
:1070A0000BC0F094E094D094C094C11CD11CE11C9E
:1070B000F11C8DE20E942D384C2FC701B601CF91F3
:1070C000FF90EF90DF90CF900C9406ADCF93DF93BD
:1070D000EC01FE0184912196882319F00E942D383D
:1070E000F8CFDF91CF910895CF93DF93D09197118F
:1070F00087E89CE10E9466388AE00E942D388091E2
:10710000160D873009F449C083E08093140D81E0A7
:107110008093860280E190E090934B1480934A1410
:1071200085E080933E14C2E8C093411484E190E16D
:10713000A0E0B0E08093421490934314A0934414D1
:10714000B09345148EEE93E10E94A93461E070E0A3
:1071500080E090E00E94B22C81E09AE590934B147D
:1071600080934A1485E390E090934D1480934C14DF
:1071700087E080933E14C093411484E890E0A0E03F
:10718000B0E08093421490934314A0934414B093BE
:1071900045148EEE93E10E94A934809197118130BD
:1071A00089F1823061F50E949E2B6093CA0570932D
:1071B000CB058093CC059093CD0581E0809397110A
:1071C0000E94C0A96093C6057093C7058093C80547
:1071D0009093C905D23089F08091B3069091B4069E
:1071E00001969093B4068093B3061092D205109244
:1071F000D3051092D4051092D50581E004C00E94F9
:10720000D02BDBCF80E0DF91CF910895CF93C82FB3
:10721000CB010E9466388BEF98E10E9466388CEEB5
:1072200098E1CC2311F081EF98E10E9466388AE062
:10723000CF910C942D38CF93DF9300D01F92CDB710
:10724000DEB784EF91E0A0E0B0E089839A83AB835E
:10725000BC83BE016F5F7F4F8CE30E948B3389E15B
:1072600099E10E9466388CB163E179E185FB88275A
:1072700080F90E940639809103016DE079E18695DD
:1072800081700E94063989B167E079E183FB882724
:1072900080F90E9406398CB16EEF78E18295817099
:1072A0000E9406394B9909C00E94C6330F900F9077
:1072B0000F900F90DF91CF9108950E94AB330F9004
:1072C0000F900F900F90DF91CF91089580919711BB
:1072D0008130C1F587EC98E10E9466388AE00E940F
:1072E0002D3881E09AE590934B1480934A1487E5FA
:1072F00090E090934D1480934C1487E080933E145B
:1073000082E88093411484E890E0A0E0B0E08093AC
:10731000421490934314A0934414B09345148EEEFA
:1073200093E10E94A93482E0809397110E94C0A942
:107330006093CE057093CF058093D0059093D105CF
:1073400081E0089580E008950F931F930E94C0A9E3
:107350000091AE061091AF062091B0063091B106B3
:10736000011511052105310509F067C02091201391
:10737000222309F45FC0E0911E13215020932013B3
:1073800021E02E0F20931E1330912113231302C0EE
:1073900010921E1324E0E29FF0011124EE5DFC4EDA
:1073A00000811181228133810093AA061093AB06DC
:1073B0002093AC063093AD06600F711F811D911DA7
:1073C0006093AE067093AF068093B0069093B106BB
:1073D0008091AC069091AD06892B61F11FB7F894AE
:1073E00086EB98E10E9466388AE00E942D3884E09E
:1073F00096E090934B1480934A1480EA90E890931F
:107400004D1480934C1487E080933E1482E880935F
:10741000411480EA90E0A0E0B0E0809342149093A1
:107420004314A0934414B09345148EEE93E10E944C
:10743000A9341FBF1F910F910895601B710B820B20
:10744000930B97FDF7CF40981092AE061092AF06BF
:107450001092B0061092B106EDCF0F931F93CF9309
:10746000DF938C01EB019091201320912113921353
:1074700005C00E94A4390E94CEC4F5CF80911F138D
:1074800034E0839FF0011124EE5DFC4E11830083F4
:10749000D383C2839F5F909320138F5F281739F0A7
:1074A00080931F13DF91CF911F910F910895109238
:1074B0001F13F8CFCF92DF92EF92FF921F93CF93DB
:1074C000DF93182F662351F01092080510920405DF
:1074D0001092050510920605109207050E94C0A99A
:1074E0006B017C018091040590910505A091060532
:1074F000B0910705A7019601281B390B4A0B5B0BBE
:10750000DA01C901B7FD3DC02091080517FD13C080
:10751000412F012E000C550B4C5F5F4F822F022E26
:10752000000C990B4817590764F184EF91E0A0E033
:10753000B0E0211724F488EE93E0A0E0B0E08C0DD9
:107540009D1DAE1DBF1D8093040590930505A0935E
:107550000605B09307052170C22F30E0D32F84E2D7
:107560008C9FB0018D9F700D7C1B112460597C4F46
:1075700082E390E00E942D3A809108058F5F80930E
:107580000805DF91CF911F91FF90EF90DF90CF9092
:107590000895CF93DF9300D01F92CDB7DEB78CE371
:1075A00098E10E9466388AE00E942D388091160D7D
:1075B0008330D9F119821A821B821C8260E0CE01CD
:1075C00001960E94EB2B19821A821B821C8261E0B9
:1075D000CE0101960E94EB2B81E0809385021092F0
:1075E000130D8093860281E09AE590934B1480936B
:1075F0004A1483E390E090934D1480934C1487E0F9
:1076000080933E1482E88093411484E890E0A0E0E7
:10761000B0E08093421490934314A0934414B09329
:1076200045148EEE93E10E94A9340F900F900F90B5
:107630000F90DF91CF9108956F927F928F929F92DA
:10764000AF92BF92CF92DF92EF92FF920F931F9370
:10765000CF93DF93CDB7DEB764970FB6F894DEBF54
:107660000FBECDBF1092D0008091D0008260809379
:10767000D0001092D50080E18093D4008091D10099
:1076800080618093D1008091D10088608093D10087
:107690008091D10080688093D1008091D1008F7D4E
:1076A0008093D1008AE580933F148093EF1385EA9D
:1076B000809340148093F013EEE8F4E18AE1DF0157
:1076C0001D928A95E9F78091120D882309F473C2FF
:1076D00083E090E090934B1480934A1485E080936C
:1076E0003E1482E8809341148FE190E1A0E0B0E085
:1076F0008093421490934314A0934414B093451480
:107700008EEE93E10E94A93484E690E090934B14AE
:1077100080934A1405E000933E1412E8109341143C
:1077200086E090E1A0E0B0E080934214909343148F
:10773000A0934414B09345148EEE93E10E94A934B3
:107740008BE090E090934B1480934A1400933E1486
:107750001093411480E092E1A0E0B0E080934214E5
:1077600090934314A0934414B09345148EEE93E188
:107770000E94A93410924B1410924A1400933E14A4
:107780001093411484E390E1A0E0B0E080934214B0
:1077900090934314A0934414B09345148EEE93E158
:1077A0000E94A93410924B1410924A1400933E1474
:1077B000109341148AE390E1A0E0B0E0809342147A
:1077C00090934314A0934414B09345148EEE93E128
:1077D0000E94A93480915E1290915F1290934B1495
:1077E00080934A1400933E141093411486E390E171
:1077F000A0E0B0E08093421490934314A09344140B
:10780000B09345148EEE93E10E94A9348091F31158
:107810009091F41190934B1480934A1400933E146A
:10782000109341148CE390E1A0E0B0E08093421407
:1078300090934314A0934414B09345148EEE93E1B7
:107840000E94A93482E090E090934B1480934A14F4
:1078500000933E14109341148EE190E1A0E0B0E05B
:107860008093421490934314A0934414B09345140E
:107870008EEE93E10E94A93481E08093850270E648
:10788000C72E70E1D72EE12CF12C10924B141092E0
:107890004A1400933E1410934114C0924214D092A3
:1078A0004314E0924414F09245148EEE93E10E944A
:1078B000A934BFEFCB1ADB0AEB0AFB0AE4E7CE16CA
:1078C000E0E1DE06E104F10401F7CE0101967C015E
:1078D00084E1D7011D928A95E9F781E08F9390E9C1
:1078E0009F938F9398E69F938F939F9381EB93E061
:1078F0009F938F93FF92EF920F940E3520E630E125
:1079000040E050E06EEB73E08EEE93E10E94A8E958
:107910002AE630E140E050E06BEC73E08EEE93E15C
:107920000E94A8E924E730E140E050E0B7018EEE84
:1079300093E10E94A8E92EE730E140E050E067EDD6
:1079400073E08EEE93E10E94A8E910924B1410921E
:107950004A1400933E14109341148EE090E1A0E08D
:10796000B0E08093421490934314A0934414B093D6
:1079700045148EEE93E10E94A93410924B1410929C
:107980004A1400933E14109341148FE090E1A0E05C
:10799000B0E08093421490934314A0934414B093A6
:1079A00045148EEE93E10E94A9340FB6F894DEBF21
:1079B0000FBECDBF4AE0C42E40E2D42EE12CF12C04
:1079C00055E0752E62E8662E460157010AE010E088
:1079D00010924B1410924A1470923E14609241140B
:1079E0008092421490924314A0924414B092451491
:1079F0008EEE93E10E94A93401501109FFEF8F1A16
:107A00009F0AAF0ABF0A0115110511F78AE0C80ED7
:107A1000D11CE11CF11C92EDC91690E2D906E104DB
:107A2000F10491F6C12C30E2D32EE12CF12C05E0CB
:107A300012E810924B1410924A1400933E141093C3
:107A40004114C0924214D0924314E0924414F09234
:107A500045148EEE93E10E94A93410924B141092BB
:107A60004A1400933E1410934114D701C6018C525E
:107A70009F4FAF4FBF4F8093421490934314A093F6
:107A80004414B09345148EEE93E10E94A934AFEFF5
:107A9000CA1ADA0AEA0AFA0ABAE0CB16B0E2DB0638
:107AA000E104F10431F62EEDC22E20E2D22EE12CBB
:107AB000F12C05E012E810924B1410924A14009336
:107AC0003E1410934114C0924214D0924314E09299
:107AD0004414F09245148EEE93E10E94A934EFEF26
:107AE000CE1ADE0AEE0AFE0AF6EECF16F0E2DF0646
:107AF000E104F10401F7CC24C39482E1D82EE12CF7
:107B0000F12C9AE0A92EB12C05E012E8B0924B14AA
:107B1000A0924A1400933E1410934114C092421450
:107B2000D0924314E0924414F09245148EEE93E107
:107B30000E94A934B0924B14A0924A1400933E14B0
:107B400010934114D701C6018096A11DB11D8093E9
:107B5000421490934314A0934414B09345148EEEB2
:107B600093E10E94A9348FEFC81AD80AE80AF80AEC
:107B700095E1C91692E1D906E104F10439F682EAE9
:107B800097E10E9466388AE00E942D3864960FB60D
:107B9000F894DEBF0FBECDBFDF91CF911F910F9143
:107BA000FF90EF90DF90CF90BF90AF909F908F901D
:107BB0007F906F90089582E090E08CCD0E941C3BF6
:107BC0001092A20581E08093860284E598E10E94EC
:107BD00066388AE00C942D380F931F93CF938C0155
:107BE000C62F8EE294E10E946638C8010E94663872
:107BF0008AE30E942D3880E38C0F0E942D388AE0A2
:107C0000CF911F910F910C942D3881EB95E10E943B
:107C1000663860E081EA95E10E94EC3D60E08CE826
:107C200095E10E94EC3D61E085E895E10E94EC3D24
:107C300061E08AE795E10E94EC3D61E08AE695E12A
:107C40000E94EC3D60E081E695E10E94EC3D61E040
:107C500087E595E10E94EC3D61E08DE495E10E94AD
:107C6000EC3D61E086E495E10E94EC3D61E08EE34D
:107C700095E10E94EC3D61E080E395E10E94EC3DDE
:107C800061E082E295E10E94EC3D60E083E195E1F4
:107C90000E94EC3D60E085E095E10E94EC3D60E0F3
:107CA0008FEE94E10E94EC3D61E08EED94E10E9444
:107CB000EC3D61E08FEC94E10E94EC3D61E088ECEA
:107CC00094E10E94EC3D60E081EC94E10E94EC3D87
:107CD00061E088EB94E10E94EC3D61E083EA94E18D
:107CE0000E94EC3D61E085E994E10E94EC3D61E099
:107CF00082E894E10E94EC3D60E085E794E10E9417
:107D0000EC3D61E080E794E10E94EC3D61E083E6B8
:107D100094E10E94EC3D60E08FE494E10E94EC3D30
:107D200060E08CE394E10E94EC3D60E087EB94E13D
:107D30000E94711D682F617083E394E10C94EC3D07
:107D400080915305827149F4809155058C7829F40E
:107D500080915605837009F475C082E40E944F1E1D
:107D6000882351F00E941D246093C10C7093C20CB3
:107D70008093C30C9093C40C83E50E944F1E88230C
:107D800051F00E94A3246093F10C7093F20C809345
:107D9000F30C9093F40C84E50E944F1E882351F05D
:107DA0000E94A3246093F50C7093F60C8093F70C5B
:107DB0009093F80C88E50E944F1E882351F00E9492
:107DC000A324609318097093190980931A0990935A
:107DD0001B0989E50E944F1E882351F00E94A324AD
:107DE00060931C0970931D0980931E0990931F09CD
:107DF0008AE50E944F1E8823B1F00E94A32460935D
:107E000020097093210980932209909323092DEC76
:107E10003CEC4CEC5DE30F94B62A181624F088E98C
:107E20009EE00E94663885E40E944F1E882351F030
:107E30000E94A32460932409709325098093260946
:107E4000909327090895AF92BF92CF92DF92EF925D
:107E50000F931F93CF93DF935B01EA01690188239E
:107E600009F463C081E99EE00E946638F5016081F3
:107E700071818281938146E00E940EBDE1100BC0AA
:107E800088E89EE00E946638688179818A819B81BA
:107E900046E00E940EBD81E89EE00E946638F60131
:107EA000608171818281938143E00E940EBD8AE7E7
:107EB0009EE00E946638F801608171818281938121
:107EC00043E00E940EBD81E79EE00E946638F60105
:107ED0002081318142815381F801608171818281E9
:107EE00093810F94853143E00E940EBDEE20F9F09E
:107EF0008AE00E942D388CE59EE00E9466386881F9
:107F000079818A819B8146E00E940EBD8AE00E94B1
:107F10002D388AE0DF91CF911F910F91EF90DF9084
:107F2000CF90BF90AF900C942D38E110E4CFDF914B
:107F3000CF911F910F91EF90DF90CF90BF90AF90B6
:107F400008950F931F93CF938C01C62F89E798E074
:107F50000E946638C8010E946638CC2331F08AE05E
:107F6000CF911F910F910C942D38CF911F910F91AC
:107F700008950E94B4ED1092AA0C109244020E943F
:107F8000E631882351F08091B41482FD06C082EB63
:107F900098E19093FA0C8093F90C61E08BEA98E1F8
:107FA0000E94A13F0C9474380F931F93CF93DF93DB
:107FB0008C016F3F19F41092D81160E02091D81114
:107FC000862F062E000C990B2817190609F08CF540
:107FD0006093D81160E085E798E10E94A13FC80155
:107FE0000E9466388AE00E942D38C8010F94032A47
:107FF000800F911FEC01C01BD10BC034D1053CF0A8
:108000000197FC012491207C2038D1F3F3CFDD27A8
:10801000AE01B80188E991E10F94242AC856DE4EDA
:10802000188288E991E1DF91CF911F910F910C9413
:108030007335DF91CF911F910F9108951092AA0C83
:10804000109244028091B41480648093B41461E06F
:1080500083E898E10E94A13F48E958E160EA78E1AD
:1080600085E00E94C2EB60E08AE898E10C94D43F7E
:108070000F931F93CF938C01C62F60E083E898E0A5
:108080000E94A13FC8010E946638CC2331F08AE0EB
:10809000CF911F910F910C942D38CF911F910F917B
:1080A000089561E08BE898E00C943840EF92FF92DD
:1080B0000F931F93CF937C018B01C42F60E083E863
:1080C00098E00E94A13FC7010E94663880E20E94AA
:1080D0002D38C8010E946638CC2319F08C2F0E94DD
:1080E0002D388AE0CF911F910F91FF90EF900C9463
:1080F0002D38DF92EF92FF920F931F93CF93DF9370
:10810000D82E7B018A01E9010E945140D0920412CD
:1081100040E0B70184E799E00E945640011511053F
:1081200031F040E0B8018DE699E00E94564020977A
:1081300031F040E0BE018DE699E00E94564061E0DA
:1081400088E699E0DF91CF911F910F91FF90EF901A
:10815000DF900C943840AF92BF92CF92DF92EF92B3
:10816000FF920F931F93CF93DF9386EE97E00E94C9
:108170006638C0E0D7E0D15021F080E20E942D386F
:10818000FACF8C2F0E94FBE9CF5FC53099F78AE0C8
:108190000E942D3807EB17E0C0E080E20E942D38E6
:1081A0008C2F0E94FBE95801D5E080E20E942D3817
:1081B000F501C080D180E280F380A7019601C7015C
:1081C000B6010F947834882369F180E20E942D383B
:1081D0008DE30E942D388DE30E942D388DE30E949F
:1081E0002D388DE30E942D388DE30E942D38D1501B
:1081F000F4E1AF0EB11CD111D8CF8AE00E942D3826
:10820000CF5F0C5F1F4FC53041F68AE0DF91CF9101
:108210001F910F91FF90EF90DF90CF90BF90AF90A4
:108220000C942D3820E030E0A901C701B6010F946D
:10823000E63387FD03C08BE20E942D3843E0C7017F
:10824000B6010E940EBDD3CF811107C08AEC9EE01B
:108250000E9466388AE00C942D388EEC9EE0F8CFB0
:10826000CF93DF93EB010E946638CE01DF91CF916F
:108270000C94B9EACF93C62F0E9466388C2FCF9109
:108280000C94FBE9CF92DF92EF92FF926A017B019F
:108290000E94663842E0C701B601FF90EF90DF9080
:1082A000CF900C940EBDCF92DF92EF92FF926A01B5
:1082B0007B010E9466384AE0C701B601FF90EF904B
:1082C000DF90CF900C944538CF93DF93EB010E9461
:1082D0006638CE01DF91CF910C9402EA4F925F9203
:1082E0006F927F928F929F92AF92BF92CF92DF92C6
:1082F000EF92FF920F931F93CF93DF9300D000D0A4
:108300001F921F92CDB7DEB78091A10581110AC4DB
:1083100080919F059091A0059C012F5F3F4F309366
:10832000A00520939F058E3E924008F4FBC38091E8
:108330005E1290915F1290934B1480934A1405E063
:1083400000933E1412E81093411486E390E1A0E0FC
:10835000B0E08093421490934314A0934414B093DC
:1083600045148EEE93E10E94A9348091F31190910F
:10837000F41190934B1480934A1400933E1410937D
:1083800041148CE390E1A0E0B0E08093421490931C
:108390004314A0934414B09345148EEE93E10E94CD
:1083A000A934809160129091611290934B14809344
:1083B0004A1400933E141093411484E390E1A0E02A
:1083C000B0E08093421490934314A0934414B0936C
:1083D00045148EEE93E10E94A9348091F51190919D
:1083E000F61190934B1480934A1400933E1410930B
:1083F00041148AE390E1A0E0B0E0809342149093AE
:108400004314A0934414B09345148EEE93E10E945C
:10841000A93481E08093A1051092A00510929F05D8
:108420008091160D882339F10E94031D811123C00C
:1084300080919E058F5F80939E0580919E05853675
:1084400020F010929E051092160DE091160DE1504D
:10845000E73008F06AC00E2E000CFF0B8827EC5C9A
:10846000FD4B8F4F0D947D313E428D4259448544E2
:10847000C644FE44914210929E05DFCF0E94AA2C72
:10848000882309F452C081E0809386028EE298E14D
:108490000E9466388AE00E942D3880E190E0909337
:1084A0004B1480934A1485E080933E1412E8109395
:1084B000411484E190E1A0E0B0E0809342149093F5
:1084C0004314A0934414B09345148EEE93E10E949C
:1084D000A93481E09AE590934B1480934A1486E383
:1084E00090E090934D1480934C1487E080933E1459
:1084F0001093411484E890E0A0E0B0E0809342142F
:1085000090934314A0934414B09345148EEE93E1DA
:108510000E94A9341092160D08C00E94AA2C88232C
:1085200021F00E94031D8823A9F3809186028823ED
:1085300009F433C78091A2058111C0C284E096E09E
:1085400090934B1480934A1480EA90E890934D14D2
:1085500080934C1417E010933E1402E800934114EA
:1085600080EA90E0A0E0B0E080934214909343143E
:10857000A0934414B09345148EEE93E10E94A93465
:108580008091810290918202A0918302B091840235
:108590000097A105B10509F03FC210924B1410924B
:1085A0004A1415E010933E14009341148AE890E1B8
:1085B000A0E0B0E08093421490934314A09344143D
:1085C000B09345148EEE93E10E94A93489E090E0C7
:1085D00090934B1480934A1410933E1400934114CB
:1085E0008CE890E1A0E0B0E08093421490934314B3
:1085F000A0934414B09345148EEE93E10E94A934E5
:108600008091810290918202A0918302B0918402B4
:108610000097F1E0AF07B10508F441C2B0934B14E5
:10862000A0934A1490934D1480934C1487E0809348
:108630003E1482E88093411488E890E1A0E0B0E025
:108640008093421490934314A0934414B093451420
:108650008EEE93E10E94A934809181029091820272
:10866000A0918302B0918402BA2FA92F982F882756
:10867000009721E0A207B10508F417C2B0934B148C
:10868000A0934A1490934D1480934C1487E08093E8
:108690003E1412E81093411481EA90E0A0E0B0E0AB
:1086A0008093421490934314A0934414B0934514C0
:1086B0008EEE93E10E94A9348091AC0C882309F4DA
:1086C000FAC183E090E090934B1480934A1485E0C4
:1086D00080933E141093411485E490E1A0E0B0E053
:1086E0008093421490934314A0934414B093451480
:1086F0008EEE93E10E94A9348091A205875E80935B
:10870000A2052091A205822F90E0253608F021C213
:1087100090934B1480934A1485E080933E1482E832
:108720008093411480E090E1A0E0B0E08093421497
:1087300090934314A0934414B09345148EEE93E1A8
:108740000E94A9340E94031D811114C20E94E631C7
:10875000811105C09091A50591FD0E94031D909186
:10876000A50580FB91F99093A50591FD03C2809129
:10877000B41482FDFFC1809197118150823008F4BA
:10878000F9C16091F5117091F611072E000C880B5C
:10879000990B0F94BD2A6B017C0120E030E0A90108
:1087A0000F94B62A882309F4BBC66091F311709127
:1087B000F411072E000C880B990B0F94BD2A2B0186
:1087C0003C0120E030E040E050E4C701B6010F94E6
:1087D0008531A30192010F94E63318160CF4C2C63A
:1087E00060915E1270915F12072E000C880B990B3E
:1087F0000F94BD2A6D837E838F839887609160126A
:1088000070916112072E000C880B990B0F94BD2AF2
:108810004B015C0120E030E040E251E40F948531EF
:108820002D813E814F8158850F94E63318160CF444
:1088300099C620E030E040E050E4C701B6010F9453
:108840008631A30192010F94B62A87FD10C020E063
:1088500030E040E251E4C501B4010F9486312D812E
:108860003E814F8158850F94B62A87FF6AC684E1FE
:1088700090E090934B1480934A1485E080933E14CB
:1088800082E88093411484E190E1A0E0B0E080931D
:10889000421490934314A0934414B09345148EEE65
:1088A00093E10E94A9348091140D81117CC682E06D
:1088B0007AC680E298E10E9466388AE00E942D38EC
:1088C00081E09AE590934B1480934A1480E490E001
:1088D00090934D1480934C1417E010933E1482E84B
:1088E0008093411484E890E0A0E0B0E080934214CB
:1088F00090934314A0934414B09345148EEE93E1E7
:108900000E94A9341093160D10CE8091030D882378
:1089100009F40BCE0E94AA2C882309F406CE0E94EB
:10892000031D811102CE82E198E10E9466388AE03F
:108930000E942D388091040D90E0B0E0A0E0895BAA
:108940009F4FAE4FB54A21E03AE530934B14209348
:108950004A1490934D1480934C1487E080933E14F6
:1089600082E88093411484E890E0A0E0B0E0809336
:10897000421490934314A0934414B09345148EEE84
:1089800093E10E94A9341092030DC4CD0E94AA2C39
:10899000882309F4CACD0E94031D8111C6CD81E050
:1089A000809386021092160D84E098E10E9466384A
:1089B0008AE00E942D3881E09AE590934B148093D1
:1089C0004A148EE490E090934D1480934C1487E009
:1089D00080933E1482E88093411484E890E0A0E004
:1089E000B0E08093421490934314A0934414B09346
:1089F00045148EEE93E10E94A93497CD0E94031D89
:108A0000811193CD19821A821B821C8262E0CE01F1
:108A100001960F94A7007ECD0196A11DB11D35E0F2
:108A2000B695A795979587953A95D1F70197A1099E
:108A3000B1090097E1E0AE07B10548F1B0934B14DE
:108A4000A0934A1490934D1480934C1410933E14A9
:108A500012E8109341148AE890E1A0E0B0E080931E
:108A6000421490934314A0934414B09345148EEE93
:108A700093E10E94A93488E090E090934B14809396
:108A80004A1485E080933E1410934114A9CD90932D
:108A90004B1480934A1485E080933E14D9CF909371
:108AA0004B1480934A1485E0C2CD90934B1480936D
:108AB0004A1485E0ECCD82E090E005CE8A3F08F0D4
:108AC00020CE8EEF8093A20583EF97E10E94663857
:108AD0008AE00E942D3881E08093860281E09AE549
:108AE00090934B1480934A148DE290E090934D1430
:108AF00080934C1487E080933E1482E88093411465
:108B000084E890E0A0E0B0E0809342149093431496
:108B1000A0934414B09345148EEE93E10E94A934BF
:108B20001092A10528960FB6F894DEBF0FBECDBFF8
:108B3000DF91CF911F910F91FF90EF90DF90CF9039
:108B4000BF90AF909F908F907F906F905F904F906D
:108B500008958456910990934B1480934A1485E0AC
:108B600080933E1482E88093411481E090E1A0E07C
:108B7000B0E0DCCD8CE090E090934B1480934A14ED
:108B800015E010933E1482E88093411484E190E153
:108B9000A0E0B0E08093421490934314A093441457
:108BA000B09345148EEE93E10E94A9340E949E2B4F
:108BB00020E13EE040E050E00F94FA30211531050D
:108BC00081E04807510508F470C050934B1440935E
:108BD0004A1430934D1420934C1487E080933E1434
:108BE00012E81093411480E190E1A0E0B0E080939E
:108BF000421490934314A0934414B09345148EEE02
:108C000093E10E94A9340E949E2B20E13EE040E0C7
:108C100050E00F94FA302CE330E040E050E00F9445
:108C2000FA3030934B1420934A1405E000933E141D
:108C30001093411482E190E1A0E0B0E080934214EF
:108C400090934314A0934414B09345148EEE93E193
:108C50000E94A9340E94F431882309F45CC48F5F18
:108C600080939D05E82EF12C833330F5EE0CFF1C2C
:108C7000F0924B14E0924A1400933E141093411466
:108C80008EE090E1A0E0B0E0809342149093431412
:108C9000A0934414B09345148EEE93E10E94A9343E
:108CA00010924B1410924A142BC030934B14209303
:108CB0004A1410933E1494CF84E690E090934B14A2
:108CC00080934A1400933E14109341148EE090E177
:108CD000A0E0B0E08093421490934314A093441416
:108CE000B09345148EEE93E10E94A934A2E3EA1AF0
:108CF000A0E8FA0AEE0CFF1CF0924B14E0924A1422
:108D000000933E14109341148FE090E1A0E0B0E096
:108D10008093421490934314A0934414B093451449
:108D20008EEE93E10E94A9340E94F43190E090937A
:108D30004B1480934A1485E080933E1482E880931C
:108D4000411486E190E1A0E0B0E08093421490935A
:108D50004314A0934414B09345148EEE93E10E9403
:108D6000A93420E030E0A9016091F3127091F4126F
:108D70008091F5129091F6120F94863120E030E048
:108D800048EC52E40F941C2B0F94F23270934B1466
:108D900060934A1405E000933E1412E810934114C6
:108DA00086E290E1A0E0B0E08093421490934314F7
:108DB000A0934414B09345148EEE93E10E94A9341D
:108DC00080917D0290917E0290934B1480934A147F
:108DD00000933E141093411480E093E1A0E0B0E0D2
:108DE0008093421490934314A0934414B093451479
:108DF0008EEE93E10E94A93420E030E040E251E49D
:108E00006091C50C7091C60C8091C70C9091C80CF4
:108E10000F941C2B0F94F93270934B1460934A14E7
:108E200000933E141093411482E492E1A0E0B0E07C
:108E30008093421490934314A0934414B093451428
:108E40008EEE93E10E94A93420E030E040E251E44C
:108E50006091C90C7091CA0C8091CB0C9091CC0C94
:108E60000F941C2B0F94F93270934B1460934A1497
:108E700000933E141093411486E492E1A0E0B0E028
:108E80008093421490934314A0934414B0934514D8
:108E90008EEE93E10E94A93420E030E040E251E4FC
:108EA0006091CD0C7091CE0C8091CF0C9091D00C34
:108EB0000F941C2B0F94F93270934B1460934A1447
:108EC00000933E14109341148AE492E1A0E0B0E0D4
:108ED0008093421490934314A0934414B093451488
:108EE0008EEE93E10E94A93420E030E040E251E4AC
:108EF0006091D10C7091D20C8091D30C9091D40CD4
:108F00000F941C2B0F94F93270934B1460934A14F6
:108F100000933E14109341148EE492E1A0E0B0E07F
:108F20008093421490934314A0934414B093451437
:108F30008EEE93E10E94A93420E030E048EC52E448
:108F40006091EB127091EC128091ED129091EE1203
:108F50000F941C2B0F94F23270934B1460934A14AD
:108F600000933E141093411486E392E1A0E0B0E038
:108F70008093421490934314A0934414B0934514E7
:108F80008EEE93E10E94A93420E030E048EC52E4F8
:108F90006091EF127091F0128091F1129091F212A3
:108FA0000F941C2B0F94F23270934B1460934A145D
:108FB00000933E14109341148AE392E1A0E0B0E0E4
:108FC0008093421490934314A0934414B093451497
:108FD0008EEE93E10E94A93480918D0290918E02D1
:108FE00090934B1480934A1400933E1410934114B1
:108FF00082E592E1A0E0B0E08093421490934314A4
:10900000A0934414B09345148EEE93E10E94A934CA
:1090100080918B0290918C0290934B1480934A1410
:1090200000933E141093411484E592E1A0E0B0E077
:109030008093421490934314A0934414B093451426
:109040008EEE93E10E94A93420E030E040E251E44A
:109050006091631270916412809165129091661212
:109060000F941C2B0F94F93270934B1460934A1495
:1090700000933E141093411486E592E1A0E0B0E025
:109080008093421490934314A0934414B0934514D6
:109090008EEE93E10E94A9342CEA35EC47E25EE3C0
:1090A00060916712709168128091691290916A12B2
:1090B0000F94803220E030E040E251E40F941C2B0A
:1090C0000F94F93270934B1460934A1400933E143A
:1090D000109341148AE592E1A0E0B0E0809342143D
:1090E00090934314A0934414B09345148EEE93E1EF
:1090F0000E94A9342CEA35EC47E25EE360916B12E2
:1091000070916C1280916D1290916E120F941C2BC5
:1091100020E030E040E251E40F941C2B0F94F93230
:1091200070934B1460934A1400933E1410934114AF
:109130008EE592E1A0E0B0E0809342149093431456
:10914000A0934414B09345148EEE93E10E94A93489
:1091500020E030E040E251E46091F8117091F911A3
:109160008091FA119091FB110F941C2B0F94F932FE
:1091700070934B1460934A1400933E14109341145F
:1091800082E692E1A0E0B0E0809342149093431411
:10919000A0934414B09345148EEE93E10E94A93439
:1091A0002CEA35EC47E25EE36091FC117091FD1111
:1091B0008091FE119091FF110F94803220E030E0F9
:1091C00040E251E40F941C2B0F94F93270934B142E
:1091D00060934A1400933E141093411486E692E182
:1091E000A0E0B0E08093421490934314A093441401
:1091F000B09345148EEE93E10E94A9342CEA35EC2D
:1092000047E25EE3609100127091011280910212B8
:10921000909103120F941C2B20E030E040E251E4C7
:109220000F941C2B0F94F93270934B1460934A14D3
:1092300000933E14109341148AE692E1A0E0B0E05E
:109240008093421490934314A0934414B093451414
:109250008EEE93E10E94A93480910D0D811105C01D
:1092600080910F0D882309F46DC060915E1270919A
:109270005F12072E000C880B990B0F94BD2A20E07B
:1092800030E048EC52E40F941C2B6B017C016091A0
:10929000601270916112072E000C880B990B0F94CD
:1092A000BD2A9B01AC01C701B6010F9480320F9417
:1092B000F9326536710510F064E670E070934B1476
:1092C00060934A1405E000933E1412E81093411491
:1092D00084E290E1A0E0B0E08093421490934314C4
:1092E000A0934414B09345148EEE93E10E94A934E8
:1092F00060915E1270915F12072E000C880B990B23
:109300000F94BD2A6B017C0120E030E04AE253E477
:109310000F94E633181624F480910D0D811146C187
:109320006091601270916112072E000C880B990BEE
:109330000F94BD2A9B01AC01C701B6010F94E6331F
:1093400087FFAFC18091030D882339F18091020D11
:1093500091E0980F9093020D90E090934B148093BE
:109360004A1485E080933E1482E88093411482E49D
:1093700090E1A0E0B0E08093421490934314A09356
:109380004414B09345148EEE93E10E94A934809169
:10939000020D8A3010F01092020D0E94342C8823A6
:1093A00009F4B5C16091FB0C7091FC0CEE24E394C0
:1093B000F12C61157105A9F090E080E00F94BB2AB3
:1093C00020E030E040E85EE30F941C2B0F94643201
:1093D00020E030E040E85FE30F9486310F94F932EB
:1093E0007B0101E010E08091FD0C811102C010E0D2
:1093F00000E080913213909133138F3F980711F45E
:109400000E9463B69093331380933213080F191F91
:10941000B80190E080E00F94BB2A20E030E040E803
:109420005EE30F941C2B0F9464324B015C01F092AD
:109430004B14E0924A1405E000933E1412E8109396
:10944000411480E193E1A0E0B0E080934214909356
:109450004314A0934414B09345148EEE93E10E94FC
:10946000A934C501B4010F94F93270934B14609381
:109470004A1400933E141093411482E193E1A0E05A
:10948000B0E08093421490934314A0934414B0939B
:1094900045148EEE93E10E94A9340EE814E1AAE18E
:1094A000FA2E8091590590915A0520919B05309193
:1094B0009C05891B8F7309F449C12A3131050CF0D1
:1094C000DBC19091590580915A054FEF5FEF9817D6
:1094D00049F0E82FF0E0E75AFA4F42818F5F8F732F
:1094E00080935A05F901E257FB4E408380918E1418
:1094F0008A3509F0B3C162E070E080E090E00E943C
:10950000B22C80919B0590919C05019690939C05AF
:1095100080939B05C6CF10924B1410924A14ACCB8B
:109520006091601270916112072E000C880B990BEC
:109530000F94BD2A20E030E0A9010F94B62A8111D2
:1095400034C98CE090E090934B1480934A1485E0EA
:1095500080933E1482E88093411484E190E1A0E07E
:10956000B0E0F3CB8DE090E090934B1480934A14DD
:1095700085E080933E1482E88093411484E190E179
:10958000A0E0B0E08093421490934314A09344145D
:10959000B09345148EEE93E10E94A9348091140D8E
:1095A000811101C081E08093140DDBCB10920D0D71
:1095B00020E030E040E251E46091050D7091060D2D
:1095C0008091070D9091080D0F941C2B0F94F2328F
:1095D00070934B1460934A1400933E1410934114FB
:1095E00084E590E1A0E0B0E08093421490934314AE
:1095F000A0934414B09345148EEE93E10E94A934D5
:1096000020E030E040E251E46091090D70910A0DD4
:1096100080910B0D90910C0D0F941C2B0F94F23236
:1096200070934B1460934A1400933E1410934114AA
:1096300088E590E1A0E0B0E0809342149093431459
:10964000A0934414B09345148EEE93E10E94A93484
:1096500082ED97E10E9466388AE00E942D3881E011
:109660009AE590934B1480934A1481E490E0909390
:109670004D1480934C1487E080933E141093411452
:1096800084E890E0A0E0B0E080934214909343140B
:10969000A0934414B09345148EEE93E10E94A93434
:1096A00051CE60910F0D662309F44CCE062E000CAE
:1096B000770B89EB97E10E9464418AE00E942D3884
:1096C00010920F0D84E090E090934B1480934A1415
:1096D00085E080933E1412E8109341148EE890E1E7
:1096E000A0E0B0E08093421490934314A0934414FC
:1096F000B09345148EEE93E10E94A93481E09AE57F
:1097000090934B1480934A1483E590E0B0CF10926D
:109710004B1410924A1405E000933E1412E8109383
:10972000411480E193E1A0E0B0E080934214909373
:109730004314A0934414B09345148EEE93E10E9419
:10974000A93410924B1410924A1493CE1216130699
:109750000CF492C08091F2139091F313A091F41342
:10976000B091F5138C34E0E19E07A105B10509F431
:10977000D7C98A349041A105B10509F4D1C920E0C7
:1097800030E040E251E46091690270916A02809198
:109790006B0290916C020F941C2B0F94F232709319
:1097A0004B1460934A1405E000933E1412E81093A2
:1097B000411488E490E1A0E0B0E0809342149093DB
:1097C0004314A0934414B09345148EEE93E10E9489
:1097D000A93420E030E040E251E460916D027091E4
:1097E0006E0280916F02909170020F941C2B0F9467
:1097F000F23270934B1460934A1400933E1410930A
:1098000041148AE490E1A0E0B0E080934214909388
:109810004314A0934414B09345148EEE93E10E9438
:10982000A93420E030E040E251E46091710270918F
:10983000720280917302909174020F941C2B0F940A
:10984000F23270934B1460934A1400933E141093B9
:1098500041148CE490E1A0E0B0E056C91216130662
:109860000CF01FCEF8012F2D11922A95E9F71092D6
:109870009C0510929B0515CE9091EF1380918E144C
:10988000981321C09091F01380918F1498131BC0EE
:1098900023303105C4F0909190149093EE13809191
:1098A00091148093F1139330D1F4982F9D7F9038C9
:1098B000B1F4909192149F3409F059C0909193148F
:1098C0009B3409F054C0EEE8F4E18AE1DF011D9217
:1098D0008A95E9F710929C0510929B053BCF83383F
:1098E00009F045C08091921490919314982789278C
:1098F0009827B0E0A0E08093F2139093F313A09325
:10990000F413B093F513C0909414D12CF12CE12CE6
:10991000C092F613D092F713E092F813F092F91375
:1099200025E934E140E050E0BA014C155D056E05D3
:109930007F0508F04AC0DB01CA01B695A795979547
:1099400087950696880F991FFC01E251FC4ED901BC
:109950008C9111969C9189279827892791838083E0
:109960004E5F5F4F6F4F7F4F2E5F3F4FDECF81388F
:1099700061F58091921490E0B0E0A0E08093F21342
:109980009093F313A093F413B093F5138091931471
:10999000482F50E070E060E04093F6135093F713C7
:1099A0006093F8137093F913A4E9B4E1EAEFF3E1DB
:1099B00090E030E020E08217930739F04D9150E0BD
:1099C000419351932F5F3F4FF6CFEEE8F4E18AE1E8
:1099D000DF011D928A95E9F710929C0510929B0574
:1099E0000F944901B7CE3F924F925F926F927F9250
:1099F0008F929F92AF92BF92CF92DF92EF92FF929F
:109A00000F931F93CF93DF938091550587FD38C047
:109A1000809156058370A1F5C091F712D091F8128C
:109A2000488159816A817B8183E297E10E944241AA
:109A30004C815D816E817F8180E79FE20E9442417F
:109A40004091F3125091F4126091F5127091F61258
:109A50008DE69FE20E9442418AE0DF91CF911F9103
:109A60000F91FF90EF90DF90CF90BF90AF909F90BD
:109A70008F907F906F905F904F903F900C942D3817
:109A80006090EB127090EC128090ED129090EE12BC
:109A9000A090EF12B090F0120091F1121091F2121A
:109AA000C090F312D090F412E090F512F090F612FC
:109AB00088E50E949D1EC82F882309F49AC00E9441
:109AC000A324362E472E582ED92F20E030E044EB29
:109AD00053EC0F94E63387FD0DC020E030E044EBFB
:109AE00053E4632D742D852D9D2F0F94B62A1816DF
:109AF0000CF081C068E671E080E197E10E9464416A
:109B000068E671E08BE097E10E94644188E097E1AC
:109B10000E946638C0E089E50E949D1E882361F19D
:109B20000E94A324362E472E582ED92F20E030E055
:109B300044EB53EC0F94E63387FD0DC020E030E09A
:109B400044EB53E4632D742D852D9D2F0F94B62A7D
:109B500018160CF055C068E671E085EF96E10E949A
:109B6000644168E671E080EF96E10E9464418DEE09
:109B700096E10E946638C0E08AE50E949D1E882317
:109B800009F443C00E94A3246B017C0120E030E073
:109B900040E151EC0F94E63387FD0AC020E030E04D
:109BA00040E151E4C701B6010F94B62A18166CF5CE
:109BB00067EF7FEF8BED96E10E94644169E070E012
:109BC00086ED96E10E94644183ED96E1DF91CF91AD
:109BD0001F910F91FF90EF90DF90CF90BF90AF90CB
:109BE0009F908F907F906F905F904F903F900C94DC
:109BF0006638C1E090CF632C742C852C9D2E8BCFC2
:109C0000A32CB42C052D1D2FB7CFCC23E1F0C3011D
:109C1000D4018093EB129093EC12A093ED12B093C9
:109C2000EE12C501D8018093EF129093F012A09329
:109C3000F112B093F212C092F312D092F412E092A9
:109C4000F512F092F612DF91CF911F910F91FF90D4
:109C5000EF90DF90CF90BF90AF909F908F907F90CC
:109C60006F905F904F903F9008958FED97E00C9428
:109C7000663889ED97E00C94663884E690E090931E
:109C8000E3058093E20510920306109202060C94FD
:109C900055E4EF92FF920F931F93CF93DF93CDB7CD
:109CA000DEB762970FB6F894DEBF0FBECDBF0E943D
:109CB0001E2A882309F43FC046E054E082FF02C018
:109CC0004AEE53E026E034E081FF02C02CEE33E0A0
:109CD00080FD2EC086E094E05F934F933F932F93D7
:109CE0009F938F938DE699E19F938F938E010F5FE2
:109CF0001F4F1F930F930F944D2A0E94394EC80196
:109D00000E943438C8010E947CED0FB6F894DEBF83
:109D10000FBECDBF81E062960FB6F894DEBF0FBED6
:109D2000CDBFDF91CF911F910F91FF90EF900895DC
:109D30008EEE93E0D1CF80E0EECFCF92DF92EF9224
:109D4000FF928AE50E949D1E882309F45AC00E9452
:109D5000A32420E030E040E050EC0F94B62AC12C60
:109D6000D12CE12C90ECF92E87FD0FC00E94A3248A
:109D700020E030E040E050E40F94E63318160CF495
:109D800062C00E94A3246B017C012091CD0C309114
:109D9000CE0C4091CF0C5091D00CC701B6010F945E
:109DA0001C2B0F94F232CB010E9405ED80E50E943E
:109DB0004F1E81114EC0A70196016091F312709160
:109DC000F4128091F5129091F6120F9486316093FF
:109DD000F3127093F4128093F5129093F6120E948E
:109DE000394E4091F3125091F4126091F512709136
:109DF000F61284EC96E10E9442418AE00E942D38DE
:109E000005C083E50E949D1E8111A1CF809155055B
:109E100087FD24C080915605837001F50E94394E5C
:109E20004091F3125091F4126091F5127091F61274
:109E300085EB96E10E9442418AE0FF90EF90DF902F
:109E4000CF900C942D38C12CD12CE12C80E4F82E2D
:109E50009CCF0E946B248111AECFD8CF82E50E94A7
:109E60004F1E8111DBCFFF90EF90DF90CF900895D0
:109E7000CF9384E50E949D1EC0E08823D9F00E9404
:109E80004B24C82F1816B4F40E94394E8DE40E945A
:109E90002D3880915005909151050E94B9EA6C2FA0
:109EA000CC0F770B88EA9FE00E9464418AE00E9411
:109EB0002D38CFEF8C2FCF9108954F925F926F92F4
:109EC0007F928F929F92AF92BF92CF92DF92EF924A
:109ED000FF92CF93DF93CDB7DEB72C970FB6F894F0
:109EE000DEBF0FBECDBF4090F7085090F8086090DD
:109EF000F9087090FA0820914F0230915002409179
:109F0000510250915202C301B2010F94863169830C
:109F10007A838B839C838090FB089090FC08A090B0
:109F2000FD08B090FE0820915302309154024091F8
:109F3000550250915602C501B4010F9486316D83CC
:109F40007E838F839887C090FF08D0900009E090AF
:109F50000109F09002092091570230915802409176
:109F6000590250915A02C701B6010F948631698790
:109F70007A878B879C8720915B0230915C024091AD
:109F80005D0250915E02C301B2010F9486312B0134
:109F90003C0120915F02309160024091610250913A
:109FA0006202C501B4010F9486314B015C0120911E
:109FB0006302309164024091650250916602C701CC
:109FC000B6010F9486316B017C010E94394E83EEFD
:109FD0009EE00E94663883E50E944F1E882321F090
:109FE0000E946B2480934D0280914D02811151C0DB
:109FF0008AEC9EE00E9466388BED9EE00E946638F7
:10A0000049815A816B817C8184E59EE10E944241B5
:10A010004D815E816F81788580E79FE20E94424199
:10A0200049855A856B857C858DE69FE20E94424179
:10A0300089ED9EE00E94663881ED9EE00E946638C0
:10A04000B301A20184E59EE10E944241B501A40151
:10A0500080E79FE20E944241B701A6018DE69FE2A0
:10A060000E9442418AE02C960FB6F894DEBF0FBEE4
:10A07000CDBFDF91CF91FF90EF90DF90CF90BF9059
:10A08000AF909F908F907F906F905F904F900C94C7
:10A090002D388EEC9EE0AECF5F926F927F928F92C2
:10A0A0009F92AF92BF92CF92DF92EF92FF920F9367
:10A0B0001F93CF93DF931F92CDB7DEB77C01390199
:10A0C0008B015B01A40EB51ED12CC12CA016B106CC
:10A0D00009F450C0F70180809180F80151908F0100
:10A0E0005982C4010F94D4305816B9F1652DC401BA
:10A0F0000F94DC30FFEFCF1ADF0AC6018F77992764
:10A10000892B21F162E070E080E090E00E948DA94F
:10A11000C4010F94D43099818917F9F00E94394E07
:10A120008FE694E00E94663881E00F90DF91CF9136
:10A130001F910F91FF90EF90DF90CF90BF90AF9065
:10A140009F908F907F906F905F90089562E070E095
:10A1500080E090E00E941126DBCFBE016F5F7F4F51
:10A16000C3010E9460E9F70180819181019691838A
:10A170008083ACCF80E0D9CFDF92EF92FF920F9334
:10A180001F93CF93DF93CDB7DEB7CA5AD1090FB66D
:10A19000F894DEBF0FBECDBFCF55DF4F18821982B6
:10A1A0001A821B82C15AD0408091F0039091F10332
:10A1B000A091F203B091F303CB55DF4F88839983CD
:10A1C000AA83BB83C55AD04084E690E09093E30510
:10A1D0008093E20510920306109202061092040684
:10A1E00022E036E044E050E0BE016B557F4F82EE46
:10A1F00095E00E944C508091E2059091E305029613
:10A200009093E3058093E2051092030610920206F4
:10A2100081E0C655DF4F8883CA5AD040CE018655AB
:10A220009F4F0E9459DA22E036E048E450E061EBAB
:10A230007CE082EE95E00E944C5022E036E040E166
:10A2400050E068E179E082EE95E00E944C508AE0AF
:10A2500097EDA3EABCE3CF55DF4F88839983AA83A8
:10A26000BB83C15AD040CE018F559F4F0E9450DA18
:10A270008DE298E00E946BDA86E292E00E9462DA58
:10A2800082E292E00E9450DA8091F3089091F40803
:10A29000A091F508B091F60889839A83AB83BC83BB
:10A2A0008E010F5F1F4FC8010E9450DACF55DF4F5C
:10A2B000188219821A821B82C15AD0407E018DE613
:10A2C000E80EF11C83E0D7018C938983CE018F5572
:10A2D0009F4F0E9450DAC7010E9459DAC8010E94BC
:10A2E00059DA4AE0D42EDA94DD2031F0CE018F55D0
:10A2F0009F4F0E9450DAF7CF8BEE92E10E946BDA0B
:10A30000CF55DF4F188219821A821B82C15AD04062
:10A310003AE0D32EDA94DD2031F0CE018F559F4FF5
:10A320000E9450DAF7CF85E0D82ED982F701D0828B
:10A33000C8010E9459DAC7010E9459DA22E036E0CA
:10A3400048E050E065EF75E082EE95E00E944C50E9
:10A3500022E036E048E050E06DEE75E082EE95E0F8
:10A360000E944C5022E036E044E650E067EB77E094
:10A3700082EE95E00E944C5019828FEFD7018C93AA
:10A38000C8010E9462DAC7010E9459DA22E036E071
:10A3900044E050E06EEF72E082EE95E00E944C5097
:10A3A0008091C6068983C8010E9462DA198A1A8AD6
:10A3B0001B8A1C8A80E090E0A0E8BFE38D879E871F
:10A3C000AF87B88B8091631290916412A09165124F
:10A3D000B091661289839A83AB83BC832CEA35ECF7
:10A3E00047E25EE360916712709168128091691292
:10A3F00090916A120F9480326D837E838F83988749
:10A400002CEA35EC47E25EE360916B1270916C12BE
:10A4100080916D1290916E120F941C2B69877A8730
:10A420008B879C8722E036E044E150E0B80182EE61
:10A4300095E00E944C5084E190E09A838983C801A2
:10A440000E943EDA8091F8119091F911A091FA11D1
:10A45000B091FB1189839A83AB83BC832CEA35ECE2
:10A4600047E25EE36091FC117091FD118091FE1155
:10A470009091FF110F9480326D837E838F83988734
:10A480002CEA35EC47E25EE3609100127091011214
:10A4900080910212909103120F941C2B69877A8786
:10A4A0008B879C87C8010E9447DA8CE0E5E9F2E0DF
:10A4B000D80101900D928A95E1F7C8010E9447DA10
:10A4C0001982C8010E9459DA8FE790E09A83898344
:10A4D000C8010E943EDAE1EAF2E0D80101900D9253
:10A4E000DA94E1F722E036E045E050E0B80182EE90
:10A4F00095E00E944C508091EC058983C8010E9430
:10A5000062DA80E2E6EAF2E0D80101900D928A95E3
:10A51000E1F722E036E040E250E0B80182EE95E05B
:10A520000E944C50F7011082C7010E9462DA80E25B
:10A5300098E00E9462DA8CE198E00E9450DACF55F0
:10A54000DF4F188219821A821B82C15AD040CE0175
:10A550008F559F4F0E9450DA80E2D8011D928A9554
:10A56000E9F722E036E040E250E0B80182EE95E003
:10A570000E944C50FE01F99688E0DF011D928A95F9
:10A58000E9F744E650E060E070E049835A836B836A
:10A590007C834D835E836F83788783E090E0A0E0C7
:10A5A000B0E089879A87AB87BC874D875E876F87C6
:10A5B000788B498B5A8B6B8B7C8B8D8B9E8BAF8B67
:10A5C000B88F898F9A8FAB8FBC8F8D8F9E8FAF8FF7
:10A5D000B8A38EE190E0A0E0B0E089A39AA3ABA37A
:10A5E000BCA38DA39EA3AFA3B8A789A79AA7ABA727
:10A5F000BCA78DA79EA7AFA7B8AB89AB9AABABABF7
:10A60000BCAB8DAB9EABAFABB8AF22E036E040E465
:10A6100050E0B80182EE95E00E944C5090E1D92EB6
:10A62000F8018D2D11928A95E9F722E036E040E19C
:10A6300050E0B80182EE95E00E944C50D8011D9286
:10A64000DA94E9F722E036E040E150E0B80182EE2A
:10A6500095E00E944C5088E299E00E9450DA2CE08C
:10A66000D22EF8018D2D11928A95E9F722E036E07D
:10A670004CE050E0B80182EE95E00E944C508CE630
:10A68000D8011D928A95E9F722E036E04CE650E0C9
:10A69000B80182EE95E00E944C5086ED95E00E9454
:10A6A00047DA22E036E048E050E064EE75E082EE02
:10A6B00095E00E944C50F7011192DA94E9F7C755E2
:10A6C000DF4F1882C95AD04080E090E0A0E4B0E4A7
:10A6D000C356DF4F88839983AA83BB83CD59D0406B
:10A6E000C7010E946BDACE0187559F4F0E9459DA4D
:10A6F000CE0183569F4F0E9450DA80E3D7011D920E
:10A700008A95E9F787EB9CE10E9466388AE00E940F
:10A710002D3822E036E040E350E0B70182EE95E0CC
:10A720000E944C5080910406811128C00091E205DE
:10A730001091E3058091020690910306F701918341
:10A74000808384E690E09093E3058093E20522E025
:10A7500036E044E050E06EE073E082EE95E00E9467
:10A760004C50C7010E943EDA91E00536134009F4CF
:10A7700090E080910406892B809304068091040662
:10A78000811105C060E08BEE9CE10E94D43F8BEC10
:10A790009CE10E9466388AE00E942D389091040660
:10A7A00081E08927C655DF4F0FB6F894DEBF0FBE94
:10A7B000CDBFDF91CF911F910F91FF90EF90DF9070
:10A7C0000895CF93DF9300D01F92CDB7DEB780916D
:10A7D000B2068823C1F083E390E09C838B831A82C6
:10A7E00019829E012F5F3F4F40E150E063EB76E01E
:10A7F000CE0103960E944C508BEC9CE10E9466387F
:10A800008AE00E942D380F900F900F900F90DF91EB
:10A81000CF910895CF92DF92EF92FF92CF93C82FFE
:10A82000809197118150823008F069C00E94C93A26
:10A83000109297110E94C0A96093CE057093CF0526
:10A840008093D0059093D105C090D205D090D305C8
:10A85000E090D405F090D5050E949E2BAB01BC0181
:10A860004093D2055093D3056093D4057093D505DA
:10A870008091B7069091B806A091B906B091BA063A
:10A880008C199D09AE09BF09840F951FA61FB71F1C
:10A890008093B7069093B806A093B906B093BA0612
:10A8A000C1110AC0C1E00E94E1538C2FCF91FF90EB
:10A8B000EF90DF90CF9008958091B5069091B60605
:10A8C00001969093B6068093B5060E949E2BC09089
:10A8D000BB06D090BC06E090BD06F090BE06C61642
:10A8E000D706E806F906F0F60E949E2B6093BB0699
:10A8F0007093BC068093BD069093BE06D3CFC0E094
:10A90000D2CF81E00C940A540E9481C10E948154EC
:10A9100080E00F942C1B809108078130A1F40E94E5
:10A92000354E82E697E00E94663860E088E597E061
:10A930000E94D43F6EE571E080E090E00E94112615
:10A9400088E0809308070895CF92DF92EF92FF92FC
:10A950001F93CF93DF9300D01F92CDB7DEB78EEE5B
:10A96000C82E82E0D82EE12CF12CC982DA82EB824B
:10A97000FC82BE016F5F7F4F8AE50E948B3381119D
:10A980000EC010E0812F0F900F900F900F90DF916D
:10A99000CF911F91FF90EF90DF90CF9008950E948C
:10A9A000E133C982DA82EB82FC82BE016F5F7F4FA6
:10A9B0008AE50E948B33182F882319F30E94354EA5
:10A9C0008CE398E00E9466380E948454DBCFCF92DB
:10A9D000DF92EF92FF921F93CF93DF9300D01F92ED
:10A9E000CDB7DEB78EEEC82E82E0D82EE12CF12C4A
:10A9F000C982DA82EB82FC82BE016F5F7F4F8AE000
:10AA00000E948B3381110EC010E0812F0F900F90A8
:10AA10000F900F90DF91CF911F91FF90EF90DF90FB
:10AA2000CF9008950E94E1330E94AB330E94C63359
:10AA30000E94AB33C982DA82EB82FC82BE016F5F77
:10AA40007F4F8AE00E948B33182F8823E9F20E94FF
:10AA5000354E8FEF97E00E9466380E948454D5CF20
:10AA6000CF93DF9300D01F921F92CDB7DEB781E066
:10AA70008093B20680E1E3EBF6E0DF011D928A9558
:10AA8000E9F70E94E15386E18D8382E390E09C83A5
:10AA90008B831A8219829E012F5F3F4F41E050E065
:10AAA000BE016B5F7F4FCE0103960E944C500F900A
:10AAB0000F900F900F900F90DF91CF910895CF934B
:10AAC000DF93CDB7DEB7A8970FB6F894DEBF0FBE01
:10AAD000CDBF8C01F42E0E9481C10E94354E88E3C7
:10AAE00097E00E9466380115110511F40FE217E096
:10AAF0008091A50580FD79C081608093A5058BE1DB
:10AB000097E00E9466388AE00E942D38CC24C394D6
:10AB10008AE5D82ED0924B14C0924A148FE090E070
:10AB200090934D1480934C1497E0792E70923E14BC
:10AB300022E8E22EE092411434E8832E912CA12CDD
:10AB4000B12C8092421490924314A0924414B0927B
:10AB500045148EEE93E10E94A934D0924B14C0921A
:10AB60004A1488E590E090934D1480934C147092B1
:10AB70003E14E09241148092421490924314A092A9
:10AB80004414B09245148EEE93E10E94A9348AE2F7
:10AB900089838A838B838C83F801DE011596BE013D
:10ABA0006F5F7F4FCD01861B970B2491319621114A
:10ABB0000CC0FB01E80FF91F8AE29F01261B370B2F
:10ABC0002832310524F48193F8CF2D93EBCF20E682
:10ABD00030E140E050E08EEE93E10E94A8E96AE0A7
:10ABE00070E080E090E00E94B22C61E086E297E0A5
:10ABF0000E94A13F89EE93E030E6019729F0232FD0
:10AC00002A950000E9F7F9CFF89489EE93E038EE41
:10AC1000019729F0232F2A950000E9F7F9CF0E9428
:10AC200081C1FF2031F00E94091F0E94221FA895B8
:10AC3000FECF0E94071FF9CF80910707882319F0E4
:10AC400010920707089540E070E060E08EED98E113
:10AC50000E945F558091170D9091180D2FEF3FEFD7
:10AC6000981751F0E92FF0E0E95EF24F228130E0D1
:10AC70009F5F9F779093180DC90108951F920F92BF
:10AC80000FB60F9211240F900FBE0F901F901895C2
:10AC90001F920F920FB60F9211240BB60F920F93C3
:10ACA0001F932F933F934F935F936F937F938F9354
:10ACB0009F93AF93BF93CF93DF93EF93FF93C09195
:10ACC000C6000091180DD091170D11E01D0F1F77D0
:10ACD00090913304913108F09FC0E92FF0E088276C
:10ACE000EB58F94A8F4F0D947D318656B556C456B0
:10ACF000D356DA560C57DE560C57E256E6560C572A
:10AD0000EA56EE56F256F9560C570457C03229F05F
:10AD100028F5CA3011F0CD3031F5011731F0ED2FA3
:10AD2000F0E0E95EF24FC283D12FD093170DFF916F
:10AD3000EF91DF91CF91BF91AF919F918F917F91D3
:10AD40006F915F914F913F912F911F910F910F90B4
:10AD50000BBE0F900FBE0F901F901895CD3481F051
:10AD600081E0CE3471F080E10CC0CA3338F4C033D6
:10AD7000A0F6C03291F2CD32B1F7CFCFCD3499F7F2
:10AD800082E080933304C9CFC13359F018F4C03244
:10AD900021F2E9CF88E0C433A1F38BE0C83389F313
:10ADA000E2CF83E0EECF84E0C03359F386E0C133D5
:10ADB00041F3D9CF85E0C833B1F6E3CF87E0C233A2
:10ADC00091F6DFCF89E0C13371F6DBCF8AE0C03383
:10ADD00051F6D7CF8CE0C73331F6D3CF8DE0C633F1
:10ADE00011F6CFCFC03209F498CF8EE0C33549F2C7
:10ADF000BACF80ED8C0F8A3008F08FCF9FE0909310
:10AE000033048093340489CFCA3019F0CD3009F06F
:10AE100084CF1092330481CFCA3019F0CD3009F0BD
:10AE20007CCF8091A8148823A1F3973089F038F45F
:10AE3000953079F7109244021092AA0CEACF9A301A
:10AE400059F09F3031F7809134040E94C831E1CF2E
:10AE500081E080933006DDCF81E080932F06D9CF4B
:10AE60008EBD0DB407FEFDCF08958FEF8EBD0DB4DE
:10AE700007FEFDCF8EB50895909164009B7F90935F
:10AE80006400982F906A96959CBD80FD03C091E068
:10AE9000863009F490E09DBD0895CF93DF93EB01D8
:10AEA0000E946638CE01DF91CF910C94CBB12F92E6
:10AEB0003F924F925F926F927F928F929F92AF924A
:10AEC000BF92CF92DF92EF92FF920F931F93CF9397
:10AED000DF93009709F0AAC11092FF0C1092FE0CAC
:10AEE0009093A4058093A305BAE0CB2EB0E2DB2EAD
:10AEF000E12CF12C15E002E846015701C4E1D0E055
:10AF0000109291131092901310938413009387134F
:10AF10008092881390928913A0928A13B0928B1317
:10AF200084E393E10E94A93421972FEF821A920AB9
:10AF3000A20AB20A209721F744E1C40ED11CE11CF9
:10AF4000F11C8AE5C81680E2D806E104F104A1F6F6
:10AF5000C12CA0E2DA2EE12CF12CD5E0C2E810924F
:10AF6000911310929013D0938413C0938713C092BF
:10AF70008813D0928913E0928A13F0928B1384E3A2
:10AF800093E10E94A9341092911310929013D093E0
:10AF90008413C0938713D701C6018C529F4FAF4FC4
:10AFA000BF4F8093881390938913A0938A13B09313
:10AFB0008B1384E393E10E94A934EFEFCE1ADE0AEB
:10AFC000EE0AFE0AFAE0CF16F0E2DF06E104F10431
:10AFD00031F6FEEDCF2EF0E2DF2EE12CF12CD5E0A4
:10AFE000C2E81092911310929013D0938413C093DF
:10AFF0008713C0928813D0928913E0928A13F0923B
:10B000008B1384E393E10E94A9342FEFC21AD20A72
:10B01000E20AF20A46EEC41640E2D406E104F10464
:10B0200001F7CC24C394E2E1DE2EE12CF12C0AE0FE
:10B0300010E0D5E0C2E81093911300939013D093E1
:10B040008413C0938713C0928813D0928913E0921F
:10B050008A13F0928B1384E393E10E94A934109336
:10B06000911300939013D0938413C0938713D70147
:10B07000C6018096A11DB11D8093881390938913FA
:10B08000A0938A13B0938B1384E393E10E94A934B5
:10B090008FEFC81AD80AE80AF80AE5E0CE16E2E10E
:10B0A000DE06E104F10439F60091FE0C1091FF0C6C
:10B0B0000115110509F0D6C08091FD0C882309F413
:10B0C000E1C02AE030E240E050E064EF73E084E366
:10B0D00093E10E94A8E9C1E0D0E003E010E0E09035
:10B0E000FE0CF090FF0C35E0332E42E8242E442471
:10B0F0004A94542C64E0662E712C7FE1C72E74E0D4
:10B10000D72E8091FE0C9091FF0C800F911FE816B6
:10B11000F90608F0D5C0C7010E94BFEA882309F4E8
:10B1200081C08091121265E072E1882311F062E122
:10B1300072E1FB0101900020E9F7CF010197861B26
:10B14000970BF4E1FC9F9001FD9F300D1124265FC9
:10B150003F4D50E040E0459710F0FB01128A84E338
:10B1600093E10E94A8E9CE018F5F9D4EB0E0A0E080
:10B1700021964E0124E0880C991C2A95E1F7FDEFF9
:10B180008F1AFFE99F0AB12CA12C2091B41424FF3F
:10B190007EC070929113609290133092841320922B
:10B1A00087138093881390938913A0938A13B09385
:10B1B0008B1384E393E10E94A934D0929113C0923F
:10B1C0009013309284132092871380928813909268
:10B1D0008913A0928A13B0928B1384E393E10E94A7
:10B1E000A934B70183E798E10E943041809112129F
:10B1F00062E172E1811102C065E072E180E798E1ED
:10B200000E944D576AE67CE08CE698E10E944D571B
:10B2100065E072E18BE698E10E944D5787E698E180
:10B220000E9466382FEFE21AF20A6BCF2091FE0CD3
:10B230003091FF0CA901415051096091A305709113
:10B24000A4056817790738F42C5F3F4F3093FF0C43
:10B250002093FE0C45CE4430510508F43DCE2450D9
:10B260003109F4CF0430110569F48091FD0C882375
:10B2700031F083E090E09093FF0C8093FE0CD0E0DF
:10B28000C0E02DCFD0E0C0E004E010E028CF109265
:10B29000911310929013309284132092871380930D
:10B2A000881390938913A0938A13B0938B1384E32C
:10B2B00093E10E94A934509291134092901381CF50
:10B2C000DF91CF911F910F91FF90EF90DF90CF9082
:10B2D000BF90AF909F908F907F906F905F904F90B6
:10B2E0003F902F900895AF92BF92CF92DF92EF924E
:10B2F000FF920F931F93CF93DF93CDB7DEB7E697FF
:10B300000FB6F894DEBF0FBECDBF00915705109168
:10B310005805F80101900020E9F731976F01C01A34
:10B32000D10AF801CF01801B910B8C159D053CF4CF
:10B3300081918F32B9F7DF0111971C92F3CF8BE126
:10B34000E4EDF4E1DE015C9601900D928A95E1F75F
:10B35000F12CE12CEC14FD040CF05DC0F801EE0DB5
:10B36000FF1D8081811103C08FEFE81AF80A580190
:10B37000AE0CBF1CF5018081882309F44CC0FFEF9F
:10B38000EF1AFF0AF801EE0DFF1D7F01E01AF10A26
:10B3900081918111FACFCE014C960E945EB68BE16D
:10B3A000FE017C96DE01119601900D928A95E1F7DF
:10B3B000B501CE0101960E946CAECE0101960E94AD
:10B3C000B52F8FE20E942D388091121281113BC05F
:10B3D00081E094E00E94CBB18091B41484FF1BC043
:10B3E00019821C8221E0A501BE01645E7F4FCE015F
:10B3F00001960E94A0B8811129C08AE00E942D38D0
:10B400000E94394EB50182E597E10E944D57CE0169
:10B4100001960E94B52F8AE00E942D38CE014C96ED
:10B420000E94B52FE6960FB6F894DEBF0FBECDBFD3
:10B43000DF91CF911F910F91FF90EF90DF90CF9010
:10B44000BF90AF90089582E192E1C4CFCE014C96B7
:10B450000E94CDB58BE1FE013196DE015C96019034
:10B460000D928A95E1F7CE0101960E94B52F72CF19
:10B470002F923F924F925F926F927F928F929F9204
:10B48000AF92BF92CF92DF92EF92FF920F931F93F2
:10B49000CF93DF9300D000D000D01F921F92CDB782
:10B4A000DEB7B82E8091040E843008F0D1C10E941E
:10B4B000C0A96B017C018091040E811108C08091AC
:10B4C000170D9091180D891B8F7709F4A4C681E69A
:10B4D000A82E13C08A3019F08D3009F0F6C01092F2
:10B4E000FF0D80919D0D90919E0DFC01E756F24F4E
:10B4F0001682892BF1F40E94CEC48091040E843010
:10B5000008F0ECC08091170D9091180D891B8F7772
:10B5100009F4E4C00E942A5697FFDCCF0E94354E02
:10B5200085EB95E00E9466388091170D8093180D89
:10B53000E4CF10929E0D10929D0D0FE91DE0F801D1
:10B540008191803209F446C08E3409F0A9C060EBC5
:10B5500075E0C8010F94332A4C01892B41F06EE449
:10B5600070E0C80104960F94D434009709F4C80120
:10B570004AE050E070E060E001960F94A3272B01B1
:10B580003C018091990D90919A0DA0919B0DB091E5
:10B590009C0D0196A11DB11D481659066A067B0631
:10B5A00029F060E08DE795E0892851F16AE270E0CA
:10B5B000C8010F9403359C01009729F1982F901B27
:10B5C000912C992349F09150F801E90FF11D8081E8
:10B5D0009826F7CF8F01B3CF4AE050E070E060E0EB
:10B5E000C90101960F94A327292D30E050E040E0D7
:10B5F000621773078407950751F060E08EE595E0C8
:10B600000E94B1F07ACF60E084E395E0F9CF4092F8
:10B61000990D50929A0D60929B0D70929C0D8091A5
:10B6200008078130E1F067E470E0C8010F94D4347A
:10B630000097A9F04AE050E070E060E001960F94B6
:10B64000A327643071058105910548F483E994E0EE
:10B650000E94663860E089E894E00E94D43FC0927E
:10B66000AF07D092B007E092B107F092B207809195
:10B670009F0D8B3309F441CF8091040E843008F084
:10B680003CCF8091060E8A9DC00111246FE97DE0B8
:10B69000895F914F0F94DF3480E00E946BF02DCFD3
:10B6A0008091B41480FFBBCF67EB7DE2C8010F949B
:10B6B000332A009731F0FC01838180538A3008F0EF
:10B6C000AECF60E08AE095E09BCF2DE93DE04FE909
:10B6D0005DE06FEF7DE00E941D1D0FCF8091B414DF
:10B6E00082FFB6C01A82198271E6F72EE0E1EE2ED3
:10B6F000F9E6DF2E8091040E843008F0A9C00E9484
:10B70000551D8111A5C041E050E0BE016B5F7F4F28
:10B7100088E196E10E9420B40D8110E0019711F0BC
:10B720000FEF1FEF8091201690912116A091221605
:10B73000B09123168093B0149093B114A093B214D7
:10B74000B093B3140E94551D0F3F100749F48111A7
:10B7500007C00E94354E83ED95E00E946638CACF3F
:10B760004091060E242F30E00A3061F00D3051F088
:10B77000882309F45FC089819A81009719F00196A6
:10B780009A8389831092BA0489819A81F29EF0018A
:10B79000F39EF00D1124EC5FF14FE80FF91F1382B7
:10B7A000892B69F50E94CEC40E94551D882309F497
:10B7B000A1CF0E949C6188E196E10E94CDB5809165
:10B7C000AB14882391F181508093AB148D9DC001FF
:10B7D000112462E0805C994F0E9422BBE091AB147F
:10B7E00024E0E29FF0011124E45CF94F6081718153
:10B7F000828193810E946E220E94D5AD7BCF1A82F6
:10B80000198281E00E946BF08091B0149091B11484
:10B81000A091B214B091B3148093000E9093010ED6
:10B82000A093020EB093030EBFCF0E94D6B5E09254
:10B83000080760CF4F9DA0011124495F514F9E0121
:10B840002F5F3F4F6AEB74E0802F0E941D1D52CF87
:10B850000E94C0A96B017C01B11004C080919611B7
:10B86000882351F0C092E911D092EA11E092EB11D5
:10B87000F092EC11BB24B39480912F059091300588
:10B88000A0913105B09132050097A105B105B1F045
:10B890004091E9115091EA116091EB117091EC1116
:10B8A000840F951FA61FB71FA7019601281B390BF0
:10B8B0004A0B5B0BDA01C901B7FF92C180911302F9
:10B8C00090911402A0911502B0911602892B8A2B37
:10B8D0008B2B09F099C10E94C0A94B015C0180919A
:10B8E000AA0C811108C02091FC129091FD1281E0F8
:10B8F000291301C080E020915E1230915F1291E027
:10B9000089272A3A31050CF480E091E04091BF0488
:10B910005091C0046091C1047091C204452B462B24
:10B92000472B09F490E0981789F0882309F4BDC1EA
:10B93000D501C40180569444A24FBF4F8093BF04E9
:10B940009093C004A093C104B093C20440907502C8
:10B950005090760260907702709078022091BB043C
:10B960003091BC044091BD045091BE04C301B201AA
:10B970000F94B62A882319F18091BF049091C004D6
:10B98000A091C104B091C2044092BB045092BC0487
:10B990006092BD047092BE04892B8A2B8B2B09F414
:10B9A00049C0D501C40180569444A24FBF4F809333
:10B9B000BF049093C004A093C104B093C2048091CB
:10B9C000BF049091C004A091C104B091C20400973B
:10B9D000A105B10579F1881A990AAA0ABB0AB7FC30
:10B9E00029C01092BF041092C0041092C10410929A
:10B9F000C20483E396E00E94663860E08FE196E03F
:10BA00000E94D43F8091601290916112181619061D
:10BA100024F490E080E00E94251F8091F511909120
:10BA2000F6111816190634F41092F6111092F51149
:10BA30000E9454C18091C7049091C804A091C90488
:10BA4000B091CA0446015701881A990AAA0ABB0A8A
:10BA5000D501C401B7FDB9C12091FC129091FD122E
:10BA60004091350280913402291323C190912C0911
:10BA7000899FC0011124880F892F881F990B9195E8
:10BA80008D8380912D09489FC0011124880F892F33
:10BA9000881F990B91958E830E94C0A969837A8330
:10BAA0008B839C8340E0BE016F5F7F4FCE01059684
:10BAB0000E946F1C6D8170E089E00E94B7A841E090
:10BAC000BE016F5F7F4FCE0105960E946F1C6E8195
:10BAD00070E087E00E94B7A880913B06882309F4B4
:10BAE00067C10091200210912102C80102972091A4
:10BAF000601230916112281739070CF459C18090F7
:10BB0000FD128F82188619861A861B868091FC1278
:10BB10009F80891509F4E7C0892D90E037E6A32EB0
:10BB2000A89EF001A99EF00D1124EF5CF64F458907
:10BB300056896789708D452B462B472B81F4418DA3
:10BB4000528D638D748D452B462B472B41F4458DCB
:10BB5000568D678D70A1452B462B472BE1F127E6CB
:10BB6000B22EB89E9001B99E300D1124A9014F5CF0
:10BB7000564F1A01FA0161817281838194810F9479
:10BB800034344B015C01F10161A172A183A194A144
:10BB90000F94BB2A2B013C01F10165A176A187A17D
:10BBA00090A50F94BB2A9B01AC01C301B2010F9475
:10BBB0008032A50194010F941C2B4B015C01288558
:10BBC00039854A855B850F94E633181624F48886F8
:10BBD0009986AA86BB868F818F5F87708F8396CF69
:10BBE0000E94354E6091AD077091AE0782EE95E0F0
:10BBF0000E944D578AE00E942D3840E070E060E0DE
:10BC000090E080E00E945F559091FC128091FD12BF
:10BC1000981749F0C092E911D092EA11E092EB1125
:10BC2000F092EC1158CEBB2019F01092CB0453CEF9
:10BC30000E94C0A90091E9111091EA112091EB1125
:10BC40003091EC118090130290901402A090150294
:10BC5000B0901602080D191D2A1D3B1D601B710BAB
:10BC6000820B930B97FDE1CF8091CB04811133CEF2
:10BC700081E08093CB045F9A8091AB0C8E7F8093A0
:10BC8000AB0C8A9A8091AB0C8D7F8093AB0C80912A
:10BC9000080180958170809306018091AB0C8B7FA9
:10BCA0008093AB0C0E94071F16CE80E090E0DC0171
:10BCB00045CE2091FD1257E6259F900111242F5C5F
:10BCC000364FF901EF59FF4F9081899FC001112430
:10BCD000880F892F881F990B91958D832E593F4F7F
:10BCE000F9018081D0CE20911A0230911B0240913F
:10BCF0001C0250911D02688579858A859B850F9469
:10BD00001C2B4B015C01B801012E000C880B990B18
:10BD10000F94BD2A9B01AC01C501B4010F9486317B
:10BD200069837A838B839C8340911E0250911F020A
:10BD3000B801CE0101960E948CC489809A80AB80A4
:10BD4000BC804090C3045090C4046090C5047090BF
:10BD5000C604A3019201C501B4010F94B62A87FF5E
:10BD600016C028E431EE4AE75FE3C301B2010F9445
:10BD70001C2B20E037ED43EA5CE30F948631A501EC
:10BD800094010F941C2B69837A838B839C83698134
:10BD90007A818B819C816093C3047093C4048093E7
:10BDA000C5049093C6040F94F232CB010E94251F64
:10BDB000F4E6CF0ED11CE11CF11CC092C704D09256
:10BDC000C804E092C904F092CA040E94CEC48091D3
:10BDD0000807882309F4E0C180912602882309F42A
:10BDE000A3C08091090581119FC080919611811196
:10BDF00008C080919711813021F08091B41482FFA6
:10BE000093C0F894649B10C0809122029091230209
:10BE1000A0912402B09125028093090690930A060E
:10BE2000A0930B06B0930C066091090670910A0668
:10BE300080910B0690910C06789420E030E0A901E7
:10BE40000F94B62A87FF70C001E000930905809126
:10BE50009611811167C088E496E00E9466388AE0F6
:10BE60000E942D3884E08093140D82E08093000DB1
:10BE700081E09AE590934B1480934A148EE490E00D
:10BE800090934D1480934C1487E080933E1482E885
:10BE90008093411484E890E0A0E0B0E080934214E5
:10BEA00090934314A0934414B09345148EEE93E101
:10BEB0000E94A9340E9451400093041240E36CE8B0
:10BEC00076E084E799E00E94564061E088E699E0D8
:10BED0000E9438401091330560E010278CE399E010
:10BEE00069F48AE796E00E94A13F80E30E942D3822
:10BEF0008AE00E942D3860E08DE596E00E94A13F27
:10BF000088E696E00E94663880E30E942D388AE039
:10BF10000E942D38112331F083E696E09093FA0CBD
:10BF20008093F90C0E949C6190910901892F809562
:10BF30008170109100021817C9F02091B41420628A
:10BF40002093B4148093000290FD3FC164EF71E030
:10BF500080E090E00E9411260E94F8B58091B41410
:10BF600083FD7CC1111133C10E94FB350E94C0A921
:10BF70006B017C01109117021123F1F080913405BF
:10BF80008823D1F04091CC045091CD046091CE042F
:10BF90007091CF0446015701841A950AA60AB70A80
:10BFA000B501A40177FD1AC0833009F42FC10CF04C
:10BFB0001EC181300CF023C1212F30E0A8EEB3E088
:10BFC0000F944E31C60ED71EE81EF91EC092CC0447
:10BFD000D092CD04E092CE04F092CF0480919711DC
:10BFE000813009F073C00E94C0A96B017C0180916F
:10BFF000D4049091D504A091D604B091D704A701A0
:10C000009601281B390B4A0B5B0BDA01C901B7FDFE
:10C010003AC0D701C601805F984DAF4FBF4F8093A4
:10C02000D4049093D504A093D604B093D704809001
:10C03000D2059090D305A090D405B090D5050E946C
:10C040009E2BAB01BC014093D2055093D305609366
:10C05000D4057093D5058091B7069091B806A0914C
:10C06000B906B091BA0688199909AA09BB09840FC3
:10C07000951FA61FB71F8093B7069093B806A0938D
:10C08000B906B093BA068091D0049091D104A091E2
:10C09000D204B091D30446015701881A990AAA0A1A
:10C0A000BB0AD501C401B7FD11C020E8C20E2EEEB7
:10C0B000D21E26E3E21EF11CC092D004D092D1041D
:10C0C000E092D204F092D3040E94E1530E94A4397A
:10C0D0000E946E4180912E05882379F10E94C0A9AB
:10C0E0006B017C0180912A0590912B05A0912C0574
:10C0F000B0912D0546015701881A990AAA0ABB0A70
:10C10000D501C401B7FD19C020912E0530E0A8EE7D
:10C11000B3E00F944E31C60ED71EE81EF91EC09232
:10C120002A05D0922B05E0922C05F0922D0580E097
:10C130000E94B2BD8AE00E942D3880912905882393
:10C1400059F10E94C0A96B017C0180912505909155
:10C150002605A0912705B0912805A7019601281B67
:10C16000390B4A0B5B0BDA01C901B7FD15C02091F1
:10C17000290530E0A8EEB3E00F944E31C60ED71E6D
:10C18000E81EF91EC0922505D0922605E0922705EB
:10C19000F09228050E9493AD2B960FB6F894DEBF5F
:10C1A0000FBECDBFDF91CF911F910F91FF90EF9008
:10C1B000DF90CF90BF90AF909F908F907F906F90C7
:10C1C0005F904F903F902F9008950E94E7B51230F6
:10C1D00008F0CCCE0E94FB3560E085EC96E050C0C4
:10C1E00083ED96E09093FA0C8093F90CBFCE8430E7
:10C1F00009F0E2CE0E94394E8AED96E004C00E941A
:10C20000394E89E097E00E946638D6CE0E94394EBA
:10C2100082EF96E0F8CF8091AF079091B007A091A0
:10C22000B107B091B207A7019601281B390B4A0B41
:10C230005B0BDA01C901885E9340A109B109B7FD22
:10C2400046C98DEC95E00E946638C092AF07D09247
:10C25000B007E092B107F092B20739C9123098F4F2
:10C260008DE996E00E9466388AE00E942D380E948F
:10C27000CD2C90E080E00E94575760E086EB96E07E
:10C280000E94D43F73CE123009F070CE0E9452BA91
:10C29000882379F081E00E9428BA42EB50E069E3FC
:10C2A00078E089EB94E10E9420B489EB94E10E944C
:10C2B000CDB50E94A32F811193CF0E948D2F0E9494
:10C2C000CEBA0E9423BA52CECF93DF938091FC1254
:10C2D0009091FD12891B8095877019F40E94385A3D
:10C2E000F5CF8091FC128F5F8770A091FC1297E6CA
:10C2F000A99FD0011124FD01EF5CF64FEF011992C7
:10C300009A95E9F798E09083AA5BB64F90E1EEE04A
:10C31000F3E101900D929A95E1F72091FC12909132
:10C32000FD12291303C094E69093F9128093FC1236
:10C33000DF91CF910C94BB2F9091FC128091FD1254
:10C34000981306C080912F0990913009892B21F014
:10C3500080E00E94385AF0CF0895CF92DF92EF929A
:10C36000FF92FC01C080D180E280F3802091D10C4B
:10C370003091D20C4091D30C5091D40CC701B6012E
:10C380000F941C2B0F94F33360931A1370931B13A9
:10C3900080931C1390931D13C0920A13D0920B1319
:10C3A000E0920C13F0920D139091FC128091FD120B
:10C3B000981731F0FF90EF90DF90CF900C9464616C
:10C3C0000E949C610E94112A40911A1350911B13E4
:10C3D00060911C1370911D1340932B0650932C06F3
:10C3E00060932D0670932E06882331F0FF90EF9016
:10C3F000DF90CF900C94BB2FFF90EF90DF90CF9009
:10C4000008954F925F926F927F928F929F92AF9218
:10C41000BF92CF92DF92EF92FF920F931F93CF9331
:10C42000DF93EC018B017A016901F901808191812F
:10C43000A281B381FA014081518162817381F80147
:10C4400080809180A280B380488059806A807B8000
:10C450004092FE125092FF126092001370920113EC
:10C460008092021390920313A0920413B0920513CA
:10C4700040930613509307136093081370930913A6
:10C4800080930A1390930B13A0930C13B0930D1386
:10C490002091D10C3091D20C4091D30C5091D40CFE
:10C4A000F60160817181828193810F941C2B0F941E
:10C4B000F3334B015C012091CD0C3091CE0C4091B7
:10C4C000CF0C5091D00CF7016081718182819381F2
:10C4D0000F941C2B0F94F3336B017C012091C90C3A
:10C4E0003091CA0C4091CB0C5091CC0CF80160817A
:10C4F0007181828193810F941C2B0F94F3332B0154
:10C500003C012091C50C3091C60C4091C70C509154
:10C51000C80C688179818A819B810F941C2B0F94B0
:10C52000F33360930E1370930F1380931013909353
:10C5300011134092121350921313609214137092BD
:10C540001513C0921613D0921713E0921813F0929D
:10C55000191380921A1390921B13A0921C13B0927D
:10C560001D139091FC128091FD12981791F0DF91AC
:10C57000CF911F910F91FF90EF90DF90CF90BF90E0
:10C58000AF909F908F907F906F905F904F900C94A2
:10C5900064610E949C610E94112A4091161350917F
:10C5A00017136091181370911913009112131091C1
:10C5B00013132091141330911513C0900E13D090C3
:10C5C0000F13E0901013F0901113C0921F06D09239
:10C5D0002006E0922106F092220600932306109393
:10C5E0002406209325063093260640932706509371
:10C5F00028066093290670932A0640911A135091D9
:10C600001B1360911C1370911D1340932B065093C4
:10C610002C0660932D0670932E06882391F0DF91EF
:10C62000CF911F910F91FF90EF90DF90CF90BF902F
:10C63000AF909F908F907F906F905F904F900C94F1
:10C64000BB2FDF91CF911F910F91FF90EF90DF9063
:10C65000CF90BF90AF909F908F907F906F905F90A2
:10C660004F9008953F924F925F926F927F928F9278
:10C670009F92AF92BF92CF92DF92EF92FF920F9371
:10C680001F93CF93DF93CDB7DEB768970FB6F894BB
:10C69000DEBF0FBECDBFD82E2A013B014801590194
:10C6A0003E2C20E030E0A901C501B8010F94B62A64
:10C6B000811110C081E08D1508F0B6C060E070E017
:10C6C00080E793E420E030E040E752E40F948032CA
:10C6D0004B015C018D8A9E8AAF8AB88E0D2D10E0C9
:10C6E000F801E853F64EE491BB24B3941E160CF403
:10C6F000B12CCC24C39420E030E0A901C301B201E5
:10C700000F94E63318160CF0C12CBC1471F092E0B3
:10C71000D9120BC0332049F081E00F942C1B69E142
:10C7200070E080E090E00E94112680E00E94C12F1E
:10C7300069837A838B839C8381E00E94C12F6D8300
:10C740007E838F83988782E00E94C12F69877A87D2
:10C750008B879C8783E00E94C12F6D877E878F87A0
:10C76000988B000F111F000F111FE1E0F0E0EC0F9C
:10C77000FD1F0E0F1F1FF8011082118212821382FB
:10C780009E01235F3F4FAE01475F5F4FBE016B5F6E
:10C790007F4FCE0101960E940162F80140825182D2
:10C7A00062827382198A1A8A1B8A1C8A80912F09D5
:10C7B00090913009892B91F4CE0141967C018E0134
:10C7C0000B5E1F4F9E01235F3F4FAE01475F5F4FE0
:10C7D000BE016B5F7F4F40970E94D5F00E949C6125
:10C7E000BC1451F092E0D91205C0332019F080E05A
:10C7F0000F942C1B0E941C5668960FB6F894DEBF4F
:10C800000FBECDBFDF91CF911F910F91FF90EF90A1
:10C81000DF90CF90BF90AF909F908F907F906F9060
:10C820005F904F903F90089560E070E88BE395E44F
:10C8300049CF4F925F926F927F928F929F92AF9269
:10C84000BF92CF92DF92EF92FF920F931F93CF93FD
:10C85000DF93CDB7DEB72C970FB6F894DEBF0FBECF
:10C86000CDBF2B013C0129873A874B875C87470165
:10C870005801F601E080F1800281138120E030E070
:10C88000A901B701C8010F94B62A882309F488C00A
:10C890005E2D4F2D302F212F852F942FA32FB22FB8
:10C8A00089839A83AB83BC8320E030E0A901B70180
:10C8B000C8010F94B62A811108C0E0904502F0909B
:10C8C00046020091470210914802C701D8018D83AA
:10C8D0009E83AF83B887A501940160917102709126
:10C8E000720280917302909174020F94B62A87FFAE
:10C8F0000CC08092710290927202A0927302B09268
:10C900007402CE0101960E94EC2A40926902509274
:10C910006A0260926B0270926C0289859A85AB857F
:10C92000BC8580936D0290936E02A0936F02B093CA
:10C930007002CE0105960E94EC2AA5019401609137
:10C9400071027091720280917302909174020F943F
:10C95000E633181664F48092710290927202A092EB
:10C960007302B0927402CE0101960E94EC2A0E94DA
:10C970009C612C960FB6F894DEBF0FBECDBFDF9141
:10C98000CF911F910F91FF90EF90DF90CF90BF90CC
:10C99000AF909F908F907F906F905F904F90089591
:10C9A00050E040E030E820E477CFCF92DF92EF9282
:10C9B000FF920F931F936A01E0907102F090720250
:10C9C0000091730210917402FB0120813181428138
:10C9D0005381FC0160817181828193810E9419647D
:10C9E0001F910F91FF90EF90DF90CF900895CF921D
:10C9F000DF92EF92FF920F931F936B01FC01E08097
:10CA0000F18002811381E9E6F2E0248135814681DB
:10CA1000578160817181828193810E9419641F9185
:10CA20000F91FF90EF90DF90CF9008950F931F9399
:10CA3000CF93DF93EC018B0181E00F942C1B69E114
:10CA400070E080E090E00E941126B801CE010E94C3
:10CA5000F764C091070780E00F942C1B1092070722
:10CA600082E00E94EB2F0E94072BC2FBCC27C0F96B
:10CA700081E08C27DF91CF911F910F910895AF92A4
:10CA8000BF92CF92DF92EF92FF920F931F93CF93BB
:10CA9000DF9300D01F92CDB7DEB7FC01E080F180BC
:10CAA00002811381611112C0A0907102B0907202D4
:10CAB000C0907302D09074029501A601B701C8011D
:10CAC0000F94B62A87FF02C07501860120E030E08E
:10CAD00048EC53E4B701C8010F94B62A87FD04C09F
:10CAE000E12CF12C08EC13E4C701D80189839A8367
:10CAF000AB83BC836AEF72E0CE0101960E94F764BB
:10CB00000F900F900F900F90DF91CF911F910F9189
:10CB1000FF90EF90DF90CF90BF90AF9008953F923D
:10CB20004F925F926F927F928F929F92AF92BF923D
:10CB3000CF92DF92EF92FF920F931F93CF93DF93E9
:10CB400000D01F92CDB7DEB7382E80E090E0A0E293
:10CB5000B1E489839A83AB83BC83C090F312D090F5
:10CB6000F412E090F512F090F61220E030E0A90106
:10CB7000C701B6010F94B62A87FF0CC0A701960122
:10CB800060E070E080E291E40F94853169837A83FC
:10CB90008B839C8360E0CE0101960E943F654090AC
:10CBA000690250906A0260906B0270906C028090F3
:10CBB0006D0290906E02A0906F02B09070023320D0
:10CBC00089F10E94E75419821A821B821C82E0902C
:10CBD0007102F09072020091730210917402CE0102
:10CBE00001966C01A5019401C301B2010E94196470
:10CBF0003092AB070E948F2B0F900F900F900F90E9
:10CC0000DF91CF911F910F91FF90EF90DF90CF9028
:10CC1000BF90AF909F908F907F906F905F904F905C
:10CC20003F9008950E94A454CECF8091AB078823F3
:10CC300019F080E00E948F6580E008952F923F9266
:10CC40004F925F926F927F928F929F92AF92BF921C
:10CC5000CF92DF92EF92FF920F931F93CF93DF93C8
:10CC6000CDB7DEB766970FB6F894DEBF0FBECDBF67
:10CC7000F82E282E312CF101E853F64ED49022E004
:10CC8000821335C08091AB07811103C081E00E94FF
:10CC90008F650E94E754811139C184EC99E10E94AB
:10CCA0008E1D20E030E0A9010F94B62A8823F9F008
:10CCB0006D2DDD0C770B880B990B0F94BD2A2B0182
:10CCC0003C0184EC99E10E948E1D4B015C0120E047
:10CCD00030E040EA50E40F94B62A11E087FF1CC010
:10CCE000812C912C90EAA92E90E4B92E15C06D2DBF
:10CCF000DD0C770B880B990B0F94BD2A2B013C019F
:10CD0000C101880F991F880F991F8454964E0E9465
:10CD10008E1D4B015C0110E0A3019201C501B4011D
:10CD20000F941C2B4B015C016101CC0CDD1CCC0C65
:10CD3000DD1CC6018055964E0E948E1DEE24E394A4
:10CD4000E12620E030E040EC5FE30F941C2BA301D0
:10CD500092010F941C2BAB01BC0100E010E0980184
:10CD60008F2D0E94326320E030E0A901C501B4019B
:10CD70000F94B62AF601EC55F64EFA8BE98B882310
:10CD800009F44DC0F2E000E010E020E431E4FF16C9
:10CD900019F000E010E09801B501A4017058E12CF1
:10CDA0008F2D0E943263A5019401C501B4010F9437
:10CDB00086316B8B7C8B8D8B9E8B22E0F216E9F09B
:10CDC000F101EF55F64E6491611107C00E94394E92
:10CDD0008FE799E10E9466386AE070E090E080E0B9
:10CDE0000F94BB2A9B01AC0160E070E088E492E400
:10CDF0000F9480328B019C0104C000E010E020EC15
:10CE000030E4EE24E3944B895C896D897E898F2D13
:10CE10000E94326332E0F312D0C00E94A45481E039
:10CE200090E0A0E0B0E00F2C04C0880F991FAA1F6B
:10CE3000BB1F0A94D2F72091AB0C282B2093AB0C8C
:10CE40002091BD05822B8093BD0589899A890E9416
:10CE50008E1DF601E759FD4F6083718382839383B2
:10CE600082E0F8121AC02091F3123091F41240912E
:10CE7000F5125091F61260917102709172028091D8
:10CE80007302909174020F948531609371027093D4
:10CE900072028093730290937402F601EF5DF74F74
:10CEA00010821182128213828F2D0E94AB1C0E946D
:10CEB000072BF601E759FD4F80819181A281B38153
:10CEC000F601E556F84F80839183A283B38392E005
:10CED000F916A9F18CE0E6ECF2E0DE011196019082
:10CEE0000D928A95E1F7E1E0F0E0EC0FFD1FEC0D0B
:10CEF000FD1D80809180A280B38020E030E0A901F8
:10CF0000C501B4010F94B62A81111EC066960FB6F2
:10CF1000F894DEBF0FBECDBFDF91CF911F910F916F
:10CF2000FF90EF90DF90CF90BF90AF909F908F9049
:10CF30007F906F905F904F903F902F9008950E9448
:10CF400015668111E3CFC6CF20E030E0A901C5010D
:10CF5000B4010F94E63387FF04C0B7FAB094B7F872
:10CF6000B094F601E759FD4F6F01A3019201C5018D
:10CF7000B4010F941C2B9B01AC01F60160817181FF
:10CF8000828193810F948531F6016083718382835E
:10CF90009383F2E080E090E0A0E4B1E4FF1621F09A
:10CFA00080E090E0A8E4B2E48D879E87AF87B88BDD
:10CFB000CE010D960E94EC2AA9CF81E090E0A0E07E
:10CFC000B0E00F2C04C0880F991FAA1FBB1F0A9442
:10CFD000D2F72091AB0C282B2093AB0C2091BD05F0
:10CFE000822B8093BD0589899A890E948E1DF60146
:10CFF000E759FD4F60837183828393834ECFCF9334
:10D00000DF9300D01F92CDB7DEB780E090E0A0EABA
:10D01000B0E489839A83AB83BC8361E0CE0101963F
:10D020000E943F650F900F900F900F90DF91CF916E
:10D0300008958F929F92AF92BF92CF92DF92EF921C
:10D04000FF920F931F93CF93DF93CDB7DEB72C974B
:10D050000FB6F894DEBF0FBECDBF8B0140E050E0AD
:10D0600068E472E44D835E836F83788740E050E02C
:10D0700060EA70E449875A876B877C878130B9F111
:10D08000823009F459C020E030E040E050E4609183
:10D0900071027091720280917302909174020F94E8
:10D0A00086314B017C0120E030E048EC53E40F94E2
:10D0B000E633181634F4812C912C88ECE82E93E496
:10D0C000F92EF801A084B184C284D3849401A7010D
:10D0D000B501C6010F94E633181614F05401670128
:10D0E000C501D60189839A83AB83BC8348C0BE0146
:10D0F000675F7F4FC80108960E94F764B8016C5FB4
:10D100007F4FAE014B5F5F4FC8010E94D5640E9404
:10D11000BB302C960FB6F894DEBF0FBECDBFDF91AB
:10D12000CF911F910F91FF90EF90DF90CF90BF9024
:10D13000AF909F908F900895F801208531854285AA
:10D140005385609171027091720280917302909187
:10D1500074020F9486316B017C0120E030E048ECD2
:10D1600053E40F94B62A87FD06C0C12CD12C28ECBD
:10D17000E22E23E4F22EC982DA82EB82FC82BE0127
:10D18000675F7F4FCE010196B7CFEF92FF920F936B
:10D190001F93CF93DF937C018B010E94B531C9E6C9
:10D1A000D2E02091790230917A0240917B02509135
:10D1B0007C02F70160817181828193810F948032BA
:10D1C0002C853D854E855F850F9486316C877D87E4
:10D1D0008E879F87C8010E94EC2ADF91CF911F9113
:10D1E0000F91FF90EF900C949C614F925F926F9221
:10D1F0007F92AF92BF92CF92DF92EF92FF920F9306
:10D200001F93CF93DF9300D000D01F921F92CDB712
:10D21000DEB75C0180E090E0A0E7B2E489839A8306
:10D22000AB83BC8380E090E0A0E8B0EC8D839E836C
:10D23000AF83B887BE016F5F7F4FCE0105960E9416
:10D24000C56868E873E180E090E00E941126C12C77
:10D25000D12C88ECE82E81E4F82EC982DA82EB82A8
:10D26000FC8280E090E0A0E8B0E48D839E83AF83F1
:10D27000B887BE016F5F7F4FCE0105960E94C568DB
:10D2800001EB1CE0F80140AC51AC62AC73ACC0AE39
:10D29000D1AEE2AEF3AE80E090E0A0E2B2E48983EA
:10D2A0009A83AB83BC83F50180819181A281B38194
:10D2B0008D839E83AF83B887BE016F5F7F4FCE01A2
:10D2C00005960E94C568F80140AE51AE62AE73AEDD
:10D2D000129A64E670E080E090E00E94112681E0FE
:10D2E00028960FB6F894DEBF0FBECDBFDF91CF9169
:10D2F0001F910F91FF90EF90DF90CF90BF90AF9074
:10D300007F906F905F904F9008951F93CF93DF931E
:10D31000CDB7DEB72C970FB6F894DEBF0FBECDBFEA
:10D32000182F882379F020E030E0A9016091F505FD
:10D330007091F6058091F7059091F8050F94B62A43
:10D340008823F9F08091AC0C8117D9F00E949C6180
:10D350008CE0E2EDF2E0DE01119601900D928A95EB
:10D36000E1F7CE0101960E943A1F8091AC0C882310
:10D3700091F089E692E00E9413271092AC0C0E9473
:10D38000072B2C960FB6F894DEBF0FBECDBFDF91F2
:10D39000CF911F91089581E08093AC0C89E692E0D3
:10D3A0000E942721ECCF2F923F924F925F926F9273
:10D3B0007F928F929F92AF92BF92CF92DF92EF9225
:10D3C000FF920F931F93CF93DF93CDB7DEB7CB546C
:10D3D000D1090FB6F894DEBF0FBECDBF2DB73EB753
:10D3E00039AF28AF87E00E94494E81110BC061E040
:10D3F00086E50E945F248DA3853060F087E39EE080
:10D400000E946638A8ADB9AD0FB6F894BEBF0FBE86
:10D41000ADBF40C33DA1332321F087E19EE00E94D0
:10D4200066386AE080E50E945F24182F8CEF810F38
:10D430008F3218F083EF9DE0E3CF60E085E40E9437
:10D440007B24882309F448C081E08FABE090F71279
:10D45000F090F812D7012D913D914D915C91609122
:10D46000690270916A0280916B0290916C020F9434
:10D470008631AB01BC0188E50E94CD2469877A879B
:10D480008B879C87F7012481358146815781609184
:10D490006D0270916E0280916F02909170020F94F4
:10D4A0008631AB01BC0189E50E94CD246D877E8762
:10D4B0008F87988BBE01635F7F4FCE0109960E94D4
:10D4C0005B2E382E81110BC063E68FED9DE00E942C
:10D4D000D43F87EC9DE094CF92E09FABB7CF8CE434
:10D4E0000E944F1E082F882309F431C10E944B244B
:10D4F0008EA3803118F080EA9DE082CFFEA1F1304A
:10D5000009F427C160E083E50E947B248AAF882369
:10D5100021F0011102C037E03EA38DA1833020F03D
:10D5200086E89DE00E9466389091AC0C9DAF80E04B
:10D530000E9485690E94E41C1D8A1E8A1F8A188E1B
:10D54000198E1A8E1B8E1C8E83EF9FE4A3ECB7E41A
:10D550008D8F9E8FAF8FB8A383EF9FE4A3ECB7ECC2
:10D5600089A39AA3ABA3BCA3A12FB0E0BCA7ABA790
:10D57000EDB7FEB724E0129FE019F10911240FB6B0
:10D58000F894FEBF0FBEEDBF8DB79EB701969CAF5E
:10D590008BAF2DA14FA9BE01635F7F4FCE010996CE
:10D5A0000F940E1C9B01AC010F947834811162C260
:10D5B0000E94C0A9611571058105910511F00F94B4
:10D5C0003C26212C1BAA1CAA1DAA1EAAAEA1A15052
:10D5D000BB0B2C96BFAFAEAF2C97E22DF0E0F8A7B7
:10D5E000EFA32BA53CA5E217F3070CF074C231960C
:10D5F000FEA7EDA73F932F93FF93EF9382E79DE064
:10D600009F938F938CE79DE09F938F931F920F942E
:10D610004A1B8DB79EB709960FB6F8949EBF0FBEF2
:10D620008DBF9EA1992309F458C10F94ED252AE0DE
:10D6300030E040E050E00F941C310F94BD2A20E010
:10D6400030E040EA50E40F94E6330FEF1FEF181676
:10D6500014F001E010E00F94ED2528E631E040E001
:10D6600050E00F941C310F94BD2A2B013C010F9404
:10D67000ED2528E230E040E050E00F941C316B5F74
:10D680007F4F8F4F9F4F0F94BD2A4B015C01ADA17F
:10D69000A430D1F4BC01A40184E69DE00E94424183
:10D6A000B301A2018CE59DE00E94424186E59DE028
:10D6B0000E9466380130110519F483E40E942D3868
:10D6C00082E59DE00E946638312CC801110FAA0B3B
:10D6D000BB0B2A968CAF9DAFAEAFBFAF2A972C96EF
:10D6E000AEADBFAD2C973A161B060CF0F6C02A96CD
:10D6F0006CAD7DAD8EAD9FAD2A970F94BD2A6B01A9
:10D700007C01BAADBB2341F1AC019B010F94863182
:10D7100020E030E040E952E40F941C2B9B01AC0167
:10D72000C301B2010F9486312B013C0120E030E0AF
:10D7300044EB53E40F94E6331816FCF420E030E099
:10D7400044EB53E4C301B2010F948531EDCF1EA227
:10D75000D9CE22E02EA3D6CE0F94ED2524E130E0E1
:10D7600040E050E00F941C31675E7F4F8F4F9F4F1A
:10D770000F94BD2AA7019601CFCF20E030E0A90188
:10D78000C301B2010F94B62A87FF0BC020E030E03E
:10D7900044EB53E4C301B2010F9486312B013C01E9
:10D7A000ECCF0091F7121091F812F8012481358125
:10D7B000468157816D857E858F8598890F94853147
:10D7C00022966CAF7DAF8EAF9FAF22972BED3FE0DF
:10D7D00049E450E4C301B2010F941C2B20E030E077
:10D7E00044E353E40F9480326B017C010F947B324D
:10D7F0006FA778AB89AB9AABD8012D913D914D9134
:10D800005C9169857A858B859C850F9485312696F8
:10D810006CAF7DAF8EAF9FAF2697A50194016FA52A
:10D8200078A989A99AA90F941C2B9B01AC01269673
:10D830006CAD7DAD8EAD9FAD26970F94863169831B
:10D840007A838B839C83C701B6010F942634A5018C
:10D8500094010F941C2B22962CAD3DAD4EAD5FADC7
:10D8600022970F9486316D837E838F83988748E655
:10D8700051E070E060E0CE0101960E948CC448E661
:10D8800051E070E060E0CE0105960E948CC4BDA11D
:10D89000B43099F449815A816B817C8186E49DE0A2
:10D8A0000E9442414D815E816F81788580E79FE2D1
:10D8B0000E9442418AE00E942D38198A1A8A1B8AE6
:10D8C0001C8AAE014F5E5F4FBE016B5F7F4FCE0182
:10D8D00001960E94D564339402CF20E04FA9BE0187
:10D8E000635F7F4FCE0109960F940E1C4B015C01C4
:10D8F000312CAC019B010F947834811102C0332488
:10D900003394A5019401C501B4010F9478348111B9
:10D91000E2C0EFA1F8A5EE0FFF1FEE0FFF1F2BAD2A
:10D920003CADE20FF31F80829182A282B382A501F7
:10D9300094016D8D7E8D8F8D98A10F94E63318160E
:10D9400024F48D8E9E8EAF8EB8A2A501940169A19C
:10D950007AA18BA19CA10F94B62A87FF04C089A24B
:10D960009AA2ABA2BCA2A50194016BA97CA98DA926
:10D970009EA90F9486316BAB7CAB8DAB9EABADA5F6
:10D98000BEA5BD01BB0F880B990B0F94BD2A6FA3D9
:10D9900078A789A79AA79B01AC016BA97CA98DA93F
:10D9A0009EA90F9480322B013C014D8A5E8A6F8ABA
:10D9B000788EEBADFCADF8ABEFA710E0C12CD12C0D
:10D9C0007601AFA5B8A96D917D918D919D91B8AB70
:10D9D000AFA7A30192010F9485319B01AC010F9475
:10D9E0001C2B9B01AC01C701B6010F9486316B0162
:10D9F0007C011F5F211628F72FA138A549A55AA53C
:10DA00000F9480320F943434698F7A8F8B8F9C8F70
:10DA1000BDA1B23068F18DA59EA50E9402EA6BA55A
:10DA20007CA581E49DE00E9464418BE39DE00E941F
:10DA3000663843E0C501B4010E940EBD80E20E9439
:10DA40002D3881E0EDA1E3300CF480E0E12C8E0173
:10DA50000F5D1F4F9E01235E3F4FAE01475E5F4F3C
:10DA6000BE016B5E7F4F0E94233F8AE00E942D38EB
:10DA70002394B3CD0E9415660E94CB1C8DAD0E94ED
:10DA800085690E94BB3088AD99AD0FB6F8949EBFF2
:10DA90000FBE8DBFE8ADF9AD0FB6F894FEBF0FBE57
:10DAA000EDBFC55BDF4F0FB6F894DEBF0FBECDBF35
:10DAB000DF91CF911F910F91FF90EF90DF90CF906A
:10DAC000BF90AF909F908F907F906F905F904F909E
:10DAD0003F902F9008950E941566332069F280E3ED
:10DAE0009DE00E94663881E0FDA11F160CF080E0E9
:10DAF000EE24E3948E010F5D1F4F9E01235E3F4F86
:10DB0000AE01475E5F4FBE016B5E7F4F0E94233FB9
:10DB1000698D7A8D8B8D9C8D0052110926E042E033
:10DB20000F9483259F938F938FE19DE09F938F9315
:10DB300089E29DE09F938F931F920F944A1B2DB70C
:10DB40003EB7295F3F4F0FB6F8943EBF0FBE2DBFC3
:10DB500093CF2F923F924F925F926F927F928F92CC
:10DB60009F92AF92BF92CF92DF92EF92FF920F936C
:10DB70001F93CF93DF93CDB7DEB76A970FB6F894B4
:10DB8000DEBF0FBECDBF83E50E944F1E182F309021
:10DB9000AC0C882319F00E946B24382E4090690247
:10DBA00050906A0260906B0270906C0280916D02DE
:10DBB00090916E02A0916F02B09170028B8B9C8B42
:10DBC000AD8BBE8B8091710290917202A091730215
:10DBD000B09174028F8B988FA98FBA8F112329F07F
:10DBE000311003C080E00E94856986E50E944F1EC7
:10DBF0008A8B20E030E0A9016091F5057091F6056F
:10DC00008091F7059091F8050F94B62A882309F4BE
:10DC1000C9C083E40E944F1E882309F49DC00E945E
:10DC2000A3246B017C01A7EBB7E0B987A887BF836A
:10DC3000AE83F5E0FD831D861E8628EC2F8702EC5F
:10DC40001A86212C88EC8B8792E49C87AE81BF8159
:10DC5000B98BA88B15E0E889F98981909190A19002
:10DC6000B190F98BE88B2A85322D4B855C85C501F7
:10DC7000B4010F94B62A87FF04C08A86292CAB868C
:10DC8000BC862D853E854F85502FC501B4010F946C
:10DC9000E633181624F48D869E86AF860B2D115020
:10DCA000D1F6FD81F150FD838E819F8144969F8343
:10DCB0008E83F111CBCF2D853E854F85502F6A8500
:10DCC000722D8B859C850F94863120E030E040E0FA
:10DCD0005FE30F941C2BA70196010F9486314B0133
:10DCE0005C012DEB37E346E855EB0F94E63387FDF7
:10DCF0000AC02DEB37E346E855E3C501B4010F94A4
:10DD0000B62A18164CF580E00E94856910E0E88478
:10DD1000F98400E0D7016D917D918D919D917D01F8
:10DD20006D01B4E0CB1AD108A50194010F9485319F
:10DD3000F6016083718382839383602F812F0F9418
:10DD40001F1A0F5F053031F71F5F8885998544964C
:10DD5000998788871530D9F6AA89AA2381F020E00F
:10DD600030E0A9016091F5057091F6058091F70505
:10DD70009091F8050F94B62A81110E94AB408AE574
:10DD80000E944F1E882351F00E94A32469837A8346
:10DD90008B839C83CE0101960F94E718832D0E94FC
:10DDA00085690BC0311003C09A89992341F30E9401
:10DDB000394E80E69CE00E946638332051F0809115
:10DDC000AC0C811106C00E94354E81E49CE00E949B
:10DDD00066380E94394E83E39CE00E946638809149
:10DDE000AC0C0E9424410E94394E86E29CE00E94C5
:10DDF0006638C090F308D090F408E090F508F090F1
:10DE0000F60820E030E0A901C701B6010F94E6331F
:10DE100018160CF053C042E0C701B6010E940EBDB7
:10DE20008DE00E942D388AE00E942D38A3019201D6
:10DE30006091690270916A0280916B0290916C020C
:10DE40000F94B62A81111FC02B893C894D895E89A8
:10DE500060916D0270916E0280916F0290917002DC
:10DE60000F94B62A81110FC02F89388D498D5A8D94
:10DE700060917102709172028091730290917402AC
:10DE80000F94B62A81110E94BB306A960FB6F8949F
:10DE9000DEBF0FBECDBFDF91CF911F910F91FF90DD
:10DEA000EF90DF90CF90BF90AF909F908F907F903A
:10DEB0006F905F904F903F902F90089581E29CE08B
:10DEC0000E946638B3CF8F929F92AF92BF92EF922B
:10DED000FF920F931F93CF93DF9380E00E94856999
:10DEE0001092F1051092F2051092F3051092F405CC
:10DEF0001092ED051092EE051092EF051092F005CC
:10DF00001092F9051092FA051092FB051092FC058B
:10DF10001092F5051092F6051092F7051092F8058B
:10DF200007EB17E0C0E0812C912C80ECA82E8FE746
:10DF3000B82E7801D0E0F70181929192A192B1922E
:10DF40007F016D2F8C2F0F941F1ADF5FD53099F74B
:10DF5000CF5F0C5E1F4FC53061F7DF91CF911F91EE
:10DF60000F91FF90EF90BF90AF909F908F9008958A
:10DF70009091FC128091FD12981308C080912F0996
:10DF800090913009892B11F40C94091F80E00E94B4
:10DF9000385AEECF83E50E949D1E8823E9F00E9447
:10DFA000C0A96093E9117093EA118093EB119093EB
:10DFB000EC110E94A32420E030E04AE754E40F94DF
:10DFC0001C2B0F94F9326093130270931402809308
:10DFD00015029093160208958091530584FD0AC09E
:10DFE0008091550587FD06C080915605837011F418
:10DFF0000C94B86F0E949C6188E50E944F1E882394
:10E0000031F05F9A8091AB0C8E7F8093AB0C89E5E9
:10E010000E944F1E882331F08A9A8091AB0C8D7F2D
:10E020008093AB0C8AE50E944F1E882359F08091A3
:10E03000080180958170809306018091AB0C8B7FE5
:10E040008093AB0C85E40E944F1E81110C94071F36
:10E0500008952F923F924F925F926F927F928F928C
:10E060009F92AF92BF92CF92DF92EF92FF920F9367
:10E070001F93CF93DF93CDB7DEB7A6970FB6F89473
:10E08000DEBF0FBECDBF8BE997E00E94342A80919E
:10E09000690C83FD7EC0209175023091760240911B
:10E0A0007702509178026091A7077091A80780913C
:10E0B000A9079091AA070F94B62A882309F469C08A
:10E0C00010912E09111161C0809167029091680230
:10E0D000019720915E1230915F12281739073CF4A6
:10E0E0000E94394E82E599E10E94663811E0209144
:10E0F00075023091760240917702509178026091DA
:10E10000A7077091A8078091A9079091AA070F947B
:10E1100085316B017C0120E030E0A9010F94E633EA
:10E1200087FF04C0F7FAF094F7F8F0942091790291
:10E1300030917A0240917B0250917C02C701B60176
:10E140000F941C2B20E030E84BE354E40F94E633AB
:10E150001816ECF40E94394E83E399E10E94663868
:10E160008091A7079091A807A091A907B091AA074D
:10E170008093750290937602A0937702B093780211
:10E1800087EA97E00E94AD6104C010E0B0CF1111A2
:10E19000E7CF2AE037ED43E25CE3609149027091FA
:10E1A0004A0280914B0290914C020F941C2B6B0100
:10E1B0007C0160917F0270918002072E000C880B19
:10E1C000990B0F94BD2A9B01AC01C701B6010F94B6
:10E1D0001C2B698B7A8B8B8B9C8B8091AC0C88234E
:10E1E00009F18090F3089090F408A090F508B090A1
:10E1F000F608C090A307D090A407E090A507F09080
:10E20000A60720E030E0A901C501B4010F94B62AA9
:10E210008823D1F1A7019601C501B4010F94E6331B
:10E22000181694F1C12CD12C76018E010F5E1F4F70
:10E2300027EA37E043EA57E06FE977E08BE997E0B8
:10E240000F94450080E1EBE9F7E0A9E6B2E0019028
:10E250000D928A95E1F7A6960FB6F894DEBF0FBE31
:10E26000CDBFDF91CF911F910F91FF90EF90DF9085
:10E27000CF90BF90AF909F908F907F906F905F9066
:10E280004F903F902F9008952091690230916A023B
:10E2900040916B0250916C0260919B0770919C07BA
:10E2A00080919D0790919E070F9485316D8B7E8B99
:10E2B0008F8B988F20916D0230916E0240916F028A
:10E2C0005091700260919F077091A0078091A10703
:10E2D0009091A2070F948531698F7A8F8B8F9C8FD5
:10E2E0002091710230917202409173025091740238
:10E2F000C701B6010F9485316D8F7E8F8F8F98A3E4
:10E300002091750230917602409177025091780207
:10E310006091A7077091A8078091A9079091AA071B
:10E320000F9485316B017C0120E030E0A9016D89FB
:10E330007E898F89988D0F94B62A81110CC020E0B8
:10E3400030E0A901698D7A8D8B8D9C8D0F94B62A52
:10E35000882309F467CF2D893E894F89588DCA01DA
:10E36000B9010F941C2B4B015C01298D3A8D4B8D0B
:10E370005C8DCA01B9010F941C2B9B01AC01C50136
:10E38000B4010F9486314B015C012D8D3E8D4F8D74
:10E3900058A1CA01B9010F941C2B9B01AC01C50106
:10E3A000B4010F9486314B015C01A7019601C701AE
:10E3B000B6010F941C2B9B01AC01C501B4010F9455
:10E3C00086310F9434344B015C012DEB37E346E882
:10E3D00055E30F94B62A87FF0FC020E030E0A90173
:10E3E000C701B6010F94E6334601570187FF04C009
:10E3F000B7FAB094B7F8B0942DEB37E346E855E39D
:10E40000C501B4010F94B62A87FD1CCF20E030E08F
:10E4100040EA51E4C501B4010F9480320F94F932FF
:10E420001B01672B19F422242394312CB10190E0B5
:10E4300080E00F94BB2A9B01AC0160E070E080E8B3
:10E440009FE30F9480322B013C01AC019B01C5017D
:10E45000B4010F941C2B4B015C01A30192016D8947
:10E460007E898F89988D0F941C2B6D8B7E8B8F8B63
:10E47000988FA3019201698D7A8D8B8D9C8D0F945D
:10E480001C2B698F7A8F8B8F9C8FA30192016D8DCE
:10E490007E8D8F8D98A10F941C2B6D8F7E8F8F8F0B
:10E4A00098A3A3019201C701B6010F941C2B69A385
:10E4B0007AA38BA39CA380E1E9E6F2E08E010F5FD3
:10E4C0001F4FD80101900D928A95E1F70E94C0A9D3
:10E4D0002B013C0128EC420E511C611C711C0DA348
:10E4E0001EA381E0281A310809F460C00E94C0A967
:10E4F0008B019C01041915092609370937FD59C0FC
:10E500002B013C0128EC420E511C611C711C80E067
:10E510000E94385A2D893E894F89588D69817A81A8
:10E520008B819C810F94863169837A838B839C8352
:10E53000298D3A8D4B8D5C8D6D817E818F81988583
:10E540000F9486316D837E838F8398872D8D3E8DCA
:10E550004F8D58A169857A858B859C850F9486316E
:10E5600069877A878B879C8729A13AA14BA15CA1F7
:10E570006D857E858F8598890F9486316D877E871E
:10E580008F87988B750164018E010F5E1F4F9E016E
:10E59000235F3F4FAE01475F5F4FBE016B5F7F4F11
:10E5A0008DA19EA10F94450081119BCF750164013F
:10E5B0003CCE0E94CEC4AECF8F929F92AF92BF92BC
:10E5C000CF92DF92EF92FF92CF93DF938090490238
:10E5D00090904A02A0904B02B0904C02FC01C08087
:10E5E000D180E280F38020E030E0A901C701B601CC
:10E5F0000F94B62A882341F0C0924902D0924A0271
:10E60000E0924B02F0924C02C0917F02D0918002C6
:10E6100084E690E09093800280937F02C09079021C
:10E62000D0907A02E0907B02F0907C0280E090E053
:10E63000A0E8BFE38093790290937A02A0937B02D3
:10E64000B0937C020E9429708092490290924A0203
:10E65000A0924B02B0924C02D0938002C0937F02F2
:10E66000C0927902D0927A02E0927B02F0927C0210
:10E67000DF91CF91FF90EF90DF90CF90BF90AF9060
:10E680009F908F9008950F931F93CF93DF9300D0A7
:10E690001F92CDB7DEB79C010BE917E090E1E9E6E8
:10E6A000F2E0D80101900D929A95E1F7F9012081ED
:10E6B000318142815381F80160857185828593851E
:10E6C0000F948631F801608771878287938780E095
:10E6D00090E0A0EAB0E489839A83AB83BC83CE0147
:10E6E00001960E94DC720F900F900F900F90DF91B7
:10E6F000CF911F910F9108952F923F924F925F9269
:10E700006F927F928F929F92AF92BF92CF92DF9241
:10E71000EF92FF921F93CF93DF93CDB7DEB72C9785
:10E720000FB6F894DEBF0FBECDBF7A011901DC0130
:10E730002D913D914D915C912D833E834F83588760
:10E74000FB014080518062807380809069029090CC
:10E750006A02A0906B02B0906C02A50194016D81D9
:10E760007E818F8198850F94B62A81110EC011E0A9
:10E77000A301920160916D0270916E0280916F020F
:10E78000909170020F94B62A811110E0D1012D9161
:10E790003D914D915C9129873A874B875C87F701C2
:10E7A000C080D180E280F38020910B0230910C0276
:10E7B00040910D0250910E02C701B6010F94B62A86
:10E7C000882309F44EC0C0920B02D0920C02E09252
:10E7D0000D02F0920E028091750290917602A09146
:10E7E0007702B091780240916D0250916E02609173
:10E7F0006F027091700280929B0790929C07A0928A
:10E800009D07B0929E0740939F075093A007609387
:10E81000A1077093A207C092A307D092A407E09229
:10E82000A507F092A6078093A7079093A807A09347
:10E83000A907B093AA0720E030E040E05FE36091D1
:10E84000DD0C7091DE0C8091DF0C9091E00C0F9448
:10E850001C2B69837A838B839C83CE0101960E9453
:10E86000DC722D813E814F81588520939B07309328
:10E870009C0740939D0750939E0740929F0750929C
:10E88000A0076092A1077092A207D1012D913D913E
:10E890004D915C916091A7077091A8078091A9079D
:10E8A0009091AA070F9486316093A7077093A807E9
:10E8B0008093A9079093AA0711112FC020E030E0A0
:10E8C000A90169857A858B859C850F94B62A81116B
:10E8D00033C060E070E088EC92E469837A838B83D4
:10E8E0009C83CE0101960E94DC722C960FB6F894A0
:10E8F000DEBF0FBECDBFDF91CF911F91FF90EF9094
:10E90000DF90CF90BF90AF909F908F907F906F904F
:10E910005F904F903F902F9008952AEF3EE74AE294
:10E920005FE36091E10C7091E20C8091E30C9091B7
:10E93000E40C0F941C2BD1CF60E070E080EA91E4EE
:10E94000CCCF0F931F93CF93DF9300D000D01F92B3
:10E950001F92CDB7DEB78B01FC0123A5211102C0A8
:10E960000F94FB1D1D821E821F82188620E030E05E
:10E9700040E05FE3609171027091720280917302D6
:10E98000909174020F94863169837A838B839C8380
:10E990009E012B5F3F4FAE014F5F5F4F6DE672E010
:10E9A00089E692E00E947C731D821E821F82188677
:10E9B00020E030E040E05FE3F8016085718582850A
:10E9C00093850F94863169837A838B839C83B80106
:10E9D0006C5F7F4F9E012B5F3F4FAE014F5F5F4FDC
:10E9E000C8010E947C7328960FB6F894DEBF0FBE54
:10E9F000CDBFDF91CF911F910F9108959B01AC0185
:10EA0000485F5F4FBC016C5F7F4F0C947C732F920B
:10EA10003F924F925F926F927F928F929F92AF92AE
:10EA2000BF92CF92DF92EF92FF920F931F93CF93FB
:10EA3000DF93CDB7DEB7A6970FB6F894DEBF0FBE53
:10EA4000CDBF8C011B015A874987409069025090C5
:10EA50006A0260906B0270906C0280906D029090E0
:10EA60006E02A0906F02B0907002DB018D919D91BB
:10EA70000D90BC91A02D8B8B9C8BAD8BBE8B9C0184
:10EA8000AD01C301B2010F9485316B017C01D1014D
:10EA900014968D919D910D90BC91A02D8F8B988F88
:10EAA000A98FBA8F9C01AD01C501B4010F948531C6
:10EAB0006B8F7C8F8D8F9E8FA985BA858D919D914F
:10EAC0000D90BC91A02D8B879C87AD87BE879C0144
:10EAD000AD01C301B2010F9485316F8F78A389A373
:10EAE0009AA3A985BA8514968D919D910D90BC919C
:10EAF000A02D8F87988BA98BBA8B9C01AD01C50186
:10EB0000B4010F9485316BA37CA38DA39EA3A701B1
:10EB10009601C701B6010F941C2B6B017C012B8D54
:10EB20003C8D4D8D5E8DCA01B9010F941C2B9B014C
:10EB3000AC01C701B6010F9486314B015C012B89F2
:10EB40003C894D895E896B857C858D859E850F947A
:10EB500085312B013C012F89388D498D5A8D6F8568
:10EB6000788989899A890F9485316B017C01A30189
:10EB70009201C301B2010F941C2B2B013C01A70190
:10EB80009601C701B6010F941C2B9B01AC01C30178
:10EB9000B2010F9486310F9434346B017C012F8DB8
:10EBA00038A149A15AA1CA01B9010F941C2B2B010C
:10EBB0003C012BA13CA14DA15EA1CA01B9010F945A
:10EBC0001C2B9B01AC01C301B2010F9486319B0148
:10EBD000AC01C501B4010F94E6331816B4F520E07A
:10EBE00030E0A901C701B6010F94E63387FF2AC0C0
:10EBF000C701B601905820E030E040EA50E40F949D
:10EC0000E633181614F5A10169857A85C8010E94BA
:10EC10000775A6960FB6F894DEBF0FBECDBFDF9185
:10EC2000CF911F910F91FF90EF90DF90CF90BF9009
:10EC3000AF909F908F907F906F905F904F903F909C
:10EC40002F900895C701B601D6CF20E030E040E014
:10EC500050E4C501B4010F94E633181624F4B10151
:10EC6000C8010E94A17419821A821B821C82BE01F3
:10EC70006F5F7F4FC1010E94FE742DEC3CEC4CECA9
:10EC80005CE3C701B6010F941C2B9B01AC01F8019A
:10EC900060817181828193810F941C2B6D837E83AF
:10ECA0008F839887D8019B968C919B978823C9F076
:10ECB0002AE939E949E95FE314966D917D918D91D7
:10ECC0009C9117970F941C2B69837A838B839C8369
:10ECD000BE016F5F7F4F8BE997E00E94FE74F801E1
:10ECE00013A6BE016B5F7F4F89859A850E94FE74D3
:10ECF00090CF3F924F925F926F927F928F929F92AE
:10ED0000AF92BF92CF92DF92EF92FF920F931F9339
:10ED1000CF93DF93CDB7DEB76C970FB6F894DEBF15
:10ED20000FBECDBFDB010C91142F100F153008F072
:10ED300067C11196DC90C22ECD0CB4E0BC1508F46E
:10ED40005FC1ED2DF0E0E65EFA4F8080912CB12C92
:10ED5000A12C002E04C0B694A794979487940A948B
:10ED6000D2F780FE4DC1EC2DF0E0E65EFA4F8080D8
:10ED7000912CB12CA12C012E04C0B694A794979489
:10ED800087940A94D2F780FE3BC1322E642F7C0117
:10ED90004090ED055090EE056090EF057090F00505
:10EDA0008091F5059091F605A091F705B091F805D1
:10EDB000898F9A8FAB8FBC8F660F770B072E000C55
:10EDC000880B990B0F94BD2A4B015C01602F000F3B
:10EDD000770B880B990B0F94BD2A298D3A8D4B8D9B
:10EDE0005C8D0F941C2BA30192010F948631A50119
:10EDF00094010F9486316D877E878F87988B612F62
:10EE0000110F770B880B990B0F94BD2A298D3A8D22
:10EE10004B8D5C8D0F941C2BA30192010F948631B6
:10EE2000A50194010F94853169837A838B839C8338
:10EE30004090F1055090F2056090F3057090F40554
:10EE40008091F9059091FA05A091FB05B091FC0520
:10EE5000898F9A8FAB8FBC8F632D660F770B072E30
:10EE6000000C880B990B0F94BD2A4B015C016D2D92
:10EE7000DD0C770B880B990B0F94BD2A298D3A8DE9
:10EE80004B8D5C8D0F941C2BA30192010F94863146
:10EE9000A50194010F948631698B7A8B8B8B9C8BA7
:10EEA0006C2DCC0C770B880B990B0F94BD2A298DF8
:10EEB0003A8D4B8D5C8D0F941C2BA30192010F9406
:10EEC0008631A50194010F9485316D837E838F83F4
:10EED0009887F70180859185A285B38589879A8770
:10EEE000AB87BC878D8B9E8BAF8BB88F47E651E08D
:10EEF00061E070E0CE0141960E948CC447E651E08B
:10EF000061E070E0CE0105960E948CC447E651E0B6
:10EF100061E070E0CE010D960E948CC447E651E09E
:10EF200061E070E0CE0101960E948CC489889A88C5
:10EF3000AB88BC8827E137EB41ED58EBC501B40144
:10EF40000F94E63387FD5CC023E030E044EB53E4EC
:10EF5000C501B4010F94B62A18160CF451C08D8463
:10EF60009E84AF84B88827E137EB41ED58EBC501AB
:10EF7000B4010F94E63387FD43C023E030E044EB57
:10EF800053E4C501B4010F94B62A1816CCF18D8054
:10EF90009E80AF80B88427E137EB41ED58EBC50187
:10EFA000B4010F94E63387FD2BC023E030E044EB3F
:10EFB00053E4C501B4010F94B62A18160CF18980E8
:10EFC0009A80AB80BC8027E137EB41ED58EBC5015F
:10EFD000B4010F94E63387FD13C023E030E044EB27
:10EFE00053E4C501B4010F94B62A18164CF0AE01D3
:10EFF0004F5F5F4FBE01635F7F4FC7010E94077580
:10F000006C960FB6F894DEBF0FBECDBFDF91CF91E7
:10F010001F910F91FF90EF90DF90CF90BF90AF9036
:10F020009F908F907F906F905F904F903F9008954A
:10F030002F923F924F925F926F927F928F929F9208
:10F04000AF92BF92CF92DF92EF92FF920F931F93F6
:10F05000CF93DF93CDB7DEB7CC58D1090FB6F89474
:10F06000DEBF0FBECDBF80E19CE00E94663887E026
:10F070000E94494E81116EC084E50E949D1E882326
:10F0800029F00E94902481110E94FCBC80E090E055
:10F09000A0E8BFE389839A83AB83BC838D839E837F
:10F0A000AF83B8878DEC9CECACE4BEE389879A878C
:10F0B000AB87BC8780E090E0A0E2B1E48D879E87BB
:10F0C000AF87B88B8CE390E09A8B898B8DEC90E0C6
:10F0D0009C8B8B8B8DEC9CECACECBEE38D8B9E8B78
:10F0E000AF8BB88F80E090E0A0EEBFE3898F9A8F5E
:10F0F000AB8FBC8F1BA61CA64AE959E969E97EE3E0
:10F100008FE40E94CD246D8F7E8F8F8F98A360E057
:10F1100083E40E947B2489A360E08BE40E947B242B
:10F120008AA382E40E949D1E882381F10E9490247C
:10F13000009761F19C01285231092536310520F1F3
:10F140006CE870E082EE9BE00E9464418DED9BE0F4
:10F150000E946638C457DF4F0FB6F894DEBF0FBE6B
:10F16000CDBFDF91CF911F910F91FF90EF90DF9076
:10F17000CF90BF90AF909F908F907F906F905F9057
:10F180004F903F902F9008959A8B898B8CE40E942A
:10F190009D1E8823E1F00E94A3246B017C01C98697
:10F1A000DA86EB86FC8620E030E0A9010F94E63396
:10F1B00087FD0AC020E030E040E050E4C701B6011E
:10F1C0000F94B62A18161CF485EB9BE0C1CF81E59D
:10F1D0000E944F1E882331F18091230590912405D0
:10F1E000892BE9F00E94A3246B017C01CD82DE8291
:10F1F000EF82F8862DEC3CEC4CE45DE30F94E633B3
:10F2000087FD0AC020E030E040E751E4C701B601C5
:10F210000F94B62A181634F484E89BE099CF89E558
:10F220009BE096CF83E50E949D1E8823E9F00E9413
:10F23000A3246B017C01CD8ADE8AEF8AF88E2DEC47
:10F240003CEC4CEC5DE30F94E63387FD0AC020E014
:10F2500030E040E050E4C701B6010F94B62A18161A
:10F260001CF482E39BE074CF80E50E944F1E88234C
:10F2700041F18091230590912405892B19F48AEF9F
:10F280009AE066CF8BA58F5F8BA70E94A3246B01AA
:10F290007C01CD86DE86EF86F88A20E030E0A90189
:10F2A0000F94E63387FD0AC020E030E048EC51E4DB
:10F2B000C701B6010F94B62A18161CF482ED9AE025
:10F2C00047CF86E40E949D1E8823E9F00E94A32474
:10F2D0006B017C01C98EDA8EEB8EFC8E20E030E073
:10F2E00040E85FE30F94E63387FD0AC020E030E09A
:10F2F00040E850E4C701B6010F94B62A18161CF472
:10F3000089EA9AE025CFC98CDA8CEB8CFC8C8D884D
:10F310009E88AF88B88CA7019601C701B6010F94EB
:10F320001C2B9B01AC0160E070E084E490E40F943E
:10F33000803229813A814B815C810F941C2B2B01F7
:10F340003C01A5019401C501B4010F941C2BA70138
:10F3500096010F941C2B2CEE31E548EB5DE30F94E6
:10F3600080329B01AC01C301B2010F941C2B698355
:10F370007A838B839C8388E40E949D1E882379F086
:10F380000E949024009759F09C01255A31092F3092
:10F39000314018F08BE79AE0DBCE9C8B8B8B85E5B8
:10F3A0000E944F1E8823C9F00E94C0A961157105F3
:10F3B0008105910511F00F943C26809123059091D1
:10F3C0002405892B91F00E94A32460931F0570935C
:10F3D0002005809321059093220582E50E944F1E0F
:10F3E000811108C087E49AE0B3CE60E070E088E461
:10F3F00092E4EBCF8091230590912405892B61F055
:10F400000E949024AD969FAF8EAFAD971816190647
:10F410004CF083E19AE09CCE8AE190E0AD969FAFFC
:10F420008EAFAD9789E50E949D1E882381F10E94D1
:10F43000A3242091FB083091FC084091FD085091D5
:10F44000FE080F9485316B017C0188E50E949D1EAA
:10F45000882331F10E94A3242091F7083091F80805
:10F460004091F9085091FA080F9485316BA37CA361
:10F470008DA39EA3CFA2D8A6E9A6FAA6CE01839615
:10F480000E940E1E811115C089EE99E061CEC090D8
:10F490006D02D0906E02E0906F02F0907002D5CFB6
:10F4A0006091690270916A0280916B0290916C0286
:10F4B000DDCF84E40E944F1E91E089270E94856978
:10F4C00080E090E0A0EAB0E48DA79EA7AFA7B8AB1C
:10F4D00060E0CE018D960E943F6590912008CD5747
:10F4E000DF4F9883C358D040109220080E94081C18
:10F4F00088EC99E00E94663889899A898A31910559
:10F500000CF044C08B899C890E94251F61E080E03B
:10F510000E949CBF811142C06FEF8DED99E00E9467
:10F52000D43F8CA5811104C0CE0101960F94FB1D20
:10F5300080E090E0A0EAB0E48093A3079093A40752
:10F54000A093A507B093A6071DA61EA61FA618AADE
:10F55000BE01635D7F4F8BE997E00E94FE74CD573B
:10F56000DF4F5881C358D040509320080E94081C98
:10F570008AA18111EFCD1092F6111092F5110E941F
:10F5800054C190E080E00E94251FE4CD0E946322D8
:10F5900081E00E9425BE8111B5CFBECF10927502C9
:10F5A00010927602109277021092780285E792E02C
:10F5B0000E94AD618BA5882309F452C020E030E0A1
:10F5C00040E751E46091E10C7091E20C8091E30C12
:10F5D0009091E40C0F9480326DA77EA78FA798AB13
:10F5E00080E1E9E6F2E0ABE9B7E001900D928A959F
:10F5F000E1F72D853E854F8558896091A707709169
:10F60000A8078091A9079091AA070F94863160936B
:10F61000A7077093A8078093A9079093AA07CE0124
:10F620008D960E94DC722D853E854F8558896091AC
:10F63000A7077091A8078091A9079091AA070F9436
:10F6400085316093A7077093A8078093A9079093CB
:10F65000AA078CA5811104C0CE0101960F94FB1D51
:10F66000EAE1F5E085E0DF011D928A95E9F780E1A6
:10F67000E9E6F2E0ABE9B7E001900D928A95E1F797
:10F6800089859A85AB85BC858093A3079093A40751
:10F69000A093A507B093A6071DA61EA61FA618AA8D
:10F6A000BE01635D7F4F8BE997E00E94FE74BE014F
:10F6B000635E7F4F8BE997E00E94FE7489A18823E7
:10F6C00009F41CC42091690230916A0240916B02D6
:10F6D00050916C02E5962CAF3DAF4EAF5FAFE59712
:10F6E00080916D0290916E02A0916F02B0917002B4
:10F6F000E1968CAF9DAFAEAFBFAFE197312C212C1F
:10F700009FEFA4969FAFA497AFEFA896AFAFA8972F
:10F71000BFEFC158DF4FB883CF57D040EFE4C05898
:10F72000DF4FE883C058D040F3ECCF57DF4FF8836A
:10F73000C158D04027E4CE57DF4F2883C258D0406D
:10F7400081E090E0A0E0B0E0022C04C0880F991F97
:10F75000AA1FBB1F0A94D2F7CC57DF4F8883998327
:10F76000AA83BB83C458D040AAE1B5E0E796BFAFF7
:10F77000AEAFE79710E000E09101032C000C440BC2
:10F78000550BC857DF4F288339834A835B83C8589A
:10F79000D040C457DF4F2882CC58D040E796AEAD5A
:10F7A000BFADE7978D91E796BFAFAEAFE79790E01B
:10F7B000B0E0A0E0CC57DF4F288139814A815B81DE
:10F7C000C458D04082239323A423B523892B8A2BAA
:10F7D0008B2B09F024C1C857DF4F688179818A815A
:10F7E0009B81C858D0400F94BD2A2091F5053091D7
:10F7F000F6054091F7055091F8050F941C2B2091C8
:10F80000ED053091EE054091EF055091F0050F9414
:10F810008631EB966CAF7DAF8EAF9FAFEB97B801A3
:10F82000012E000C880B990B0F94BD2A2091F9052D
:10F830003091FA054091FB055091FC050F941C2B6B
:10F840002091F1053091F2054091F3055091F405B6
:10F850000F9486316B017C01EB962CAD3DAD4EAD26
:10F860005FADEB97E5966CAD7DAD8EAD9FADE59749
:10F870000F9485312B013C01A7019601E1966CADF7
:10F880007DAD8EAD9FADE1970F9485314B015C014D
:10F89000A3019201C301B2010F941C2B2B013C0167
:10F8A000A5019401C501B4010F941C2B9B01AC016F
:10F8B000C301B2010F9486310F9434344B015C01C3
:10F8C000EB962CAD3DAD4EAD5FADEB976BA17CA142
:10F8D0008DA19EA10F9485312B013C01A7019601BA
:10F8E0006FA178A589A59AA50F9485316B017C013C
:10F8F000A3019201C301B2010F941C2B2B013C0107
:10F90000A7019601C701B6010F941C2B9B01AC0106
:10F91000C301B2010F9486310F94343420E030E0FB
:10F9200040E751E40F948032A50194010F94863191
:10F930006B017C0180901F0590902005A09021050F
:10F94000B090220520E030E040E85FE3C501B4015B
:10F950000F94E6331816F4F4C501B4010F94F23293
:10F960004B015C0160E070E0CB01181419041A042B
:10F970001B0434F40F94ED25A50194010F941C3160
:10F980000F94BD2A9B01AC01B601C7010F948631CB
:10F990006B017C01C158DF4F2881CF57D040C05840
:10F9A000DF4F3881C058D040CF57DF4F4881C15812
:10F9B000D040CE57DF4F5881C258D040B601C70162
:10F9C0000F94B62A87FF2BC0A4960FAFA497C457F5
:10F9D000DF4F3881CC58D040A8963FAFA897EC961F
:10F9E000CFAEEC97ED96DFAEED97EE96EFAEEE97DD
:10F9F000EF96FFAEEF97C158DF4FC882CF57D04088
:10FA0000C058DF4FD882C058D040CF57DF4FE88270
:10FA1000C158D040CE57DF4FF882C258D0400F5F58
:10FA20001F4F0530110509F0B9CE4FEF241A340AE3
:10FA300055E02516310409F083CEA4968FADA49726
:10FA4000E82FF0E0E65EFA4F208181E090E0A0E050
:10FA5000B0E0A8960FACA89704C0880F991FAA1F02
:10FA6000BB1F0A94D2F7822B8083A8969FADA897DC
:10FA70006A969FAF6A97A496AFADA4976B96AFAF07
:10FA80006B97EC968FADEC97ED969FADED97EE965C
:10FA9000AFADEE97EF96BFADEF976F968CAF9DAF82
:10FAA000AEAFBFAF6F97A896BFADA897BF3F09F4A1
:10FAB00009C2A496EFADA497EF3F09F403C26B2FE0
:10FAC000BB0F770B880B990B0F94BD2A2091F5057E
:10FAD0003091F6054091F7055091F8050F941C2BD5
:10FAE0002091ED053091EE054091EF055091F00524
:10FAF0000F948631162F072F382E292E862F902F00
:10FB0000A32DB22D65968CAF9DAFAEAFBFAF6597FD
:10FB1000A496FFADA4976F2FFF0F770B880B990B5F
:10FB20000F94BD2A2091F9053091FA054091FB050B
:10FB30005091FC050F941C2B2091F1053091F2059A
:10FB40004091F3055091F4050F9486316B017C01CF
:10FB50006996CCAEDDAEEEAEFFAE6997CE018F5AA0
:10FB60009F4F0E940E1E882309F4B0C120E030E0B0
:10FB700040EA50E4612F702F832D922D0F9486312F
:10FB80004B015C01CB01D50121968CAF9DAFAEAF8F
:10FB9000BFAF21972596CCAEDDAEEEAEFFAE25977A
:10FBA000A8962FADA8972111E3C1A4963FADA497C5
:10FBB0003111B3C120E030E040EA50E4C701B601A2
:10FBC0000F9486316B017C01A4964FADA49744231A
:10FBD00009F4C5C1A4968FADA49784300CF0BFC1C1
:10FBE00022ED422E23E5522E2BE7622E21E4722EC7
:10FBF00021968CAC9DACAEACBFAC219725968CAD5C
:10FC00009DADAEADBFAD2597A7968CAF9DAFAEAF06
:10FC1000BFAFA7979C01AD0169966CAD7DAD8EAD70
:10FC20009FAD69970F948531AB966CAF7DAF8EAF6A
:10FC30009FAFAB97A501940165966CAD7DAD8EAD80
:10FC40009FAD65970F9485312D966CAF7DAF8EAFCC
:10FC50009FAF2D97AB962CAD3DAD4EAD5FADAB9745
:10FC600061962CAF3DAF4EAF5FAF6197A501940198
:10FC70006091690270916A0280916B0290916C02AE
:10FC80000F9485314B015C01A7962CAD3DAD4EAD77
:10FC90005FADA79760916D0270916E0280916F02C7
:10FCA000909170020F948531A7966CAF7DAF8EAFA7
:10FCB0009FAFA797812F902FA32DB22D8DA79EA721
:10FCC000AFA7B8ABC9AADAAAEBAAFCAAC984DA849E
:10FCD000EB84FC84CDAADEAAEFAAF8AE2DEC3CECB6
:10FCE0004CEC5CE3C301B2010F941C2B29813A81D7
:10FCF0004B815C810F941C2B209175023091760210
:10FD000040917702509178020F94863169AF7AAFB3
:10FD10008BAF9CAFA5019401C501B4010F941C2BBE
:10FD20004B015C01A7962CAD3DAD4EAD5FADA797E5
:10FD3000CA01B9010F941C2B9B01AC01C501B40190
:10FD40000F94863120E030E040E050E40F94E63339
:10FD50001816ACF420E030E040E05FE3C701B601E4
:10FD60000F94863129966CAF7DAF8EAF9FAF2997E8
:10FD7000BE01635C7F4FCE0101960E94A17489850C
:10FD80009A85AB85BC8529968CAF9DAFAEAFBFAFD2
:10FD90002997A3961CAE1DAE1EAE1FAEA397BE0143
:10FDA000615A7F4FCE01CD960E94FE748CA58823A8
:10FDB000C1F02AE939E949E95FE36D817E818F81EC
:10FDC00098850F941C2BA3966CAF7DAF8EAF9FAF21
:10FDD000A397BE01615A7F4F8BE997E00E94FE74A2
:10FDE0001CA6E090D90CF090DA0C0091DB0C10917D
:10FDF000DC0CA090D50CB090D60CC090D70CD09055
:10FE0000D80C9501A601B701C8010F94E633181666
:10FE100014F4750186018090490290904A02A090E6
:10FE20004B02B0904C022DEC3CEC4CEC5DE3B70186
:10FE3000C8010F941C2B6093490270934A0280936F
:10FE40004B0290934C0240E0BE01675B7F4FCE01B6
:10FE50008D960E940EC980E1E9E6F2E0ABE9B7E0D9
:10FE600001900D928A95E1F78092490290924A02A0
:10FE7000A0924B02B0924C0220E04FEFBE01675AB5
:10FE80007F4FCE0101960E94797620E041E0BE01CD
:10FE9000675A7F4FCE0101960E9479762FEF40E09E
:10FEA000BE01675A7F4FCE0101960E94797621E00C
:10FEB00040E0BE01675A7F4FCE0101960E947976DD
:10FEC0000E949C618091170D8093180DAD964EADE8
:10FED0005FADAD9741505109AD965FAF4EAFAD9755
:10FEE000452B09F419CB6A968FAD6A9787FD14CB21
:10FEF0006B968FAD6B9787FFE1CB0ECB2BA13CA10F
:10FF00004DA15EA1E5962CAF3DAF4EAF5FAFE5973B
:10FF10008FA198A5A9A5BAA5EBCB812F902FA32DD2
:10FF2000B22D21968CAF9DAFAEAFBFAF219720E031
:10FF300030E040EA50E4C701B6010F9485312596C0
:10FF40006CAF7DAF8EAF9FAF2597A4965FADA497A2
:10FF500054300CF42FCE182D092D3A2C2B2C92ED69
:10FF6000492E93E5592E9BEF692E90E4792E40CED1
:10FF7000A8969FADA89794300CF452C0A496AFAD4C
:10FF8000A497A4300CF120E030E040EA50E4612F67
:10FF9000702F832D922D0F94853121966CAF7DAFFC
:10FFA0008EAF9FAF219720E030E040EA50E4C701D8
:10FFB000B6010F9485316B017C01A496EFADA49737
:10FFC000E4300CF40DCECBCF812F902FA32DB22D8A
:10FFD00021968CAF9DAFAEAFBFAF219720E030E050
:10FFE00040EA50E4C701B6010F94863125966CAF04
:10FFF0007DAF8EAF9FAF2597A496BFADA497B111EB
:020000021000EC
:10000000D2CF20E030E040EA50E4612F702F832D02
:10001000922D0F948531162F072F382E292E9FCF22
:10002000A496FFADA497F1110DC020E030E040E2AE
:1000300051E4B401C5010F948531162F072F382ED6
:10004000292ECECDA4962FADA49724309CF020E08D
:1000500030E040E251E4B401C5010F9485312196AE
:100060006CAF7DAF8EAF9FAF2197182D092D3A2C25
:100070002B2CB6CD182D092D3A2C2B2C82ED482E89
:1000800083E5582E8BEF682E81E4782EB1CD2F9228
:100090003F924F925F926F927F928F929F92AF9218
:1000A000BF92CF92DF92EF92FF920F931F93CF9365
:1000B000DF93CDB7DEB7EE970FB6F894DEBF0FBE75
:1000C000CDBF8091AC0C888B87E50E944F1E8823A2
:1000D00009F423C120E030E0A9016091F505709199
:1000E000F6058091F7059091F8050F94B62A8111D5
:1000F00008C00E94354E8DE09DE00E94663810E0F9
:100100001FC18AE50E949D1E882339F10E94A32405
:100110002091FF0830910009409101095091020996
:100120000F9485316B017C0120E030E040E251EC1E
:10013000C701B6010F94E63387FD0AC020E030E026
:1001400040E251E4C701B6010F94B62A181674F4C0
:100150000E94354E80E09DE0D0CFC0907102D090DB
:100160007202E0907302F0907402DECF40E050E043
:1001700060EC7FE788E50E94CD242091F70830915C
:10018000F8084091F9085091FA080F9485312B0135
:100190003C0140E050E060EC7FE789E50E94CD241F
:1001A0002091FB083091FC084091FD085091FE0819
:1001B0000F9485314B015C016FEF89E40E945F244D
:1001C000182F6FEF8AE40E945F24082FA301920189
:1001D000C301B2010F94783481116EC0A50194015E
:1001E000C501B4010F947834811166C08BA19CA124
:1001F000ADA1BEA18BAB9CABADABBEAB2091ED0571
:100200003091EE054091EF055091F005C301B20128
:100210000F9485312B013C0120E030E040E05FE3AA
:100220006BA97CA98DA99EA90F941C2B9B01AC01E5
:10023000C301B2010F9486312BA93CA94DA95EA937
:100240000F9480320F94F232162F4FA058A469A455
:100250007AA42091F1053091F2054091F305509177
:10026000F405C501B4010F9485314B015C0120E018
:1002700030E040E05FE3C301B2010F941C2B9B010F
:10028000AC01C501B4010F948631A30192010F9412
:1002900080320F94F232062F812F012E000C990B21
:1002A00097FD33C005979CF5802F002E000C990B0D
:1002B00097FD2FC005977CF5153008F020CF05304D
:1002C00008F01DCF80E00E94856995E01902F001D9
:1002D0001124E00FF11D07FDFA95EE0FFF1FEE0F41
:1002E000FF1FE954F84FC082D182E282F382602F6F
:1002F000812F0F941F1A88890E9485698889882315
:1003000009F4FDCE0E94BB30FACE10E0CDCF14E050
:10031000CBCF00E0D1CF04E0CFCF8AE40E944F1EC4
:10032000182F811127C070E060E086E50E949424B8
:100330009A838983059708F18BED9CE00E946638CB
:10034000812FEE960FB6F894DEBF0FBECDBFDF91C2
:10035000CF911F910F91FF90EF90DF90CF90BF90C2
:10036000AF909F908F907F906F905F904F903F9055
:100370002F9008950E94636FC2CE60E084E40E94D3
:100380007B248F8740E050E0BA018AE50E94CD24AB
:100390006BA77CA78DA79EA740E050E86BE376E4AF
:1003A00083E50E94CD2420E030E040E752E40F9442
:1003B0008032609345027093460280934702909387
:1003C0004802E090F712F090F812D7018D909D90BE
:1003D000AD90BC9020E030E0A901C501B4010F94BC
:1003E00086316BAF7CAF8DAF9EAF20E030E040E454
:1003F00050E40F94B62A87FF06C01BAE1CAEB0E4D3
:10040000BDAFE0E4EEAF20E030E044EB53E4C501E3
:10041000B4010F948631662E7BAB8FAB98AF20E092
:1004200030E842EB53E40F94E63318163CF4612CA9
:10043000F0E8FBAB22EB2FAB33E438AFD7011496D7
:100440008D909D90AD90BC90179720E030E0A90171
:10045000C501B4010F948631D62EE72EF82E092F50
:1004600020E030E040EE51E40F94B62A87FF05C04B
:10047000D12CE12CF0EEFF2E01E420E030E044EB43
:1004800053E4C501B4010F948631B62EC72E89AF4F
:100490009AAF20E030E046EA53E40F94E6331816B2
:1004A00034F4B12CC12CB6EAB9AFE3E4EAAF88E486
:1004B0000E944F1E882309F416C20E94A3240F94A1
:1004C000F2321B0177FF02C06F5F7F4F7595679512
:1004D0007195619571096C547F4F072E000C880B44
:1004E000990B0F94BD2A762E872E982EA92E2D2D8E
:1004F0003E2D4F2D502F0F94E63318161CF4D72C99
:1005000074010A2D2BAD3CAD4DAD5EAD672D782D40
:10051000892D9A2D0F94E633181624F07BAC8CAC01
:100520009DACAEAC872D982DA92DBA2D8B8B9C8BB5
:10053000AD8BBE8B8D2D9E2DAF2DB02F8F8B988FB9
:10054000A98FBA8FB101330C880B990B0F94BD2A78
:100550001B012C01AC019B016D2D7E2D8F2D902F49
:100560000F948631D62EE72EF82E092F2B2D3C2DF9
:1005700049AD5AAD0F94B62A87FF04C0BD2CCE2CCE
:10058000F9AE0AAFA2019101672D782D892D9A2D20
:100590000F948631D62EE72EF82E092F262D3BA953
:1005A0004FA958AD0F94B62A87FF04C06D2CEBAA53
:1005B000FFAA08AF862D9BA9AFA9B8AD8B8F9C8FE2
:1005C000AD8FBE8F8B2D9C2DA9ADBAAD8F8F98A30B
:1005D000A9A3BAA3BE01695E7F4FCE0143960E94D4
:1005E0005B2E882309F4B0C1BE01615E7F4FCE014E
:1005F0004B960E945B2EE82E882309F4A5C12F8913
:10060000388D498D5A8D6F8D78A189A19AA10F944B
:10061000853120E030E040E85EE30F941C2B4B0175
:100620005C012B893C894D895E896B8D7C8D8D8D1C
:100630009E8D0F94853120E030E040E85EE30F941A
:100640001C2B6BA37CA38DA39EA38FA298A6A9A607
:10065000BAA689819A811816190674F489EA9CE071
:100660000E9466388F85882321F08FE99CE00E94E4
:1006700066388AE00E942D380E949C610E94E41C2A
:1006800080E00E94856980E090E0A0E2B1E48FA75D
:1006900098ABA9ABBAAB60E0CE018F960E943F65E4
:1006A0002091F5053091F6054091F7055091F80538
:1006B0006BA17CA18DA19EA10F94B62A811130C09F
:1006C0002091F9053091FA054091FB055091FC0508
:1006D0006FA178A589A59AA50F94B62A811120C08B
:1006E0002091ED053091EE054091EF055091F00518
:1006F0006B897C898D899E890F94B62A811110C0DF
:100700002091F1053091F2054091F3055091F405E7
:100710006F89788D898D9A8D0F94B62A8823A9F0D8
:100720000E94636F88E0FE01B396A5EFB5E00190EB
:100730000D928A95E1F788E0FE017396ADEEB5E083
:1007400001900D928A95E1F7188A60E085E40E9495
:100750007B24882309F4FBC0F1E0FBAB1B861C86DD
:100760001D861E861A8A9E2C4FE6C42E4CE0D42E7F
:100770005DE7A52E5CE0B52E1A8915300CF0F7C0A8
:100780006B857C858D859E859B01AC010F947834AB
:100790008111EDC0992009F4DDC031E03FAB35E0B7
:1007A000232E91E09926F12EFF0CFF0CF10EF3940D
:1007B000898B19896A89121509F4D5C0062E000C97
:1007C000770B880B990B0F94BD2A2FA138A549A54B
:1007D0005AA50F941C2B2F89388D498D5A8D0F9453
:1007E00086312B013C01612F110F770B880B990B80
:1007F0000F94BD2A2BA13CA14DA15EA10F941C2BEF
:100800002B893C894D895E890F9486316B837C836B
:100810008D839E834F82588669867A8689819A81E4
:10082000892B79F06F2D8BE89CE00E943A4169E1B9
:1008300070E089E89CE00E94644186E89CE00E94A8
:1008400066381F9299E19F931F92FF92DF92CF9299
:10085000BF92AF921F920F944A1B29814BA9BE01F0
:10086000695F7F4FCE0103960F940E1C2B013C0154
:100870004B865C866D867E860FB6F894DEBF0FBE13
:10088000CDBFAC019B010F947834811169C0898878
:100890003A8825E0382D320380011124030D111D03
:1008A00037FC1A95000F111F000F111F0954184F24
:1008B000A30192016BA57CA58DA59EA50F94863101
:1008C000D8016D937D938D939C931397632D882D01
:1008D0000F941F1A188A81E00E94385AF39489896C
:1008E000BFA98B0F65CF4D2D5E2D6F2D702F86E428
:1008F0000E94CD241B012C014BAD5CAD6DAD7EADD6
:100900008CE40E94CD246B8B7C8B8D8B9E8B2F8AED
:10091000388E498E5A8E4B2D5C2D69AD7AAD82E4AE
:100920000E94CD246B017C01462D5BA96FA978AD97
:1009300082E50E94CD246B8F7C8F8D8F9E8FCF8E12
:10094000D8A2E9A2FAA246CE8FEB9CE0F7CC22E037
:100950002BAB04CF8FEF8FAB22242A9484E021CFDE
:1009600088890E9485698A898F5F8A8B05CF0E945A
:10097000B4ED0E941566882359F088890E94856924
:1009800080E090E0A0ECBFE78B879C87AD87BE87B7
:100990006B857C858D859E859B01AC010F94783499
:1009A000811159C08F85811126C082E0F82E02E0A6
:1009B00094E0C92E12E0DC2CD11A21E041E0612F35
:1009C000802F0E947C2221E04FEF612F8F2D0E940B
:1009D0007C222FEF41E06D2D802F0E947C222FEF93
:1009E0004FEF6D2D8F2D0E947C22115020F701506A
:1009F000F3940F3FF9F60E94AB400E94AA1E8F8528
:100A0000811124C081E792E00E94941D4B015C019A
:100A100089E692E00E943A1F9B01AC01C501B40136
:100A20000F941C2B9B01AC016091710270917202BA
:100A300080917302909174020F94853160937102DA
:100A40007093720280937302909374028F85811168
:100A5000E888E092AC0C0E94CB1C8091AC0C811118
:100A60000E94072B0E94FF670E94BB306B857C852C
:100A70008D859E8511E09B01AC010F947834811126
:100A80005FCC3DCB8F929F92AF92BF92CF92DF927D
:100A9000EF92FF920F931F93CF93DF9300D01F929B
:100AA000CDB7DEB75C016B017A01122F0023E1F1B3
:100AB0000E94394E88E999E00E94663861E0812FF2
:100AC0000E945A3A9090340583E08093340581E087
:100AD0008093AA0C0E94514082E08093041240E36C
:100AE00068E879E084E799E00E94564040E069E1D7
:100AF00071E18DE699E00E94564061E088E699E058
:100B00000E9438408AE799E00E9438228091AA0C1E
:100B1000882341F060E0812F0E945A3A81E00E94D0
:100B2000385AF4CF9092340520E030E0A901F50165
:100B300060817181828193810F94B62A882371F03C
:100B400080E090E0A0ECB0E489839A83AB83BC831F
:100B5000BE016F5F7F4FC5010E94C56820E030E095
:100B6000A901F60160817181828193810F94B62A77
:100B7000882351F18090E90C9090EA0CA090EB0C46
:100B8000B090EC0C80E090E0A0E7B1E48093E90C39
:100B90009093EA0CA093EB0CB093EC0C80E090E007
:100BA000A0EAB1E489839A83AB83BC83BE016F5F03
:100BB0007F4FC6010E94C5688092E90C9092EA0CB2
:100BC000A092EB0CB092EC0C20E030E0A901F70110
:100BD00060817181828193810F94E633181674F4D9
:100BE00080E090E0A0E4B0E489839A83AB83BC8387
:100BF000BE016F5F7F4FC7010E94C56880910905E4
:100C000029E131E1882311F029E439E047E559E091
:100C100061E679E081E00E9479400E94514081E0E4
:100C20000F900F900F900F90DF91CF911F910F9128
:100C3000FF90EF90DF90CF90BF90AF909F908F90FC
:100C40000895CF93C82F8091690C83FD14C08091C3
:100C50002E09811110C080916702909168029C0159
:100C6000215031094091601250916112421753078F
:100C700014F40E94251FCC2329F061E080E0CF917D
:100C80000C949CBF80912E0991E0892780934402A7
:100C900080914402882389F080915E1290915F12C6
:100CA0002091601230916112821B930B97FF03C059
:100CB000919581959109029744F410924402809194
:100CC000690C83FF06C0C1E01AC080E00E94385A58
:100CD000DFCFC0912E09C11112C08091670290919F
:100CE000680201972091601230916112281739072C
:100CF00054F70E94394E8BE299E00E9466388C2F9F
:100D0000CF910895AF92BF92CF92DF92EF92FF9270
:100D10000F931F93CF93DF93CDB7DEB764970FB6D2
:100D2000F894DEBF0FBECDBF0E94384F87FDAFC025
:100D30008AE50E949D1E882309F4BAC040E050E075
:100D4000BA018AE50E94CD247B018C0120917102B9
:100D500030917202409173025091740260E070E031
:100D600088EC93E40F9485315B016C019701A80135
:100D70000F94E633181614F07501860120E030E078
:100D8000A901B701C8010F94E633181624F4E12C29
:100D9000F12C00E010E0B701C8010F94F232072EE9
:100DA000000C880B990B0F94BD2A698B7A8B8B8B67
:100DB0009C8B20E030E0A9010F94B62A882321F013
:100DC000CE0141960E94437380E090E0A0EAB1E436
:100DD0008D879E87AF87B88B19861A861B861C86DF
:100DE0008CE40E944F1E882309F467C00E94A3244C
:100DF0006B017C0120E030E0A901C701B6010F942E
:100E0000E63387FF04C0F7FAF094F7F8F094CD8248
:100E1000DE82EF82F88620916012309161122430D8
:100E2000310574F080915E1290915F12821B930BDA
:100E300097FF03C091958195910901E004970CF407
:100E400000E080E00E942186882359F022E0AE0174
:100E5000435F5F4FBE016B5F7F4FCE0109960E94DB
:100E6000428569897A898B899C898B019C013058DC
:100E700009831A832B833C8320E030E0A9010F947F
:100E8000B62A882321F0CE0101960E94437364960E
:100E90000FB6F894DEBF0FBECDBFDF91CF911F918B
:100EA0000F91FF90EF90DF90CF90BF90AF9008959B
:100EB000E12CF12C00E211E449CFC090E805D0907C
:100EC000E905E090EA05F090EB0594CF7F928F92D0
:100ED0009F92AF92BF92CF92DF92EF92FF920F93C9
:100EE0001F93CF93DF9300D000D01F921F92CDB7F6
:100EF000DEB76C015B014A01722E78010091350664
:100F00000E94311F80916012909161128E159F0591
:100F10001CF4C7010E94251F80E00E9421868823BF
:100F200031F0272DA401B501C6010E9442851E148F
:100F30001F043CF4C7010E94251F60E080E00E946E
:100F40009CBF81E00E94218680E090E0A0E7B2E4AF
:100F500089839A83AB83BC8380E090E0A0E8B0EC07
:100F60008D839E83AF83B887BE016F5F7F4FCE01B5
:100F700005960E94C56887E00E941E2A811158C00C
:100F80008091710290917202A0917302B0917402EB
:100F900040910E0550910F0560911005709111055B
:100FA000C0900A05D0900B05E0900C05F0900D055F
:100FB000C0929B07D0929C07E0929D07F0929E07FB
:100FC00040939F075093A0076093A1077093A207D7
:100FD0008093A3079093A407A093A507B093A607B7
:100FE00080E090E0A8E4B2E489839A83AB83BC8379
:100FF000CE0101960E94DC7280911205909113053A
:10100000A0911405B09115058093A3079093A407B0
:10101000A093A507B093A60780E090E0A0EAB0E413
:1010200089839A83AB83BC83CE0101960E94DC72D4
:10103000C12CD12C80E7E82E82E4F82EC982DA8216
:10104000EB82FC8280E090E0A0E8B0E48D839E8398
:10105000AF83B887BE016F5F7F4FCE0105960E94B8
:10106000C56820E030E0A901609116057091170570
:1010700080911805909119050F94B62A87FF0BC02F
:10108000C982DA82EB82FC82BE016F5F7F4F86E10C
:1010900095E00E94C5688091160590911705A09172
:1010A0001805B09119058093750290937602A0936C
:1010B0007702B09378028093A7079093A807A09334
:1010C000A907B093AA0787EA97E00E94AD618091D3
:1010D000EC0581110F94651961E087EB99E00E949E
:1010E000A13F8091961181508093961148E958E173
:1010F0006FEB79E085E00E94C2EB80919611882326
:1011000039F00E94D5AD809196118150809396114F
:1011100080E00F942C1B0E94B53180919711823092
:1011200011F40E9474380E94B4ED28960FB6F8941A
:10113000DEBF0FBECDBFDF91CF911F910F91FF900A
:10114000EF90DF90CF90BF90AF909F908F907F9067
:101150000895CF92DF92EF92FF920F931F93CF9358
:10116000DF9300D01F92CDB7DEB77C016B018A01FF
:1011700061E08CE399E00E94A13F48E958E163E413
:1011800079E085E00E94C2EB9091961181E0890F91
:10119000809396118091B41482FF06C08B7F809358
:1011A000B4149E5F909396110E94663980E1E9E63F
:1011B000F2E0AAE0B5E001900D928A95E1F70E9475
:1011C0009C6181E00F942C1B20E030E0A901F70125
:1011D00060817181828193810F94B62A8823F1F016
:1011E00080912E0981110CC0809167029091680254
:1011F000019720915E1230915F122817390774F021
:1012000080E090E0A0E7B2E489839A83AB83BC835B
:10121000BE016F5F7F4FC7010E94C56887E00E94D3
:101220001E2A811103C0B6010E94196820E030E037
:10123000A901F80160817181828193810F94B62A9E
:10124000882341F080E00E942186882319F0C8019C
:101250000E94F568129A64E670E080E090E00E94D7
:10126000112681E00F900F900F900F90DF91CF919A
:101270001F910F91FF90EF90DF90CF900895CF9244
:10128000DF92EF92FF92CF93DF936B017C01D42F1B
:10129000C091340583E08093340581E08093AA0CEB
:1012A000C114D104E104F10431F00E94C0A9C60EBA
:1012B000D71EE81EF91E8091AA0C882389F0C1145C
:1012C000D104E104F10421F48D2F0E94385AF3CFA8
:1012D0000E94C0A96C197D098E099F0997FDF4CF62
:1012E0001092AA0CC0933405DF91CF91FF90EF903C
:1012F000DF90CF9008950F931F93CF93DF93C82F64
:10130000162F0E94394EC11194C0CFE8D8E0CE010B
:101310000E94663861E0812F0E945A3A0E94C0A95B
:10132000685370458F4F9F4F60933106709332061C
:10133000809333069093340610923506009134055D
:1013400083E08093340530E020E049E151E16DE134
:1013500079E082E00E9479408DE199E00E94382294
:1013600081E08093AA0C8091AA0C882309F464C0C0
:1013700060E0812F0E945A3A80913506882309F453
:1013800054C00E94394E83E099E00E94663830E0F4
:1013900020E04DEE58E064EF78E082E00E94794072
:1013A00084EF98E00E94382241E060E070E0CB01D9
:1013B0000E943F8930E020E050E040E060EE78E0BD
:1013C00085E00E94794080EE98E00E94BC350E9442
:1013D000311F80E00E9421860E94394ECE010E947A
:1013E00066380E94C0A9685370458F4F9F4F609325
:1013F0003106709332068093330690933406109230
:10140000350630E020E049E151E164ED78E082E02A
:101410000E94794083EC98E00E94382281E080931A
:10142000AA0C61E0812F0E945A3A81E00E94385A4A
:101430009ACFC4EAD8E06BCF00933405DF91CF9107
:101440001F910F910895CF92DF92EF92FF920F9329
:101450001F93CF93DF93CDB7DEB7A0970FB6F89465
:10146000DEBF0FBECDBF0E94384F87FDCCC085E4E4
:101470000E944F1E882309F4D5C00E94A3246B014B
:101480007C0120E030E0A9010F94E63387FF04C01F
:10149000F7FAF094F7F8F094F7FAF094F7F8F0947C
:1014A000CD8EDE8EEF8EF8A28CE0EEEDF2E0DE0166
:1014B000119601900D928A95E1F78AE50E949D1E92
:1014C000882351F040E050E0BA018AE50E94CD2423
:1014D00069877A878B879C8788E50E949D1E882371
:1014E00051F040E050E0BA0188E50E94CD246983C4
:1014F0007A838B839C8389E50E949D1E882351F00B
:1015000040E050E0BA0189E50E94CD246D837E83DE
:101510008F83988785E50E944F1E882309F489C030
:101520000E94A3246B017C0120E030E0A901C701E7
:10153000B6010F94E63387FF04C0F7FAF094F7F88A
:10154000F094F7FAF094F7F8F094C98EDA8EEB8EF7
:10155000FC8E1D8A1E8A1F8A188E8CE40E944F1EE4
:10156000882309F46FC00E94A3246B017C0120E052
:1015700030E0A901C701B6010F94E63387FF04C02C
:10158000F7FAF094F7F8F094C98ADA8AEB8AFC8AC1
:1015900062E070E082E40E949424F82E809196111B
:1015A000811131C021E0AE01475E5F4FBE016F5F28
:1015B0007F4FCE014D960E94A988882321F16F2D7F
:1015C00081E00E947B8982E50E949D1E882309F4A8
:1015D00042C00E94902440E050E060EA71E44D87F0
:1015E0005E876F87788B20919611222361F08C01A2
:1015F0002F2DAE01435F5F4FBE016F5E7F4FCE0167
:1016000045960E946687A0960FB6F894DEBF0FBE7F
:10161000CDBFDF91CF911F910F91FF90EF90DF90A1
:10162000CF900895C12CD12C80E8E82E80E4F82ECC
:1016300033CFC090E405D090E505E090E605F0904A
:10164000E70572CFC090E805D090E905E090EA0583
:10165000F090EB058CCF90E080E0BDCFCF92DF9291
:10166000EF92FF920F931F93CF93DF93CDB7DEB727
:101670006C970FB6F894DEBF0FBECDBF8CE40E940E
:101680004F1E882309F4B0C00E94A3246B017C0183
:1016900020E030E0A9010F94E63387FF04C0F7FA99
:1016A000F094F7F8F094F7FAF094F7F8F094C98E04
:1016B000DA8EEB8EFC8E8CE0EEEDF2E0DE01119620
:1016C00001900D928A95E1F788E50E949D1E88237E
:1016D000A1F040E050E0BA0188E50E94CD242091BD
:1016E000F7083091F8084091F9085091FA080F94E2
:1016F000853169837A838B839C8389E50E949D1E53
:101700008823A1F040E050E0BA0189E50E94CD2491
:101710002091F7083091F8084091F9085091FA08A3
:101720000F9485316D837E838F8398878AE50E942D
:101730009D1E882351F040E050E0BA018AE50E94E6
:10174000CD2469877A878B879C871D861E861F8696
:10175000188A80919611811138C020E0AE01435F54
:101760005F4FBE016F5F7F4FCE0149960E94A988EF
:10177000882359F18091EC0581110F94651960E07F
:1017800080E00E947B89898D9A8DAB8DBC8DB0588D
:101790008D8B9E8BAF8BB88F198A1A8A1B8A1C8AF5
:1017A0001D861E861F86188A80919611882369F0EF
:1017B00010E000E020E0AE014B5E5F4FBE016F5EC7
:1017C0007F4FCE010D960E9466876C960FB6F894F7
:1017D000DEBF0FBECDBFDF91CF911F910F91FF9064
:1017E000EF90DF90CF900895C12CD12C80E8E82EA7
:1017F00080E4F82E58CF2F923F924F925F926F92D3
:101800007F928F929F92AF92BF92CF92DF92EF9290
:10181000FF920F931F93CF93DF93CDB7DEB7E5977A
:101820000FB6F894DEBF0FBECDBF8DAB209134054F
:101830002CAB81E080933405809152058D3409F4FE
:10184000C6C4843511F40C945AA0873409F091C1B0
:1018500080915005909151058B31910509F4DDC1BE
:1018600008F079C18430910508F030C12091080753
:101870008230910508F48EC1213009F091C111E048
:10188000029709F010E00E94E42419821A821B8258
:101890001C821D821E821F82188682E50E949D1E68
:1018A000882309F490C10E94A3246B017C0120E0ED
:1018B00030E0A9010F94B62A882309F4EAC04090C9
:1018C000690250906A0260906B0270906C02809185
:1018D0006D0290916E02A0916F02B09170028CA780
:1018E0009DA7AEA7BFA780909B0790909C07A09054
:1018F0009D07B0909E0780919F079091A007A091AF
:10190000A107B091A20788AB99ABAAABBBABA5016D
:101910009401C301B2010F94B62A81110DC028A908
:1019200039A94AA95BA96CA57DA58EA59FA50F9491
:10193000B62A882309F4ADC0A3019201C501B40100
:101940000F94853120E030E040E05FE30F941C2BE2
:1019500068A779A78AA79BA72CA53DA54EA55FA53B
:1019600068A979A98AA99BA90F94853120E030E064
:1019700040E05FE30F941C2B2B013C0120E030E0A2
:10198000A901C701B6010F94B62A881F8827881FAE
:10199000181709F40FC180E090E0A0E8BFEB8CA716
:1019A0009DA7AEA7BFA728A539A54AA55BA5CA01D3
:1019B000B9010F941C2B4B015C01A3019201C301DF
:1019C000B2010F941C2B9B01AC01C501B4010F9413
:1019D00086310F9434344B015C01AC019B01C7018B
:1019E000B6010F94853168AB79AB8AAB9BABA5018F
:1019F0009401C701B6010F9486319B01AC0168A91F
:101A000079A98AA99BA90F941C2B6B017C0120E06A
:101A100030E0A9010F94E63387FDD1C0C701B601BC
:101A20000F9434346B017C01C301B2019058A501BD
:101A300094010F9480322CA53DA54EA55FA50F946F
:101A40001C2BA70196010F941C2B28A539A54AA58C
:101A50005BA50F94863169837A838B839C83A50170
:101A6000940168A579A58AA59BA50F9480322CA521
:101A70003DA54EA55FA50F941C2BA70196010F94C1
:101A80001C2BA30192010F9486316D837E838F837B
:101A9000988720E030E0A90169817A818B819C815F
:101AA0000F94B62A8111A3C020E030E0A9016D8116
:101AB0007E818F8198850F94B62A811198C00E94EB
:101AC000354E8BEB9FE00E9466386AC085319105E8
:101AD00009F466C08A31910509F49CC0049709F0A5
:101AE00048C080E50E949D1EC12CD12C7601882320
:101AF00021F00E941D246B017C0183E50E949D1E44
:101B0000882361F00E94A32420E030E04AE754E4F7
:101B10000F941C2B0F94F9326B017C010E949C6185
:101B200080919811811105C060E081ED9FE00E94D5
:101B3000D43F0E94C0A9C60ED71EE81EF91E0E94FF
:101B4000C0A96C197D098E099F0997FF29C080E003
:101B50000E94385AF4CF8A32910509F4ADC160F47D
:101B60008D31910509F4D6C008F470C04E9709F480
:101B700029C10F94D11B14C08B35910509F47FC284
:101B80008C35910509F47FC28A35910591F7109241
:101B90001B0806C0213021F40E94E4240E94297011
:101BA0003DA9311102C00F947E1B8CA9809334058E
:101BB0000C947C9880E090E0A0E8BFE3F0CEC12CCC
:101BC000D12C760131CF89E40E949D1E882331F00B
:101BD0000E94A32469837A838B839C838AE40E9476
:101BE0009D1E882309F455CF0E94A3244ECF412F78
:101BF000BE016F5F7F4F8BE997E00E940EC90E9484
:101C0000C0A96093E9117093EA118093EB1190934E
